:0200000480007A
:100000006F00000413000000130000001300000044
:100010001300000013000000130000001300000094
:10002000732E2034732E3034B74E0C00370F01F08E
:10003000930F40000FF00E000FF0EF03730020301D
:10004000130E10001303F0011303F3FF0F700302EC
:10005000E31C03FE130E200037020C00B70201F070
:10006000130300000F7002000F70530237120C00D0
:10007000B70201F0130310000F7002000F7053025B
:1000800037220C00B70202F0130320000F700200A9
:100090000F70530237320C00B70202F01303300026
:1000A0000F7002000F705302130E30003702001061
:1000B000B70200C0370300C1B7030020370400C2F5
:1000C000B70400C3370500C4371611111306161103
:1000D000B726222293862622373733331307373346
:1000E0002320C200032E020003AE0200032E0300F1
:1000F00023A0D31003AE0310032E041003AE04108C
:10010000130E4000032E02002320E30003AE020082
:10011000032E0200130E5000032E0500130E600084
:10012000130E700037620C00B70200F01303F001E9
:100130000F7002000F705302130000001300000044
:10014000130000001300000013000000370200C677
:1001500067000200130000001300000013000000FD
:08016000130000001300000071
:100168001305000067800000130500006780000089
:1001780013050000678000006FF09FFE1305000064
:10018800678000001305000067800000B70710F0C3
:1001980023A0A7F067800000130101FF232481003A
:1001A800232611001304050003450500630A050012
:1001B80013041400EFF09FFD03450400E31A05FE45
:1001C8008320C1000324810013010101678000001E
:1001D800130101FF2320210123261100232481007C
:1001E8002322910013090600630E060013840500FC
:1001F800B384C5000345040013041400EFF01FF98D
:10020800E39A84FE8320C1000324810013050900BA
:1002180083244100032901001301010167800000C4
:100228006780000037150180130101FF1305C527FA
:1002380023261100EF00C0058320C100B70710F086
:1002480023A007F2130500001301010167800000D5
:10025800130101FC2324C1022326D1022328E10231
:10026800232AF102232C0103232E110313860500F0
:100278008325850093068102232E11002326D100B1
:10028800EF0040068320C1011301010467800000CC
:10029800130101FC2324C1022326D102232AF102DF
:1002A8002322B1022328E102232C0103232E110368
:1002B800973701009387078583A7070093064102B4
:1002C8001306050083A5870013850700232E110058
:1002D8002326D100EF0000018320C101130101048E
:1002E80067800000130101E32326111C2322911CBF
:1002F8002320211D232E311B2320A11B1389050038
:1003080093040600138D06002324811C232C411B13
:10031800232A511B2328611B2326711B2324811B9D
:100328002322911B232EB11993090500EF40104792
:1003380083270500138507002324F102EF60503757
:10034800232AA1002328010C232A010C232C010CA9
:10035800232E010C638A090083A78903639607008B
:1003680013850900EF2080518317C90013972701CF
:1003780063420702B726000003274906B3E7D70000
:100388002316F900B7E7FFFF9387F7FFB377F70066
:100398002322F9068357C90093F78700638E07065F
:1003A80083270901638A07068357C9001307A0003A
:1003B80093F7A7016390E7088317E90063CC070662
:1003C80093060D00138604009305090013850900A0
:1003D800EF10906F232CA1008320C11C0324811CE3
:1003E800032581018324411C0329011C8329C11B86
:1003F800032A811B832A411B032B011B832BC11A50
:10040800032C811A832C411A032D011A832DC1193B
:100418001301011D67800000930509001385090079
:10042800EF105076E30205F89307F0FF232CF10054
:100438006FF09FFA9307C10E2322F10C2326010CBB
:100448002324010C130A0000138B0700232A01023E
:10045800232801022324010023220102232601026A
:10046800232C01001384040013075002834704005F
:10047800638407006392E70CB30A9440638A0A0412
:100488008327C10C23209B0023225B01B3875701DC
:100498002326F10C8327810C13077000130B8B00A4
:1004A800938717002324F10C635EF7001306410CB1
:1004B8009305090013850900EF80101F631A05765C
:1004C800130BC10E83278101B3875701232CF10039
:1004D80083470400639407006F10505B9307140070
:1004E8002328F100A303010A930CF0FF232E010037
:1004F80013040000930B9000130CA0028327010142
:1005080083CA0700938717002328F10093870AFE00
:100518001307A0056374F7006F10C02417170100B4
:10052800130747D693972700B387E70083A70700E9
:10053800B387E70067800700130414006FF01FF308
:1005480097170100938707EF232AF1029377040294
:10055800639407006F104003130D7D00137D8DFF1A
:1005680093078D00832D0D00032D4D002326F100E8
:1005780093771400638E0700B3E7AD01638A070021
:10058800930700032304F10AA304510B1364240006
:100598001374F4BF930720006F00106913850900D6
:1005A800EF40D01F83274500138507002326F1025B
:1005B800EF6010102322A10213850900EF40101EDE
:1005C800832785002324F10083274102E38807F26B
:1005D80083278100E38407F283C70700E38007F2DB
:1005E800136404406FF09FF18347710AE39807F0A2
:1005F80093070002A303F10A6FF05FF0136414007D
:100608006FF0DFEF83270D00130D4D00232EF1004F
:10061800E3D607EEB307F040232EF100136444003D
:100628006FF0DFED9307B0026FF0DFFC8327010165
:1006380083CA0700938D170063988A05832C0D00E1
:1006480093074D0063D40C00930CF0FF138D070043
:100658002328B1016FF09FEA13850C009305A000D1
:100668002322F100EF00417C83274100938D1D0078
:1006780083CAFDFFB30CF50093870AFDE3FEFBFC7C
:100688002328B1016FF09FE8930C00006FF0DFFEA4
:10069800136404086FF09FE6832D0101232E0100E7
:1006A8000325C1019305A000938A0AFDEF00C177D5
:1006B800938D1D00B387AA0083CAFDFF232EF10086
:1006C80093870AFDE3FEFBFC6FF09FFB1364840035
:1006D8006FF0DFE28327010103C707009307800655
:1006E800631CF70083270101136404209387170014
:1006F8002328F1006FF09FE0136404046FF01FE0FB
:100708008327010103C707009307C006631CF7008E
:1007180083270101938717002328F100136404023B
:100728006FF0DFDD136404016FF05FDD93074D00A8
:100738002326F10083270D00A303010A2306F112E3
:1007480023220100930C1000930D0000130C0000ED
:10075800930B0000130D00009304C1122320B10372
:1007680063D49D01232091030347710A630807009E
:1007780083270102938717002320F102937724002F
:10078800232CF1026388070083270102938727003F
:100798002320F10293774408232EF102639C070675
:1007A8008327C101032701023387E7406354E0062A
:1007B800930E0001171E0100130E8EC3130F700055
:1007C8008326810C2320CB010326C10C93861600B7
:1007D80093058B0063D4EE006F00107A2322EB00A0
:1007E8003307C7002326E10C2324D10C130770001C
:1007F800138B05006350D7021306410C93050900BB
:1008080013850900EF80406A630405006F10D0214A
:10081800130BC10E0347710A630A07041307710A11
:100828002320EB00130710002322EB000327C10C41
:1008380093067000130B8B00130717002326E10C97
:100848000327810C130717002324E10C63D0E60269
:100858001306410C9305090013850900EF80C06455
:10086800630405006F10501C130BC10E832781030E
:10087800638A07041307810A2320EB00130720006B
:100888002322EB000327C10C93067000130B8B0087
:10089800130727002326E10C0327810C13071700F1
:1008A8002324E10C63D0E6021306410C93050900EA
:1008B80013850900EF80405F630405006F10D016B0
:1008C800130BC10E8327C10313070008639AE706B9
:1008D8008327C10103270102B387E7406352F0066B
:1008E800930E0001171E0100130E8EB1130F700036
:1008F8008326810C2320CB010327C10C9386160085
:1009080013068B00E3C6FE6C3387E7002322FB0047
:100918002326E10C2324D10C13077000130B0600C7
:100928006350D7021306410C93050900138509008B
:10093800EF808057630405006F10100F130BC10E72
:10094800B38D9D416352B007130E000117180100C3
:10095800130808AB930E70000327810C23200B01AA
:100968008326C10C1307170013068B00E34EBE6BDA
:100978002322BB01B38DDD002326B10D2324E10C16
:1009880093067000130B060063D0E6021306410CB1
:100998009305090013850900EF80005163040500E1
:1009A8006F109008130BC10E13770410832DC10C20
:1009B800E314076C8327810C3383BC0123209B003D
:1009C8009387170023229B012326610C2324F10C13
:1009D80013077000130B8B006344F7006F10801629
:1009E8001306410C9305090013850900EF80C04BDD
:1009F800630405006F105003130BC10E6F108014B1
:100A08001364040193770402638E0704130D7D00B9
:100A1800137D8DFF93078D00832D0D00032D4D0051
:100A28002326F100635E0D00B30DB041B337B0016A
:100A3800330DA041330DFD409307D002A303F10A03
:100A48009307F0FFE390FC38E3120D409307900002
:100A5800E3EEB73F938D0D03A307B1199304F11883
:100A68006F00503C93074D002326F1009377040153
:100A780063880700832D0D0013DDFD416FF09FFA99
:100A880093770404832D0D0063880700939D0D015F
:100A980093DD0D416FF05FFE93770420E38E07FC32
:100AA800939D8D0193DD8D416FF01FFD9377840039
:100AB800638C070A93074D002326F10083270D0056
:100AC80003A6070083A6470003A7870083A7C700DC
:100AD8002328C10C232AD10C232CE10C1305010D6A
:100AE800232EF10CEF40C0442326A10A93072000CF
:100AF800631CF50A8327010D9305010813050109F5
:100B08002328F1088327410D232001082322010807
:100B1800232AF1088327810D2324010823260108AD
:100B2800232CF1088327C10D232EF108EFC0D07ABA
:100B3800635605009307D002A303F10A93077004D4
:100B4800971401009384048D63C65701971401001C
:100B58009384048C1374F4F723220100930C30005F
:100B6800930D00006F00102D130D7D00137D8DFF78
:100B780083250D0003264D0093078D0013050109F9
:100B88002326F100EFF0D04F832701092328F10C29
:100B980083274109232AF10C83278109232CF10C8F
:100BA8008327C1096FF09FF3930710006318F502BC
:100BB8008327C10D63D607009307D002A303F10A68
:100BC800930770049714010093844485E3C457F98C
:100BD80097140100938444846FF0DFF793FBFAFDC8
:100BE80093071004639EFB04930700032304F10A90
:100BF80013071006930780056394EA00930780079C
:100C0800A304F10A930730061364240063D6974BB4
:100C180093851C0013850900EF40006493040500C8
:100C28006312054A8357C90093E707042316F9009E
:100C38008357C90093F70704638007FA6FF0CFFE64
:100C48009307F0FF6384FC48930770042322010094
:100C58006394FB0063820C48032AC10D9367041058
:100C68002320F102232C0102832E010D032E410DB6
:100C7800832D810D635A0A00B707008033CA4701E4
:100C88009307D002232CF10293071004639AFB48C0
:100C9800130501092328D109232AC109232CB109E5
:100CA800232E4109EFF0D0621306C10AEF50105A03
:100CB800138605009305050013050109EFF0503C64
:100CC8008327010913060106930501072328F10666
:100CD800832741091305010823200106232AF10669
:100CE800832781092322010623240106232CF106E8
:100CF8008327C109232EF106B707FC3F2326F106F7
:100D0800EFC0907303280108032641088326810851
:100D1800832DC1089305010813050109232801093A
:100D280023220105232AC1082320C104232CD1082A
:100D3800232ED102232EB1092320010823220108E2
:100D48002324010823260108EFC050368326C10357
:100D58000326010403284104631605001307100045
:100D68002326E10A13071006170C0100130C8C6CDC
:100D78006396EA00170C0100130C8C6A138EFCFFB3
:100D8800138D0400B7070340930501082322C10807
:100D980013050109130601072324C10523200109AE
:100DA8002324D1082326B109232EF106232801067E
:100DB800232A0106232C0106EFC010680326010927
:100DC8008326410983278109130501092322C104C8
:100DD8002320D104232EF102EFF0407C9305050077
:100DE800130A050013050109832DC109EFF05011FD
:100DF8008327C1030326410483260104232CF1061B
:100E0800832701092328C106930501072320F1063A
:100E18008327410913060106130501082322F10659
:100E280083278109232EB107232AD1062324F1061B
:100E38008327C109130D1D002326F106EFE0C02505
:100E4800B3054C0183C50500032E8104832EC10818
:100E580083220108832F4108032F8108232EC10311
:100E6800A30FBDFE9307F0FF938D0E00630CFE06E3
:100E7800130EFEFF9305010813050109232ED10562
:100E8800232CE105232AF105232851042326C10533
:100E98002328510823245104232AF1092322F10588
:100EA800232CE1092320E105232ED1092320010861
:100EB800232201082324010823260108EFC0101F5C
:100EC800832601040326410403288104032EC10458
:100ED80083220105832F4105032F8105832EC10538
:100EE800E31205EAB70DFE3F930501081305010952
:100EF8002328510823265104232AF1092324F10524
:100F0800232CE1092322E105232ED1092320D10531
:100F18002320010823220108232401082326B109DC
:100F2800EFC090256346A0048322C104832F810467
:100F3800032F4104832E01049305010813050109B9
:100F480023285108232AF109232CE109232ED1094A
:100F58002320010823220108232401082326B1099C
:100F6800EFC0D0146314051A137A1A0063000A1A22
:100F78000346FC00232EA10B930500038326C10B17
:100F88009387F6FF232EF10A83C7F6FF638CC714F5
:100F980013069003639CC7148347AC00A38FF6FE27
:100FA800130A0D0013077004330A9A40032DC10A6F
:100FB8006396EB2A1307D0FF6344ED0063D2AC338A
:100FC800938AEAFF930BFDFF2326710B93F6FAFD34
:100FD8009305100413F7FA0F130600006398B60080
:100FE8001307F7001377F70F13061000230AE10A17
:100FF8009307B00263D80B00930B1000B38BAB417F
:101008009307D002A30AF10A9307900063DC7729BB
:10101800130C310C930D0C00930C90009305A00059
:1010280013850B00EFF0D06A13050503A30FACFE80
:101038009305A00013850B00EFF05061130DFCFF22
:10104800930B050063C2AC24930B0503130CECFF50
:10105800A30F7DFF9307610B636CBC231307410B40
:10106800B387E7402328F102B38C470193071000A8
:1010780063C64701937714006386070083274101FD
:10108800B38CFC001374F4BF936704102320F1029F
:10109800130C0000930B0000130D0000832781033D
:1010A800638607001307D002A303E10A03240102A1
:1010B800930D00006FF08FEA232201009304C11200
:1010C8006FF09FB92322A1006FF01FB923220100FE
:1010D800930C60006FF05FB823229101930C10000D
:1010E8006FF09FB7A38FB6FE6FF05FE99387170085
:1010F80093F7F70F6FF09FEA130A1A00A30FEAFE9F
:10110800B3074D41E3DA07FE6FF0DFE98327C10338
:10111800130A0D0013070003330DFD006FF05FFE87
:1011280093076004638EFB0093075004138C1C0024
:101138006384FB00138C0C00130620006F00C000B2
:10114800138C0C00130630009307010B1308C10B16
:101158001307C10A93060C009305010913850900BA
:101168002328D1092320D105232AC109232EC1030D
:10117800232CB109232E4109EF304017930770043F
:1011880093040500032EC103832E01046396FB001C
:10119800937714006384070A93076004338D8401EE
:1011A8006392FB0603C70400930700036318F70460
:1011B80093050108130501092328D1092320D10526
:1011C800232AC109232EC103232CB109232E410947
:1011D80023200108232201082324010823260108CB
:1011E800EFC0C06C032EC103832E01046308050001
:1011F80093071000338C87412326810B8327C10A6C
:10120800330DFD0093050108130501092328D109B1
:10121800232AC109232CB109232E410923200108BF
:10122800232201082324010823260108EFC00068AF
:1012380013070003631E0500232EA10B032AC10B0D
:101248006FF05FD693861700232ED10A2380E7001C
:101258008327C10BE3E8A7FF6FF05FFE1307600465
:10126800E392EBD66352A00763960C001377140041
:101278006302070C832741013307FD00B38CEC00A0
:10128800930A60066F004009130C0D006FF01FD918
:10129800130C1C000347FCFF93871700A38FE7FE7E
:1012A8006FF09FDB1307610B6318060093070003B9
:1012B800230BF10A1307710B938B0B03930717008A
:1012C800230077016FF09FD963960C001377140001
:1012D8006306070683274101138717006FF01FFA7B
:1012E80063404D0313771400930C0D006306070049
:1012F80083274101B30CFD00930A70066F00C001FB
:1013080083274101930A7006B30CFA006346A001D3
:101318003383AC41930C1300937B0440130C0000FF
:10132800E38E0BD6930B0000E35AA0D79306F00F79
:101338006F008003930C0D006FF09FF4930A600612
:10134800930C10006FF05FFD6356A703832781009D
:10135800330DED4003C71700630807029387170092
:10136800938B1B002324F1008327810003C7070008
:10137800E31CD7FC8325410233858B01EFF0D02A8B
:10138800B30C95016FF09FD1130C1C006FF0DFFDBB
:1013980013074D002326E1001377040283270D006D
:1013A800630007020327810123A0E7001357F741D1
:1013B80023A2E700032DC100832401016FF08F8A67
:1013C80013770401630807000327810123A0E700BE
:1013D8006FF05FFE13770404630807000357810169
:1013E8002390E7006FF01FFD13740420E30E04FC44
:1013F800034781012380E7006FF0DFFB13640401DA
:101408009377040263880704130D7D00137D8DFF15
:1014180093078D00832D0D00032D4D002326F10029
:101428001374F4BF93070000A303010A1307F0FF26
:101438006380EC1A13070400B3E6AD011374F4F7E4
:101448006398061863820C30130710006396E71838
:101458006FF04FE093074D002326F10093770401C6
:1014680063860700832D0D006F0000019377040445
:1014780063880700835D0D00130D00006FF05FFAAD
:1014880093770420E38007FE834D0D006FF0DFFEA5
:1014980093074D002326F100B787FFFF93C7078303
:1014A8002314F10A97070100938787F7832D0D000E
:1014B800232AF102130D000013642400930720006F
:1014C800930A80076FF05FF693074D002326F1001B
:1014D800A303010A9307F0FF83240D006384FC0231
:1014E80013860C009305000013850400EF40404963
:1014F8002322A100630605E6B30C954023220100D0
:101508006FF00FE613850400EF50901A930C050056
:101518006FF0DFFE1364040193770402638207020D
:10152800130D7D00137D8DFF93078D00832D0D0016
:10153800032D4D002326F100930710006FF0DFEE16
:1015480093074D002326F100937704016386070073
:10155800832D0D006F000001937704046388070052
:10156800835D0D00130D00006FF01FFD93770420BD
:10157800E38007FE834D0D006FF0DFFE9707010043
:10158800938707EA6FE05FFC93074D002326F1007D
:101598009377040163860700832D0D006F00000117
:1015A8009377040463880700835D0D00130D000022
:1015B8006FE01FFC93770420E38007FE834D0D0046
:1015C8006FF0DFFE13070400930710006FF0DFE6EB
:1015D80013071000638AE7C613072000638AE7121F
:1015E800930701199316DD0113F77D0093DD3D0084
:1015F80013070703B3EDB601135D3D00A38FE7FEA4
:10160800B3E6AD019384F7FF639E06029376140058
:10161800638A0600930600036306D700A38FD4FEEF
:101628009384E7FF93070119938D0C00232201008F
:10163800B38C9740130C0000930B0000130D0000AF
:101648006FF0CF91938704006FF0DFF913770440B0
:10165800130A0000930701192322E100930BF00FEE
:10166800130C90001306A0009306000013850D00CC
:1016780093050D009384F7FF2320F102EFA0106378
:101688008327010213050503130A1A00A38FA7FE77
:1016980083274100638807048327810083C70700E5
:1016A8006312FA0463007A0563140D00637CBC03BB
:1016B800832741028325C102130A0000B384F44042
:1016C8001386070013850400EF505000832781001C
:1016D80083C7170063880700832781009387170053
:1016E8002324F10013850D0093050D001306A000B7
:1016F80093060000EFA0C07D138D0500B3E5A5009B
:10170800930D0500E38005F2938704006FF09FF5C1
:10171800930401190327410393F7FD009384F4FF11
:10172800B307F70083C7070093DD4D002380F4005B
:101738009317CD01B3EDB701135D4D00B3E7AD01CC
:10174800E39A07FC6FF01FEE93040119E39C07EC82
:1017580013771700E30807EC93070003A307F118B2
:101768006FF0CFAFE3840A3223065113A303010AB3
:101778002326A1016FE0DFFC130606012322DB010B
:101788002326C10C2324D10C635EDF021306410C0F
:1017980093050900138509002326E1052324C105C3
:1017A8002322D1052320E104EF700070E31E0526F3
:1017B800032FC104032E8104832E4104032701044F
:1017C8009305C10E130707FF138B05006FE05FFF3A
:1017D800130707012322DB012326E10C2324D10C64
:1017E800635EDF021306410C9305090013850900A7
:1017F8002322E1052320C105232ED103232CF10246
:10180800EF70806AE3120522032F4104032E0104BE
:10181800832EC103832781031306C10E938707FF15
:10182800130B06006FF0CF8C938606012322CB01A1
:101838002326D10C2324E10C63DAEE021306410CB3
:1018480093050900138509002320D105232E0103E0
:10185800232CC103EF704065E318051C832E010497
:101868000328C103032E81031306C10E938D0DFFB8
:10187800130B06006FF04F8E13075006635257750F
:101888000327010D93050108130501092328E10821
:101898000327410D2320010823220108232AE108F8
:1018A8000327810D2324010823260108232CE1089E
:1018B8000327C10D232EE108EFB0507F631C0512EA
:1018C80097070100938747B82320FB009307100070
:1018D8002322FB008327810C938D1D002326B10D45
:1018E800938717002324F10C13077000130B8B0048
:1018F800635EF7001306410C930509001385090080
:10190800EF70805AE3120512130BC10E8327C10A28
:1019180063C64701937714006386072283278102F1
:1019280003274101130B8B00232CFBFE8327410166
:10193800232EFBFE8327C10CB387E7002326F10C77
:101948008327810C13077000938717002324F10C59
:10195800635EF7001306410C93050900138509001F
:10196800EF708054E312050C130BC10E9304FAFFB9
:10197800635A901C930B0001970A0100938A4AA8A6
:10198800130C70008327810C23205B010327C10CF3
:101998009387170093068B0063C29B0223229B0048
:1019A800B384E4002326910C2324F10C1307700060
:1019B800138B06006358F7186FF08F82130707011F
:1019C80023227B012326E10C2324F10C635EFC0017
:1019D8001306410C9305090013850900EF70C04CEC
:1019E800E31405049306C10E938404FF138B0600C9
:1019F8006FF05FF90327C10A634CE01C97070100E9
:101A0800938787A42320FB00930710002322FB0061
:101A18008327810C938D1D002326B10D9387170012
:101A28002324F10C13077000130B8B00635EF7007F
:101A38001306410C9305090013850900EF70C04691
:101A48006314057E130BC10E8327C10A6398070030
:101A580063160A00937714006386070E83278102B2
:101A68000327410193088B002320FB0083274101B2
:101A78002322FB008327C10CB387E7002326F10C40
:101A88008327810C13077000938717002324F10C18
:101A9800635EF7001306410C9305090013850900DE
:101AA800EF708040631205789308C10E832AC10A3B
:101AB80063D20A06B30A504113870800130C0001C9
:101AC800970B0100938BCB93930D70008327810CA8
:101AD800232077018326C10C9387170093888800F9
:101AE800634C5C0B23225701B38ADA002326510D7D
:101AF8002324F10C13077000635EF7001306410CF2
:101B08009305090013850900EF70003A631E0570FC
:101B18009308C10E8327C10C23A0980023A2480173
:101B2800B38747012326F10C8327810C1307700024
:101B3800138B8800938717002324F10C6354F70054
:101B48006FE01FEA1374440063100468832AC1011C
:101B58008327010263D4FA00938A0700832781014F
:101B6800B3875701232CF1008327C10C638C07002E
:101B78001306410C9305090013850900EF70C03264
:101B88006314056A832741002324010C6398076EB8
:101B9800130BC10E6FF01F82938606012322870163
:101BA8002326D10C2324F10C63DEFD001306410C1F
:101BB8009305090013850900EF70002F6316056669
:101BC8009308C10E938A0AFF138708006FF01FF06D
:101BD800930A0D006354AA01930A0A006352500540
:101BE8000327810CB38DBA0123209B00130717002C
:101BF80023225B012326B10D2324E10C93067000F8
:101C0800130B8B0063DEE6001306410C93050900F5
:101C180013850900EF70402963180560130BC10E86
:101C280063D40A00930A0000B30A5D416350500769
:101C3800930C000197FD0000938D8D7C13037000B9
:101C48000327810C2320BB018326C10C130717002F
:101C580013068B0063C25C1B23225B01B38ADA0084
:101C68002326510D2324E10C93067000130B060064
:101C780063DEE6001306410C93050900138509008D
:101C8800EF7080226312055A130BC10E937704403C
:101C9800B38AA40163840702930D7000338D440155
:101CA80097FC0000938CCC7563980B1863180C187C
:101CB800B387440163F45701938A07008327C10A55
:101CC80063C6470193771400638A07048327810258
:101CD80003274101130B8B00232CFBFE83274101B3
:101CE800232EFBFE8327C10CB387E7002326F10CC4
:101CF8008327810C13077000938717002324F10CA6
:101D0800635EF7001306410C93050900138509006B
:101D1800EF708019631A0550130BC10EB384440188
:101D2800B38754418324C10AB3049A4063D497000B
:101D380093840700635490048327C10C23205B011C
:101D480023229B00B387F4002326F10C8327810C00
:101D580013077000130B8B00938717002324F10CD3
:101D6800635EF7001306410C93050900138509000B
:101D7800EF708013631A054A130BC10E9387040092
:101D880063D40400930700008324C10AB3049A4073
:101D9800B384F440E35890DA930B000197FA0000FB
:101DA800938A0A66130C70008327810C23205B0139
:101DB8000327C10C9387170093068B00E3D09BBEC3
:101DC8001307070123227B012326E10C2324F10CAE
:101DD800635EFC001306410C930509001385090096
:101DE800EF70800C631205449306C10E938404FFC0
:101DF800138B06006FF05FFB9386060123229B017D
:101E08002326D10C2324E10C6352E3021306410C70
:101E18009305090013850900232C6102EF70C0089F
:101E280063140540032381031306C10E938A0AFF36
:101E3800130B06006FF0DFE063020C0E130CFCFFBF
:101E48008327C10203274102130B8B00232CFBFEBF
:101E580083274102232EFBFE8327C10CB387E700AB
:101E68002326F10C8327810C938717002324F10C78
:101E780063DEFD001306410C930509001385090074
:101E8800EF7080026312053A130BC10E832781009D
:101E980033075D4183C707006354F70093070700C2
:101EA8006356F0040327C10C23205B012322FB00A7
:101EB8003387E7002326E10C0327810C130B8B00E3
:101EC800130717002324E10C63D2ED021306410C1B
:101ED8009305090013850900232CF102EF60D07CDB
:101EE8006314053483278103130BC10E138707007E
:101EF80063D407001307000083278100130800013B
:101F080083C70700B387E7406346F006832781004D
:101F180083C70700B38AFA006FF01FD983278100AF
:101F2800938BFBFF9387F7FF2324F1006FF05FF19A
:101F38009386060123220B012326D10C2324E10CCE
:101F480063D6ED021306410C9305090013850900B9
:101F5800232E0103232CF102EF6010756316052C64
:101F68000328C103832781031306C10E938707FF44
:101F7800130B06000327810C23209B018326C10C29
:101F88001307170013068B00E344F8FA2322FB001B
:101F9800B387D7002326F10C2324E10C130B06008A
:101FA800E3D6EDF61306410C9305090013850900E5
:101FB800EF60906F631A0526130BC10E6FF01FF5C3
:101FC8008327810C1307100023209B00938D1D008D
:101FD80093871700930B8B00634647019376140091
:101FE8006388061C130710002322EB002326B10D7B
:101FF8002324F10C13077000635EF7001306410CED
:102008009305090013850900EF60106A631E052017
:10201800930BC10E8327810203274101938B8B0009
:1020280023ACFBFE8327410123AEFBFE8327C10CB3
:10203800B387E7002326F10C8327810C1307700070
:10204800938717002324F10C635EF7001306410CF5
:102058009305090013850900EF6010656316051CD8
:10206800930BC10E8327010D930501081305010980
:102078002328F1088327410D930AFAFF232001083A
:10208800232AF1088327810D23220108232401082C
:10209800232CF1088327C10D23260108232EF108DC
:1020A800EFB0D000630605088327C10C0327810C15
:1020B800938414009387F7FFB3874701130717002A
:1020C80023A09B0023A25B012326F10C2324E10C0F
:1020D80093077000938B8B0063DEE7001306410CB7
:1020E8009305090013850900EF60105C631E051253
:1020F800930BC10E9307410B23A0FB008327010319
:1021080003270103138B8B0023A2FB008327C10C39
:10211800B387E7002326F10C8327810C130770008F
:10212800938717002324F10CE35EF7A06FE05F8B21
:10213800E35250FD130C000197F400009384442CE3
:10214800930D70000327810C23A09B008327C10CEB
:102158001307170093868B0063405C03B387FA006C
:1021680023A25B012326F10C2324E10C93077000C2
:10217800938B06006FF05FF69387070123A28B010C
:102188002326F10C2324E10C63DEED001306410C39
:102198009305090013850900EF60105163160508BF
:1021A8009306C10E938A0AFF938B06006FF09FF97E
:1021B8002322EB002326B10D2324F10C1307700012
:1021C800E35AF7F26FF09FF18327C1010327010259
:1021D8003384E740E35C8096930A000197F400009B
:1021E80093840421930B70008327810C23209B0088
:1021F8000327C10C9387170063C68A0423228B0028
:102208003304E4002326810C2324F10C1307700007
:10221800E35EF7921306410C930509001385090044
:10222800EF609048E3040592832741006394070018
:102238006FE01FA09385070013850900EF00D011F8
:102248006FE01F9F1307070123225B012326E10C80
:102258002324F10C130B8B0063DEFB001306410CE7
:102268009305090013850900EF601044E31E05FA81
:10227800130BC10E130404FF6FF01FF783254100F1
:1022880013850900EF00500D6FF09F908327C10C54
:10229800639407006FE0DF991306410C930509006A
:1022A80013850900EF6050406FE09F989717010071
:1022B8009387478593060600138605009305050056
:1022C80003A507006FE00F8283D7C500130101B88B
:1022D800232C814693F7D7FF231AF10083A74506DD
:1022E80013840500232A91462326F10683D7E500A7
:1022F80023282147232E1146231BF10083A7C5015C
:1023080013090500232001022322F10283A74502B5
:10231800930581002326F102930701072324F10086
:10232800232CF100930700402328F100232EF1000D
:10233800EFD05FFB93040500634C05009305810013
:1023480013050900EF004038630405009304F0FF0B
:102358008357410193F70704638807008357C40034
:1023680093E707042316F4008320C1470324814719
:1023780013850400032901478324414713010148B9
:1023880067800000130101FF970701009387877793
:10239800232291009304050003A50700232481004C
:1023A800232611001384050063080500832785038D
:1023B80063940700EF00804C0317C40093170701CC
:1023C80093D7070193F68700639E060693F60701E5
:1023D800639606029307900023A0F400136707048E
:1023E8002316E4001305F0FF8320C10003248100B5
:1023F80083244100130101016780000093F747001F
:10240800638C070283250403638C05009307040487
:102418006386F50013850400EF0000742328040286
:102428008357C4002322040093F7B7FD2316F40052
:10243800832704012320F4008357C40093E787000F
:102448002316F40083270401639007028357C4000E
:102458001307002093F707286388E7009305040013
:1024680013850400EF2050508357C40013F717005A
:10247800630C07028327440123240400B307F040B8
:10248800232CF4008327040113050000E39E07F4BE
:102498008317C40013F70708E30807F493E7070452
:1024A8002316F4006FF01FF493F7270013070000BA
:1024B80063940700032744012324E4006FF09FFC82
:1024C8008397C500130101FE232C81001397070190
:1024D80013570701232A9100232E110023282101D5
:1024E80023263101937687009304050013840500A1
:1024F800639C06163717000013070780B3E7E70049
:1025080003A745002396F5006346E00203A7C50329
:102518006342E002130500008320C1010324810106
:1025280083244101032901018329C1001301010208
:102538006780000003278402E30E07FC03A9040058
:102548009396370123A004008325C40163D8060CA1
:10255800032604058357C40093F74700638E0700DA
:10256800832744003306F640832704036386070065
:102578008327C4033306F640832784028325C401D6
:102588009306000013850400E78007009307F0FF17
:102598008356C4006312F50283A704001307D00111
:1025A800636CF70A37074020130717003357F70003
:1025B800137717006302070AB7F7FFFF9387F77FC0
:1025C80003270401B3F7D7009397070193D707416F
:1025D8002320E4002316F400232204001397370174
:1025E800635C07009307F0FF6316F50083A70400F8
:1025F800639407002328A4048325040323A024014B
:10260800E38A05F0930704046386F5001385040044
:10261800EF008054232804026FF0DFEF1306000058
:102628009306100013850400E70007009307F0FFE6
:1026380013060500E310F5F283A70400E38C07F006
:102648001307D0016386E700130760016392E7066A
:1026580023A024016FF01FEC93E706042316F4006F
:102668001305F0FF6FF05FEB83A90501E38409EA26
:1026780003A905001377370023A035013309394131
:10268800930700006314070083A745012324F4007F
:10269800E35220E9832744028325C40193060900F5
:1026A8001386090013850400E78007006348A0002B
:1026B8008357C40093E707046FF05FFAB389A90052
:1026C8003309A9406FF0DFFC130101FE232C8100C0
:1026D800232E110013040500630C050083278503CE
:1026E800639807002326B100EF0040198325C10035
:1026F8008397C500638C0700130504000324810138
:102708008320C101130101026FF09FDB8320C10107
:1027180003248101130500001301010267800000F2
:1027280093050500631E0500970701009387473D41
:1027380003A5070097050000938545F96F0080738E
:10274800970701009387073C03A507006FF0DFF7A1
:102758001305000067800000977500009385857653
:102768006F004071130101FF23248100232611000B
:10277800130405002316B5002317C5002320050000
:10278800232205002324050023220506232805000B
:10279800232A0500232C050013068000930500005A
:1027A8001305C505EF30002097470000938747437E
:1027B8002320F40297470000938707482322F40256
:1027C800974700009387874F2324F4029747000018
:1027D80093874754232E84002326F4028320C100C4
:1027E8000324810013010101678000001305000024
:1027F80067800000130101FF2320210113890500D0
:102808002324810093058006130405001305F9FFAE
:102818002326110023229100EFE00061930545076C
:102828009304050013050400EF201023130405008A
:102838006300050223200500232225011305C50096
:102848002324A4001386840693050000EF30801526
:10285800130504008320C100032481008324410060
:102868000329010013010101678000009707010097
:102878009387072903A507006FF01FEE83278503B9
:10288800639E0706130101FF2326110023248100FC
:1028980097070000938787EC232EF50293073000F3
:1028A8002322F52E9307C52E130405002324F52EA5
:1028B8002320052E0325450013060000930540003C
:1028C800EFF05FEA032584001306100093059000DB
:1028D800EFF05FE90325C4001306200093052001EB
:1028E800EFF05FE893071000232CF4028320C10067
:1028F8000324810013010101678000006780000044
:10290800130101FF970701009387871F2322910076
:1029180083A40700232021012326110083A7840311
:10292800232481001309050063960700138504001A
:10293800EFF0DFF49384042E03A4840083A74400FB
:102948009387F7FF63DA070083A70400638E070005
:1029580083A404006FF05FFE0317C4006304070438
:10296800130484066FF0DFFD93054000130509008A
:10297800EFF05FE823A0A400E31C05FC9307C00068
:102988002320F90013040000130504008320C1006C
:10299800032481008324410003290100130101015C
:1029A80067800000B707FFFF9387170023220406FC
:1029B8002320040023220400232404002326F400F7
:1029C80023280400232A0400232C04001306800073
:1029D800930500001305C405EF20D07C23280402CA
:1029E800232A040223220404232404046FF0DFF9B9
:1029F8006780000067800000678000006780000033
:102A0800970701009387071003A5070097050000A3
:102A1800938545D46F00003C970701009387870E84
:102A280003A5070097050000938585DC6F00803AB1
:102A3800130101FD23248102232291022320210373
:102A4800232E31012326B100232611021309050084
:102A580097090100938949CAEF30800283A789004A
:102A68008325C10083A44700B71700001384F7FE2D
:102A780093F4C4FF3304B440330494001354C400E3
:102A88001304F4FF1314C4006356F4021305090079
:102A9800EF20507F130500008320C1020324810228
:102AA80083244102032901028329C101130101037F
:102AB800678000009305000013050900EF3050748B
:102AC80083A78900B3879700E312F5FCB30580401C
:102AD80013050900EF30D0729307F0FF6312F50475
:102AE8009305000013050900EF30907103A78900D2
:102AF8009306F000B307E540E3DAF6F8970601001D
:102B08009386860083A6060093E717002322F70022
:102B18003305D5409706010023A6A6006FF01FF7DE
:102B280083A78900B384844093E4140023A2970008
:102B380097070100938707FF83A70700130509007C
:102B4800338487409707010023AE87FCEF209073FA
:102B5800130510006FF05FF4638C0526130101FF65
:102B68002324810023229100130405009384050087
:102B780023261100EF20D07083A5C4FF938684FF1D
:102B880017050100130545B793F7E5FF3386F600EF
:102B9800032746000328850093F515001377C7FF20
:102BA800631AC806B387E7006390050203A784FF8A
:102BB800B386E64003A68600B387E70003A7C600EE
:102BC8002326E6002324C70013E7170023A2E60004
:102BD800170701002326D7B217070100130707F3C9
:102BE8000327070063ECE70097070100938707F3C3
:102BF80083A5070013050400EFF09FE31305040005
:102C0800032481008320C1008324410013010101B2
:102C18006F2050672322E600130800006396050220
:102C280083A584FF97080100938888ADB386B640D2
:102C3800B387B70083A58600638C150B83A8C600ED
:102C480023A6150123A4B800B305E60083A5450013
:102C580093F51500639C0502B387E70003278600F8
:102C6800631C080897050100938585A96316B708B2
:102C780017060100232CD6A8170601002326D6A87C
:102C880023A6E60023A4E6001308100013E71700A4
:102C980023A2E6003387F6002320F700E31008F6A6
:102CA8001307F01F6362F70693D7370013D6274040
:102CB800130710003317C700032645009387170032
:102CC800939737003367C700B307F500170601006D
:102CD8002326E6A203A70700138687FF23A6C600BC
:102CE80023A4E60023A0D7002326D7006FF01FF106
:102CF800130810006FF05FF50326C6002326C700EF
:102D08002324E6006FF09FF813D6970013074000BE
:102D1800636AC70413D767001307870313061700EE
:102D2800131636003306C500930586FF03260600F2
:102D38006396C50893071000135727403397E70099
:102D4800832745003367F7009707010023A8E79A10
:102D580023A6B60023A4C60023A4D5002326D600A4
:102D68006FF0DFE9130740016366C7001307B60574
:102D78006FF0DFFA130740056368C70013D7C70071
:102D88001307E7066FF09FF9130740156368C7003C
:102D980013D7F700130777076FF05FF893054055CF
:102DA8001307E007E3ECC5F613D727011307C70796
:102DB8006FF0DFF6032686006388C5000327460008
:102DC8001377C7FFE3E8E7FE8325C6006FF05FF8D7
:102DD80067800000130101FD2324810223202103C1
:102DE800232C4101232A5101232611022322910277
:102DF800232E31011304052E13090000130A1000B5
:102E0800930AF0FF631604028320C102032481029F
:102E18001305090083244102032901028329C10102
:102E2800032A8101832A41011301010367800000FD
:102E380083248400832944009389F9FF63D6090019
:102E4800032404006FF01FFC83D7C4006370FA02E8
:102E58008397E400638C5701138504002326B1008F
:102E6800E78005008325C1003369A900938484069F
:102E78006FF09FFC130101FD23248102232021030D
:102E8800232C4101232A51012328610123267101A2
:102E98002326110223229102232E3101130A050051
:102EA800938A05001304052E13090000130B100064
:102EB800930BF0FF631A04028320C10203248102EA
:102EC8001305090083244102032901028329C10152
:102ED800032A8101832A4101032B0101832BC100AD
:102EE80013010103678000008324840083294400C0
:102EF8009389F9FF63D60900032404006FF09FFB50
:102F080083D7C400637EFB008397E400638A77015C
:102F18009385040013050A00E7800A003369A900B5
:102F2800938484066FF0DFFC9307450113052500A1
:102F3800231F05FEE31CF5FE67800000930745018B
:102F4800130525000357E5FF93852500239FE5FE1C
:102F5800E398A7FE678000009307A50113052500E5
:102F6800231F05FEE31CF5FE67800000130785019B
:102F780093870500130525008356E5FF93872700EF
:102F8800239FD7FEE318A7FE239C05006780000057
:102F980093074500938545001305A50193872700EE
:102FA8009385250083D6E7FF03D7E5FF6398E600FE
:102FB800E316F5FE130500006780000013051000F6
:102FC8006364D7001305F0FF67800000930645008F
:102FD800930700001305A5013786FFFF03D70600F6
:102FE800937517006384050093E7170093F527008E
:102FF8001357170063900502939717002390E60074
:10300800939707019386260093D70701E318D5FC09
:10301800678000003367C7006FF01FFE93066501E5
:103028001307000083D7260013960701135606419D
:1030380063540600136717009397170093970701C7
:103048001376270093D7070163100602131717009A
:103058002391F600131707019386E6FF135707011C
:10306800E312D5FC6780000093E717006FF01FFE9E
:1030780093074500130700001305A50183D6070031
:103088009387270013D686003367C700239FE7FE80
:10309800139786001317070113570701E310F5FE6E
:1030A80067800000930765011307000083D6270097
:1030B8009387E7FF139686003367C7002392E700DC
:1030C80013D78600E314F5FE6780000093074500D8
:1030D800130785019387270083D60700239FD7FE10
:1030E800E31AF7FE231C050067800000930785019B
:1030F8001307A501930645009387E7FF03D607004A
:103108001307E7FF2310C700E398F6FE2312050014
:103118006780000093858501130765019306000009
:103128008357270003D605001307E7FF9385E5FFBC
:10313800B387C700B387D7002391F50093D707015A
:1031480093F61700E31EE5FC678000009385850170
:10315800130765019306000083D70500035627006F
:103168001307E7FF9385E5FFB387C740B387D740C9
:103178002391F50093D7070193F61700E31EE5FCAA
:1031880067800000130101FB232E3103B7090100FA
:10319800232481042322910423202105232C410385
:1031A80023261104130A0500231501022316010220
:1031B80093848501138945001304C1029389F9FF9B
:1031C80003D504001304E4FF9384E4FF63180504A3
:1031D800231F04FEE31699FE930740001307A0017E
:1031E80093054101B385F50083D50500B306F600C4
:1031F800938727002390B600E394E7FE8320C10459
:103208000324810483244104032901048329C1037D
:10321800032A8103130101056780000093050A0052
:103228002326C100EFD0504003572400B37735015F
:1032380013550501B387E700035704002311F40071
:1032480093D707013305E5003305F5002310A400E3
:1032580013550501231FA4FE0326C1006FF09FF735
:103268008357250193C7F7FF13971701631C0700BE
:1032780093072501130525000357E5FF6318070089
:10328800E39AA7FE130500006780000013051000ED
:1032980067800000130101FF232481002326110009
:1032A80013040500EFF0DFFB631E0500031524017E
:1032B8001355F5018320C100032481001301010186
:1032C80067800000130500006FF0DFFE83172501FB
:1032D800130101FF232611002324810023229100DA
:1032E8002320210163D807069307F0FF2390F500F8
:1032F80003572501B78700009387F7FF33F7E700E7
:103308002391E500130905016316F70613840500E8
:1033180093040500EFF0DFF46302050493076400EB
:10332800231204001385C4FF1309E9FF035729007A
:1033380093872700239FE7FEE318A9FE8320C10097
:1033480003248100832441000329010013010101A2
:1033580067800000239005006FF09FF993074400F1
:103368009305A40193872700239F07FEE39CB7FEDC
:103378006FF0DFFC93876500239205001305E5FFD6
:103388001309E9FF0357290093872700239FE7FEC6
:10339800E318A9FE239C05006FF05FFA130101FBF7
:1033A80023229104232021052326110423248104A8
:1033B8001309050093840500EFF09FEA6310050EDA
:1033C80013850400EFF0DFE9130405006318050C0A
:1033D8009305810013050900EFF05FEF93054102A3
:1033E80013850400EFF09FEE0357810083574102D5
:1033F8006380E70693072000930680011306810087
:103408003306F60003560600631C06021306410243
:103418003306F60003560600631406029387270056
:10342800E39ED7FC130504008320C1040324810410
:103438008324410403290104130101056780000066
:1034480013041000E30007FE1304F0FF6FF09FFD64
:1034580013061000638407001306F0FF93070000AB
:1034680093058001130781003307F700835607008F
:10347800130741023307F700035707006398E60074
:1034880093872700E390B7FE6FF0DFF91304060077
:10349800E36AD7F83304C0406FF0DFF81304E0FFA5
:1034A8006FF05FF88357250193C7F7FF139717014C
:1034B80063100702130101FF23261100EFF05FDA02
:1034C8008320C10013351500130101016780000036
:1034D80013050000678000009307250113052500E8
:1034E800231F05FEE31CF5FE835705003787000000
:1034F8001307F7FFB3E7E7002310F5006780000024
:10350800130101FE232C810023282101232E110001
:10351800232A91002326310123244101232251012A
:10352800130905001384050063D20510330AB0405F
:1035380093090A0093040000930AF00063CE3A034B
:1035480013554A00930500FFEFD0100E3304854051
:1035580093090400130A7000634C3A0313553400AE
:10356800930580FFEFD0500C33048500631E0402DE
:10357800333590006F00400983578901130509000E
:10358800938909FFB3E4F400EFF05FB66FF01FFB17
:103598008347890113050900938989FFB3E49700DC
:1035A800EFF01FAD6FF05FFB83578901130509002A
:1035B8001304F4FF93F71700B3E49700EFF01FA18B
:1035C8006FF0DFFA13050900EFF05FB0938404FF92
:1035D800E3CA99FE13554400930500FFEFD0D004C9
:1035E8003304A400930404009309700063C699048B
:1035F80013553400930580FFEFD010033304A40063
:1036080063140404130500008320C101032481010D
:1036180083244101032901018329C100032A810070
:10362800832A41001301010267800000938405008A
:103638009309F0006FF0DFF913050900EFF09FA67A
:10364800938484FF6FF09FFA13050900EFF01F9D24
:103658001304F4FF6FF0DFFA83574500130101FFED
:1036680023229100232611002324810023202101F5
:10367800930405006392070883176500130400008C
:103688001309000A63D80702130504008320C10048
:10369800032481008324410003290100130101014F
:1036A800678000001385040013040401EFF01FA2D3
:1036B800E30C24FD83D76400E38607FE83D7640008
:1036C80093F707F0638207021309000A83976400DF
:1036D800E3CC07FA1385040013041400EFF01F94D9
:1036E800E35689FE6FF05FFA13850400EFF09F9BA5
:1036F800130484006FF09FFC93F707F01304000095
:1037080063860700EFF0DF96130480FF130900F7C4
:103718006F004001138504001304F4FFEFF01F8BC2
:10372800E34424F783D74400E39607FE6FF0DFF500
:103738009307050113052500231F05FEE31CF5FE6D
:10374800B7C7FFFF2310F500B787FFFF93C7F7FF41
:103758002311F50067800000130705008356070052
:10376800138505008357270063860600B786FFFF89
:10377800B3E7D7002319F50003562700B7860000E2
:103788009386F6FF93076700631ED6001307A70109
:1037980083D607006398060293872700E39AE7FE1B
:1037A8006FF09FD31305050113078701938727003F
:1037B80083D6E7FF1305E5FF2311D500E398E7FE5D
:1037C800678000006FF0DFF6130101FD23229102EC
:1037D80093040500130541002324810223261102C6
:1037E80013840500EFF04FF703D7E40093170701A0
:1037F80093D7074163C2070423120100B78600006C
:103808009386F6FF3377D7009387E400631CD706C7
:103818001387040083560700638606021305040015
:10382800EFF01FF18320C1020324810283244102A7
:1038380013010103678000009307F0FF2312F100D2
:103848006FF0DFFB13072700E396E7FC130504007E
:10385800EFF08FED13050400EFF01FC88397E40025
:10386800E3D207FC13050400EFF09F9FE31C05FA61
:10387800835724013787FFFFB3C7E7002319F400F4
:103888006FF05FFA2313E100930641009387E7FF87
:1038980003D60700938626002392C600E398F4FE19
:1038A800631C07002314010093050400130541005D
:1038B800EFF09FEA6FF01FF7930710009305F0FFF2
:1038C800130541002314F100EFF09FC36FF0DFFDF3
:1038D800130101FE232C8100232A910023282101B2
:1038E8002326310123244101232251011389060093
:1038F80013840700232E1100930405009389050003
:10390800130A0600930A0700EFF01FD59307000972
:103918003309A94063D4A704B78700009387E7FF5A
:1039280063C6272D938724009384A40193872700D7
:10393800239F07FEE39C97FE8320C1010324810196
:1039480083244101032901018329C100032A81003D
:10395800832A41001301010267800000635E0900A9
:10396800930700F7634CF9129305090013850400C7
:10397800EFF01FB96310051463860A220327440079
:10398800832704006306F7061305A401EFF0CFDCD4
:103998008327440013078003638EE7166340F712FA
:1039A800130780016386E71A130750036382E71839
:1039B8001307C0002324E400370701801307F7FF2B
:1039C800232AE40013071000231CE4001307B000A7
:1039D8002326E4000327C4008356840113078700C5
:1039E800131717003307E4002315D7002320F4002A
:1039F800634220030327440093070009630CF70080
:103A080083D784011385040093F71700B3E9F900FD
:103A1800EFF0CFDB8326840003564401832544005E
:103A2800139716003387E40083570700B3F7C700DE
:103A38001306F008634AB6009386160013060700BB
:103A48009305C00063DAD510835644010356070076
:103A580093C6F6FFB3F6C6002310D70003576401D8
:103A6800B376F700638A06106312F70263940910AD
:103A78008327C4000357840193971700B387F40082
:103A880083D70700B3F7E7006388070E9385040020
:103A98001305A401EFF00FE86F00000E93872400D0
:103AA8009384A40193872700239F07FEE39C97FE36
:103AB8006FF09FE8930910006FF01FEC13070004E4
:103AC8006388E70213071007E394E7EE378700409F
:103AD8001307F7FF9306A000232AE4002324D40049
:103AE8003787FFFF231CE4002326D4006FF09FEEE6
:103AF800130770002324E400370701801307F7FF3A
:103B0800232AE40013071000231CE40013076000B5
:103B18006FF01FEC93066000370780001307F70F5C
:103B2800232AE4002324D400130700106FF09FFB1E
:103B3800370700041307F77F93066000232AE40081
:103B4800371700002324D400130707806FF09FF96C
:103B5800930640006FF05FFC0355260063040500E0
:103B680093E7170023110600938616001306260014
:103B78006FF05FEDE30C0AF0634C2001032744006B
:103B8800930700096306F70013850400EFF00FC9D7
:103B980083D744006388070013850400EFF00FC340
:103BA80013091900B7870000239C04009387E7FFD7
:103BB80063D42703B787FFFF93C7F7FF2391F40068
:103BC80093874400938484012390070093872700F8
:103BD800E39CF4FE6FF05FD663560900239104005E
:103BE8006FF09FD5239124016FF01FD5E3980AD871
:103BF800239C04006FF01FFC130101FE23244101E4
:103C0800035A2500232C810013840500232E11005C
:103C1800232A910023282101232251012320610115
:103C280013090600130B460323263101930A0500E6
:103C3800EFF09FA283542400330AAA40130504001E
:103C4800EFF09FA1B384A44013050B00EFF0CFB0B1
:103C580063D2440513050400032481018320C101B4
:103C68008329C100032A8100832A4100032B010014
:103C78009307090093860400032901018324410165
:103C8800130700001306000093050000130101024A
:103C98006FF01FC49305040013850A00EFF04FAFBF
:103CA80093090000634AA0009305040013850A00E5
:103CB800EFF0CFC99309100013050B00EFF00FB612
:103CC8008357C904130504009384F4FFB3E9F9008A
:103CD80023163905EFF08FB46FF09FF7130101F742
:103CE800232481082322910823202109232E310728
:103CF80023261108232C4107232A5107232861076B
:103D080023267107232481072322910793040500A2
:103D1800138405001309060093890600EFF04FD4B9
:103D2800630205049305090013850400EFF00FA151
:103D38008320C1080324810883244108032901083A
:103D48008329C107032A8107832A4107032B010717
:103D5800832BC106032C8106832C4106130101091C
:103D68006780000013050400EFF08FCF630805009B
:103D780093050900130504006FF05FFB1385040029
:103D8800EFF04FF26314050613050400EFF08FF10E
:103D9800630C050097D500009385456B13850400D7
:103DA800EFF0CFDF630E050413850400EFF08FEF0B
:103DB8006318050013050400EFF0CFEE630C05044B
:103DC80013850400EFF00FCD9304050013050400DC
:103DD800EFF04FCC638CA402B787FFFF2319F900DB
:103DE80013050900EFF04FEF6FF09FF497D500002F
:103DF8009385C56513050400EFF04FDAE31605F85F
:103E080013050900EFF0DF926FF09FF22319090004
:103E18006FF01FFD138504009305C100EFF00FCB71
:103E28001305040093058102EFF04FCA0354E10023
:103E38008354A1026314040293070000130760016E
:103E48009306C100B386F60083D62600638A06105F
:103E58001305C100EFF05F803304A0408357A1022F
:103E6800138C040063920702130760019306810212
:103E7800B386F60083D62600638E060E13058102EC
:103E8800EFF08FFD338CA44083578102938B490355
:103E980093848903239AF9028357A102138A0B009A
:103EA800239BF9029387E904239004009384240058
:103EB800E39C97FE930A0000130B0000930CC0FECE
:103EC8009307C100B387570103D58701630E050027
:103ED8009305810213064104EFF0CFAA93850B00E6
:103EE80013054104EFF00FA383D7C90413850B0012
:103EF800938AEAFF336BFB00EFF04F9FE3929AFD42
:103F08009307810203570A00130A2A0093872700A0
:103F1800239FE7FEE3189AFEB7C6FFFF3304840128
:103F2800938626009387090013070004B306D4007C
:103F38001306000093050B0013058102EFF05F994B
:103F48000357C10083578102631CF702231401023F
:103F58009305090013058102EFF01F806FF05FDD04
:103F680093872700E39EE7EC13050900EFE0DFFBEA
:103F78006FF01FDC93872700E39AE7EE6FF0DFFE10
:103F88009307F0FF2314F1026FF09FFC130101F770
:103F9800232481082322910823202109232A510759
:103FA80023261108232E3107232C410723286107D4
:103FB8002326710723248107232291072320A107A1
:103FC800930405001384050013090600938A06006C
:103FD800EFF00FA963040504930509001385040095
:103FE800EFE0DFF58320C10803248108832441081A
:103FF800032901088329C107032A8107832A410766
:10400800032B0107832BC106032C8106832C410651
:10401800032D010613010109678000001305040040
:10402800EFF00FA4630805009305090013050400C9
:104038006FF01FFB97D50000938545411385040059
:10404800EFF0CFB5630E051E13850400EFF08FC5A2
:104058009309050013050400EFF0CFC4639209200B
:1040680063180520138504009305C100EFF00FA61F
:104078001305040093058102EFF04FA58354A102B4
:104088000354E100639404029307000013076001DE
:1040980093068102B386F60083D626006380062045
:1040A80013058102EFF04FDBB304A0408357E10012
:1040B800930B040063920702130760019306C10083
:1040C800B386F60083D626006380061E1305C1005A
:1040D800EFF08FD8B30BA440835781020357A10296
:1040E80093894A03239AFA0293878A03239BEA0255
:1040F800138A07001387EA0493872700239F07FE84
:10410800E39CE7FE13058102EFE05FEC035C21010D
:10411800370B01009305FBFF13050C00EFC0D050CF
:10412800130D0500938CA901130BFBFF0355C10266
:104138008357E10213040B00131505013305F5003D
:10414800636AAD0093050C00EFC0D050131405014D
:10415800135404019305C100130504001306410418
:10416800EFF04F829305810213054104EFE05FE20F
:104178006356A002930541041305C100EFE01FFD3B
:104188009305810213054104EFE09FE0634CA01200
:104198001304F4FF1314040113540401930581025A
:1041A80013054104EFE09FFA1305810223108A00EA
:1041B800130A2A00EFE09FF1E31A9AF79307000029
:1041C800930500001307600193068102B386F60089
:1041D80083D6460093872700B3E5D500E396E7FE2C
:1041E800B335B0009307810203D7090093892900EA
:1041F80093872700239FE7FEE3183AFFB74600009E
:10420800B38474419386F6FF93870A00130700046A
:10421800B386D4001306000013058102EFF04FEBBC
:104228000357C10083578102631CF70A2314010254
:104238009305090013058102EFF00FD26FF09FDAA2
:1042480097D500009385852013050400EFF00F959E
:10425800E31C05DE13050900EFF08FCD6FF09FD842
:10426800E31A05FE13050900EFE01FCC6FF09FD796
:1042780013850400EFF00F82930405001305040072
:10428800EFF04F81638CA402B787FFFF2319F90071
:1042980013050900EFF04FA46FF0DFD493872700D0
:1042A800E398E7DE6FF01FFC93872700E398E7E0C9
:1042B8000357C10083578102E318F7FC231909004B
:1042C8006FF01FFD1304E4FF131404019305410468
:1042D8001305C10013540401EFE05FE76FF01FEC12
:1042E8009307F0FF2314F1026FF09FF403AE05006B
:1042F80003A3450083A8850083A5C500130101E237
:10430800232C811C2326B10213840700832505046E
:104318009307F0FF2328F114930700092328211D90
:104328002326311D2324411D232E711B232E111CEE
:10433800232A911C2322511D2320611D232C811B1C
:10434800232A911B2328A11B2326B11B2326010105
:104358002320C1032322610223241103232AF114F9
:1043680013090500130A060093890600930B07003A
:104378006380050283274504130710003317F700ED
:1043880023A2F50023A4E500EF10807A2320090476
:104398001305010293050105EFF00FC3130501058D
:1043A800EFE05FEF630E0518930710002320F40079
:1043B80093073000630AFA1893044001630A0A005D
:1043C8009384F9FF9307A00263D497009304A00293
:1043D80083274115130501052328F100EFE05FE865
:1043E8001304050097D500009385852BE31605284F
:1043F800930700099305C10613050105232AF11443
:10440800EFE0DFB38357E107930A00001397070132
:1044180013570741635E0700378700001307F7FF4C
:10442800B3F7E700B70A0100231FF106938AFAFFE2
:104438009305810817D5000013058502EFE01FB02A
:104448000357E107E31A07201307C1069307000083
:10445800930690000356070063140610938717000D
:1044680013072700E398D7FE9305010C130581086D
:10447800EFE0DFE5930581081305010CEFE01FAFBE
:104488009305010C1305C106EFE05FE49305C1062F
:104498001305010CEFE09FAD130601159305C10646
:1044A80013058108EFF04FF5035BC11917DC000015
:1044B800130CCCF9631A0B0093050C001305C10605
:1044C800EFE0DFED6310056C9307D00263940A00F8
:1044D80093070002230AF11093073000138C04009D
:1044E8006318FA00338C84009307A002E3C0872383
:1044F8009307A000631EFB6C93071003A30AF11037
:104508009307E002230BF110130B7111635A80011A
:1045180093070003A30BF110130CFCFF130B81117D
:104528001304140063500C6C1306040097D50000A4
:104538009385451913050B00EF20C0626F00D01456
:10454800232004006FF0DFE6938409006FF09FE7F3
:104558008317C10797D5000093858516E3DE0710FA
:104568009305C10617D50000130585EFEFE01FE39B
:10457800E30C05EE635805469305410A1305C10689
:10458800EFE0DF9BB74700009387E708231BF10A9A
:10459800B78700009387F7FF232AF100B7C7FFFF0B
:1045A80093872700130C0000930C0001232CF100C3
:1045B80097D70000938707F633858701930601157F
:1045C800130681089305410AEFF05F9C13058108E3
:1045D8009305C103EFE09F9683274101035BE10444
:1045E80003278101B377FB003385E700634EA004FE
:1045F8001305010CEFE05F93131B0B01135B0B41D9
:1046080063500B12930700001307C1033307F70029
:10461800835607001307010C3307F70003570700F9
:10462800638AE63A17D50000130585E3EFE05FC318
:10463800630805089305010C17D50000130545E22A
:10464800EFE0DF8F6F00C00D93070009B38DA7401F
:104658009305010C1305C103EFE05F8E6352B00DA3
:104668009306010C13870D001306F0006342E6045D
:1046780013D54D009307010C13171500930500FF80
:10468800338DE700EFC0407A3305B50197D70000B6
:104698009387C7DB131515003385A70083560D00D4
:1046A8008357C512B3F7D7002310FD006FF0DFF46E
:1046B80023900600130707FF938626006FF01FFB61
:1046C8001305010CEFE0DFB9630805009305010C41
:1046D800138505006FF0DFF617D50000130545D8E0
:1046E800EFE05FDC130D05001305010CEFE09FDB25
:1046F800130B0500630C0D146302051217D5000097
:10470800130505D6EFE01FB9130B05001305010CBF
:10471800EFE05FB86314AB101305010CEFF04F81A5
:1047280093070000130781083307F7008356070033
:104738001307010C3307F700035707006390E602DD
:104748009387270013072001E39EE7FC9305410A9E
:1047580013058108EFE08FFE33049401130C4C011C
:104768009307400693DC1C00E314FCE48357610BB9
:104778000357E1079305C1061305410AB387E7000C
:1047880037C7FFFF130727F7B387E700231BF10A93
:10479800EFE0CFFA9305810817D50000130545CC43
:1047A800EFE0CFF9130B0000B71C0000930D401089
:1047B80097D70000938707CC9305410A17D50000C7
:1047C800130545DA338C6701EFE05FBDE34EA0C8FF
:1047D8009305410A13050C00EFE05FBC6348A00293
:1047E8001306410A930506009306011513050C00EC
:1047F800EFF0CFF91306810893060115930506001B
:1048080013050C00EFF08FCD33049401130B4B010B
:1048180093DC1C00E31EBBF96FF01FC517D5000021
:10482800130505C49305010CEFE04FF11305010CC6
:10483800EFE01FA3E31605EE8357210D3787FFFF2F
:10484800B3C7E7002319F10C6FF09FEDE31005E8FB
:104858009305C10D17D50000130585C0EFE01FA70C
:104868009305810F1305010CEFE05FA60357C10DF7
:10487800835DA10F8357E10D1347F7FF131D070150
:10488800135D0D01231EA10DB387B7416354F008D2
:10489800930541111305810F232EF100EFE00FED71
:1048A8009305810F1305C10DEFE04FEC9305C10D82
:1048B80013054111EFE08FEB8327C101835DA10F41
:1048C800B307F0401307F0F663C6E70893850700BF
:1048D8001305C10DEFE0DFC2130D05000357C10D2D
:1048E8008357810F9305810F1305C10D631EF70CC4
:1048F800EFE05F82930701151307000493860D000C
:1049080013060B0093050D001305810FEFE05FFC04
:104918006F004004E39807FA9305810F1305C10D52
:10492800EFE00FE7631805068357810F6388A70137
:104938001305010CEFE04FDF6FF09FDE63940D026B
:104948000317E10F93070000634007021305810F67
:10495800EFE0CFEC9305010C1305810FEFE0DFDFEB
:104968006FF01FDC93070000130760019306810FA7
:104978003386F6000356260063080600938D1D0053
:10498800231DB10F6FF01FFD93872700E390E7FE0B
:104998006FF01FFF130D0000E352A0F493054111BF
:1049A8001305810FEFE08FDC9305810F1305C10D0F
:1049B800EFE0CFDB9305C10D13054111EFE00FDBED
:1049C800130D0B006FF09FF1EFE04FF8130B100081
:1049D8006FF05FF29387270013072001E396E7C281
:1049E8006FF01FD48357E10717DB0000130B8BB759
:1049F8006388070A9305010C1305C106374B0000AD
:104A0800EFE0DF8C130BEBFF130C50FD8357810D88
:104A180093F77700639207069305410A1305010C83
:104A2800EFE0CFD41305410AEFE04FDA1305410A4E
:104A3800EFE0CFD99305410A1305010CEFE08FEDA4
:104A48008357610A938737002313F10A8357810A32
:104A5800639007128357C10B639007028357610A5B
:104A6800636CFB009305010C1305410A1304F4FF62
:104A7800EFE0CFCFE31C84F99305C1061305010CC1
:104A8800EFE09FCD6F0040021306C10693060115A3
:104A98009305060013050B00EFF04FA41304F4FF71
:104AA8008317C107E3D207FE9305010C1305C1065E
:104AB800EFE0CFC89305810817D500001305459A84
:104AC800EFE0CFC7930C000037FBFFFF17DD0000B6
:104AD800130D4D9A930D401097D70000938707AC9C
:104AE800338797019305010C17D5000013054597E7
:104AF800232AE100EFE09F8A330C9D01032741013F
:104B0800635AA0049305010C13050700EFE01F8901
:104B1800634805021306010C930506009306011568
:104B280013050C00EFF08F9B1306810893060115FF
:104B38009305060013050C00EFF04F9A3304640147
:104B48001357FB01330B6701938C4C01135B1B401C
:104B5800E394BCF9130681089306011597D5000064
:104B68009385059013050600EFF04FC26FF0DF8FB5
:104B78001305410AEFE08FC58357610A9387170031
:104B88006FF09FEC1305C106EFE04FC99305410A8A
:104B98001305C106EFE08FBD1305410AEFE00FC80A
:104BA8001305410AEFE08FC79305C1061305410AB3
:104BB800EFE04FD6130601159305C10613058108CA
:104BC800EFF08F831304F4FF035BC1196FF09F8E1E
:104BD800130B0B039307E002A30A6111230BF110D7
:104BE800130B7111930A0B00B3876A416356FC04D7
:104BF8008357C11913074000138BFAFFE356F79246
:104C0800130750006384E70893070B001306E002BC
:104C180093058003930600039387F7FF03C70700F4
:104C28001377F70763580C0A130710032380E7006C
:104C3800130414006FF05F8F1305C106EFE00FBE79
:104C48009305410A1305C106EFE04FB21305410A67
:104C5800EFE0CFBC1305410AEFE04FBC9305C10656
:104C68001305410AEFE00FCB130601159305C106A2
:104C780013058108EFE05FF88347C119938A1A008A
:104C880093870703A38FFAFE6FF01FF69305810839
:104C98001305C106EFE05FAC97C500009385057B5F
:104CA80013058108EFE08FEFE31005F6E34E0C865D
:104CB80083C7EAFF938727FD93B7170093C7F7FFCA
:104CC800B307FB0083C7070093F71700E38E078439
:104CD8006FF09FF36314C70203C7F7FF93068003BF
:104CE80063E8E60013071700A38FE7FE6FF0DF8382
:104CF80013041400130710036FF01FFF63E8E500A7
:104D0800130717002380E7006FF01F822380D70066
:104D18006FF09FF01304140023A08B0093870A0000
:104D28009306E00203C70700631607001307500441
:104D38006F00C002630CD700938717006FF09FFEC7
:104D480003C7170093871700A38FE7FE03C7070061
:104D5800E31807FE6FF09FFD9387F7FF83C60700F0
:104D68006384E600E3EAFAFE238007006F0000157B
:104D7800938717006F004015138406006F00C01555
:104D88001304F4FF230004000347F4FF6316D7005D
:104D980033075441E3C6E7FE9307300013879900B1
:104DA8006314FA0283270116B384F40063D804005D
:104DB800230A011023A00B0013840A0083A70B0009
:104DC800B389F900138739002322090493074000A7
:104DD80093864701832549046378D706130509009C
:104DE800EF00904A2320A90493850A009304050044
:104DF800EF20400A8327C100638807003304544129
:104E08003384840023A087008320C11D0324811DCF
:104E1800138504000329011D8324411D8329C11C16
:104E2800032A811C832A411C032B011C832BC11BD1
:104E3800032C811B832C411B032D011B832DC11ABD
:104E48001301011E67800000938515002322B90411
:104E5800939717006FF0DFF7B78700009387F7FF86
:104E68006318F7EE97D500009385C58463860A001A
:104E780097D5000093854583130541113724000019
:104E8800EF10504E1304F470832701011305010538
:104E980023208116232AF114EFE0CFE0930A411171
:104EA8006318050013050105EFE08FBBE30405E671
:104EB800B72700009387F77023A0FB0093870A00A9
:104EC800130600029306D00203C70700E302C7EAED
:104ED800E300D7EA13840A009387170003C7F7FF94
:104EE80093061400A38FE6FEE31807E813072000D3
:104EF800930710006308EA008327011663D497001C
:104F080093870400930600036FF01FE89307A0003F
:104F1800130CA002E31EFBCA93071003A30AF110A7
:104F28009307E002230BF110130CA0026FF04FDE81
:104F380083270500130101FC930541012320F1009B
:104F480083274500232E11022322F10083278500A1
:104F58002324F1008327C500130501002326F1004F
:104F6800EFE09F86835761021305000093C7F7FFA0
:104F780013971701631A070013054101EFE04FAEBD
:104F880013351500130515008320C103130101040F
:104F9800678000001305050F6780000097E7000091
:104FA800938747B683A7070003A547036316050041
:104FB80017D500001305855D1305050F67800000F0
:104FC80097E70000938707B483A7070003A5470363
:104FD8006316050017D500001305455B1305050F7B
:104FE8006780000063080606130101FF97C50000EB
:104FF8009385C56D1305060023248100232611001F
:1050080013040600EF1050516308050297C500000D
:105018009385856B13050400EF101050630E05008F
:1050280097C500009385C52513050400EF10D04EE1
:10503800930700006316050097C700009387C768A9
:105048008320C10003248100138507001301010197
:105058006780000097C700009387076713850700DC
:105068006780000097E700009387C7A983A7070018
:1050780083A747036396070097D7000093870751D4
:1050880003C58712678000000325C50E67800000EE
:1050980097E70000938707A783A7070083A747031D
:1050A8006396070097D700009387474E03A5C70E5E
:1050B8006780000097E700009387C7A41386050060
:1050C8009305050003A507006FF0DFF1130101FA4E
:1050D800232A9104938405008395E500232C8104F9
:1050E800232E11041304060063DE050083D7C400D1
:1050F80023A0060093F70708639807049307004066
:105108006F00C004130641012326D100EF500004AC
:105118008326C100E34C05FC03278101B7F7000093
:1051280037150000B3F7E70037E7FFFFB387E7005D
:1051380093B7170023A0F600930700402320F4003C
:10514800130505806F000001930700042320F40075
:10515800130500008320C10503248105832441052C
:10516800130101066780000083D7C500130101FE03
:10517800232C8100232E1100232A910023282101AA
:1051880093F7270013840500638807029307340404
:105198002320F4002328F40093071000232AF400A6
:1051A8008320C101032481018324410103290101D2
:1051B80013010102678000009306C10013068100F5
:1051C80093040500EFF09FF0832581001309050083
:1051D80013850400EF004008631005028317C4001C
:1051E80013F70720E31E07FA93F7C7FF93E7270093
:1051F8002316F4006FF09FF997D7FFFF93870756A0
:1052080023AEF4028357C4002320A4002328A4005B
:1052180093E707082316F40083278100232AF40064
:105228008327C100638207028315E4001385040005
:10523800EF50003D630A05008357C40093F7C7FF8A
:1052480093E717002316F4008357C4003369F90065
:10525800231624016FF0DFF4130101FD2326110248
:10526800232481022322910223202103232E3101AA
:10527800232C4101232A510123286101232671018E
:10528800232481019387B500130760016374F70431
:1052980093F487FF63D204049307C0002320F5002A
:1052A800130500008320C1020324810283244102E4
:1052B800032901028329C101032A8101832A4101AB
:1052C800032B0101832BC100032C8100130101036F
:1052D8006780000093040001E3E0B4FC13090500B3
:1052E800EF00007A9307701F97D900009389C9408F
:1052F80063EA9704138784003387E900032447008F
:10530800930687FF93D734006318D4000324C7009B
:105318009387270063008708832744000327C40076
:105328008326840093F7C7FFB307F40023A6E6009B
:105338002324D70003A747001367170023A2E70019
:105348006F00C00A13D794009307F003630A07009D
:105358009307400063E4E70A93D7640093878703C1
:1053680013871700131737003387E9000324470012
:10537800930587FF1305F000630CB400032744006E
:105388001377C7FF330697406352C50C9387F7FF1F
:105398009387170003A4090197D500009385453624
:1053A8006302B414032744009306F0001377C7FF81
:1053B8003306974063DEC60A93E714002322F400FD
:1053C800B306940097D7000023A2D73497D70000DC
:1053D80023ACD7329367160023A6B60023A4B600E1
:1053E80023A2F6003307E4002320C70013050900B1
:1053F800EF004069130584006FF0DFEA930740016E
:1054080063E6E7009307B7056FF09FF5930740053C
:1054180063E8E70093D7C4009387E7066FF05FF46B
:105428009307401563E8E70093D7F400938777075D
:105438006FF01FF3930640559307E007E3E2E6F2A7
:1054480093D724019387C7076FF09FF18326C40081
:10545800634C06008327840023A6D70023A4F60004
:10546800B307E4006FF01FED138406006FF0DFF060
:1054780097D6000023ACB62897D6000023A6B628F6
:10548800634C06003307E4008327470093E71700BF
:105498002322F7006FF09FF59306F01F03A8490039
:1054A80063E2E61A13573700135627409306100095
:1054B80013071700B396C600131737003387E900A0
:1054C800B3E6060117D60000232AD6228326070052
:1054D800130687FF2326C4002324D4002320870033
:1054E80023A6860013D72740130310003313E300C5
:1054F80003A74900636C6706B3766700639C0600E0
:1055080093F7C7FF13131300B37667009387470019
:10551800E38A06FE130EF00093963700B386D9008F
:1055280013880600138507000324C800631E041DA2
:10553800130515001377350013088800E31607FED6
:1055480013F737006314072403A749009347F3FFB1
:10555800B377F70017D700002322F71A03A74900EB
:1055680013131300636467006316032483AB890075
:1055780003A44B00937AC4FF63E89A0033879A40E8
:105588009307F00063C0E73697D700009387075961
:1055980003A4070097D700009387075783A607003F
:1055A8001307F0FF33848400138A07006398E6200A
:1055B800130404019305040013050900EF10404487
:1055C8009307F0FF130B05006302F52AB3875B010D
:1055D8006374F500639C3B2917DC0000130C8C54A2
:1055E80003270C003307E40097D6000023ACE652EB
:1055F8006392671F93964701639E061C83A78900E1
:1056080033848A001364140023A2870017D700008C
:105618001307875083270C00032707006376F700DA
:1056280017D70000232AF74E17D700001307874E15
:1056380003270700637CF72217D70000232CF74CB9
:105648006F00C022135697009306400063E8C60413
:105658009356670093868603138616001316360042
:105668003386C900130586FF032606006314C508A0
:105678001307100093D62640B316D700B3E60601E9
:1056880017D70000232CD7062326A4002324C40000
:1056980023248500232686006FF0DFE4930640016B
:1056A80063E6C6009306B6056FF01FFB9306400538
:1056B80063E8C6009356C7009386E6066FF0DFF9E5
:1056C8009306401563E8C6009356F700938676075D
:1056D8006FF09FF8130540559306E007E36EC5F693
:1056E800935627019386C6076FF01FF70326860097
:1056F8006308C5008326460093F6C6FFE368D7FE15
:105708000325C6006FF05FF8032744000326C40092
:105718001377C7FFB308974063541E0593E7140037
:105728002322F40083278400B30694003307E4009F
:1057380023A6C7002324F60097D7000023A8D7FC88
:1057480097D7000023A2D7FC93E7180023A6B6003A
:1057580023A4B60023A2F600232017016FF01FC967
:1057680063C208023307E4008327470093E7170062
:105778002322F7008327840023A6C7002324F600EA
:105788006FF0DFC6130406006FF05FDA138786FF39
:1057980083A606009387F7FFE384E6DA6FF01FDC41
:1057A8009387470013131300B3766700E38A06FE56
:1057B8006FF09FD6930705006FF01FFFB717000023
:1057C8009387F7003304F400B7F7FFFF3374F4004E
:1057D8006FF05FDE03260A009306F0FF631CD60A0B
:1057E80097D7000023A2673393757B006388050071
:1057F80093078000B385B740330BBB00B717000091
:10580800B385F50033048B009387F7FF3374F400F6
:10581800338A854093050A0013050900EF10401EDE
:105828009307F0FF6316F50013050B00130A000039
:1058380083270C0033056541B3874701330A4501C7
:1058480017D700002320F72E136A1A0097D70000F5
:1058580023A867EB23224B01E38A3BDB1307F00005
:1058680063645705930710002322FB0083A7890070
:1058780083A7470093F7C7FF3387974063E69700EE
:105888009307F00063C0E70613050900EF00801FC7
:105898006FF01FA1B307FB40B387E70017D70000DD
:1058A8002322F7286FF05FF483A74B0013844AFF85
:1058B800137484FF93F71700B3E7870023A2FB0054
:1058C80093065000B3878B0023A2D70023A4D700E8
:1058D800E37E87D293858B0013050900EFD0CFA70D
:1058E8006FF0DFD203A4890093E714002322F400A9
:1058F800B307940097D6000023A4F6E06FF0DFA367
:1059080097D700009387072083A7070083A747033B
:105918006396070097D70000938747C703A3470EEE
:1059280067000300639A0502130101FF9305C10094
:1059380013050000630E06001305E0FF638A0600E6
:105948008347060023A0F500034506003335A00071
:1059580013010101678000001305000063000602BF
:105968001305E0FF638C06008347060023A0F500BB
:10597800034506003335A0006780000067800000FB
:1059880093F5F50F3306C5006316C500130500002F
:105998006780000083470500E38CB7FE13051500F8
:1059A8006FF09FFE1303F00013070500637EC30228
:1059B8009377F7006390070A63920508937606FFCA
:1059C8001376F600B386E6002320B7002322B7003B
:1059D8002324B7002326B70013070701E366D7FE81
:1059E8006314060067800000B306C3409396260040
:1059F80097020000B38656006780C6002307B700E9
:105A0800A306B7002306B700A305B7002305B70010
:105A1800A304B7002304B700A303B7002303B70008
:105A2800A302B7002302B700A301B7002301B70000
:105A3800A300B7002300B7006780000093F5F50FB7
:105A480093968500B3E5D50093960501B3E5D50097
:105A58006FF0DFF69396270097020000B386560092
:105A680093820000E78006FA93800200938707FF7D
:105A78003307F7403306F600E378C3F66FF0DFF339
:105A880067800000678000008327C504130101FFB9
:105A980023229100232021012326110023248100A1
:105AA80093040500138905006382070403A7C4044F
:105AB80093172900B307F70003A50700631005062D
:105AC800130410003314240113065400131626007F
:105AD8009305100013850400EF40C02E63020502F1
:105AE80023222501232485006F00C003130610021A
:105AF80093054000EF40002D23A6A404E31805FAFF
:105B0800130500008320C100032481008324410081
:105B18000329010013010101678000000327050024
:105B280023A0E70023280500232605006FF09FFD2A
:105B38006380050283A74500139727008327C504C0
:105B4800B387E70003A7070023A0E50023A0B70059
:105B580067800000130101FD2322910283A405013F
:105B6800232A5101B70A010023248102232021039B
:105B7800232E310123286101232671012324810169
:105B880023261102232C410123229101130B050026
:105B980013840500930B06001389060093894501B9
:105BA800130C0000938AFAFF83AC090093850B005D
:105BB8009389490033F55C01EFB00027330A2501CA
:105BC80093850B0013D50C01EFB0002693570A01FB
:105BD8003305F50013590501337A5A0113150501E8
:105BE8003305450123AEA9FE130C1C00E34E9CFAB5
:105BF800630009068327840063C0F40483254400F6
:105C080013050B0093851500EFF01FE80326040128
:105C18009305C400930905001306260013162600F1
:105C28001305C500EF40D0279305040013050B00AA
:105C3800EFF01FF01384090093874400939727001F
:105C4800B307F40023A227019384140023289400A7
:105C5800130504008320C102032481028324410226
:105C6800032901028329C101032A8101832A4101F1
:105C7800032B0101832BC100032C8100832C4100DD
:105C88001301010367800000130101FE232C81002A
:105C98002324410113840500130A0500930590008D
:105CA80013858600232A91002328210123225101EC
:105CB800232E11002326310193040600938A06003F
:105CC80013090700EFB08018930710009305000030
:105CD80063C2A70813050A00EFF01FDB9307100043
:105CE8002328F500232A25019307900063DA9706F5
:105CF8001309940093090900330494009389190047
:105D080083C6F9FF930505001306A000938606FDD8
:105D180013050A00EFF01FE4E39289FE33049900AB
:105D2800130484FFB3848440B307940063C0570509
:105D38008320C10103248101832441010329010136
:105D48008329C100032A8100832A4100130101022B
:105D58006780000093971700938515006FF05FF731
:105D68001304A400930490006FF0DFFB13041400E5
:105D78008346F4FF930505001306A000938606FDED
:105D880013050A00EFF01FDD6FF01FFA3707FFFF5A
:105D98003377E50093070500130500006316070035
:105DA8009397070113050001370700FF33F7E70052
:105DB800631607001305850093978700370700F0DF
:105DC80033F7E7006316070013054500939747006C
:105DD800370700C033F7E7006316070013052500EF
:105DE8009397270063CC07001397170063560700A3
:105DF8001305150067800000130500026780000086
:105E08008327050013F77700630E070293F6170040
:105E180013070000639C060013F72700630C0700B4
:105E280093D717002320F500130710001305070068
:105E38006780000093D727002320F5001307200070
:105E48006FF0DFFE9396070193D606011307000053
:105E58006396060093D707011307000193F6F70F1F
:105E6800639606001307870093D7870093F6F70019
:105E7800639606001307470093D7470093F6370049
:105E8800639606001307270093D7270093F6170099
:105E98006398060093D71700638807001307170055
:105EA8002320F5006FF09FF8130700026FF01FF82A
:105EB800130101FF232481001384050093051000BA
:105EC80023261100EFF05FBC232A85008320C10040
:105ED80003248100130710002328E50013010101A2
:105EE8006780000003A7050183270601130101FA53
:105EF800232A910423244105232E1104232C8104F1
:105F08002328210523263105232251052320610555
:105F1800232E7103232C8103232A91032328A10311
:105F28002326B103138A0500930406006356F7007D
:105F3800130A06009384050003290A0183A90401B2
:105F480083278A0083254A00330C390163D48701EB
:105F580093851500EFF05FB3930B4501931C2C005C
:105F6800130D0500B38C9B0193870B0063E497091D
:105F7800130A4A0113192900B3072A01938444011B
:105F8800939929002326F100B70A0100B387340149
:105F98002328F100938AFAFF8327010163E2F406BC
:105FA80063588001938CCCFF83A70C00638A071881
:105FB8008320C1050324810523288D0113050D00C5
:105FC80083244105032901058329C104032A810487
:105FD800832A4104032B0104832BC103032C81036F
:105FE800832C4103032D0103832DC10213010106F4
:105FF8006780000023A00700938747006FF01FF712
:1060080083AD0400B3FD5D0163880D0813890B009F
:1060180013070A00930900000326070093850D0063
:106028000324090033755601232AE100232CC100FB
:10603800EFA0905F0326810103274101337B5401C0
:10604800330B6501130747001355060193850D00AF
:10605800330B3B01232AE100232EE10013540401F2
:10606800EFA0905C3305850013540B0133058500C0
:1060780093590501337B5B01131505018327C10083
:10608800032741011306490033656501232EA6FE47
:106098006360F70A2322390103D92400630409083D
:1060A80003A40B00938D0B0093090A0093060000CC
:1060B80003A5090093050900232AD100337555016A
:1060C800EFA0905603DB2D00832641013374540161
:1060D800330B6501330BDB0013150B0133648500AB
:1060E80023A08D009389490003D5E9FF13864D004D
:1060F80093050900232AC100EFA0105303A44D0003
:106108008327C100135B0B013374540133048500EA
:1061180033046401935604010326410163EEF90038
:1061280023A28D0093844400938B4B006FF0DFE62D
:10613800130906006FF05FEE930D06006FF05FF72E
:10614800130CFCFF6FF0DFE5130101FE232A910019
:106158002328210123263101232E1100232C81001D
:1061680023244101937736001309050093040600A0
:1061780093890500638407029387F7FF17B7000028
:106188001307C75593972700B307F70003A607001F
:1061980093060000EFF01F9C9309050093D4244058
:1061A8006380040803248904631E040093051027F0
:1061B80013050900EFF0DFCF2324A9041304050019
:1061C8002320050093F714006384070293850900D0
:1061D8001306040013050900EFF0DFD0130A0500C9
:1061E8009385090013050900EFF09F9493090A00AD
:1061F80093D414406386040203250400631E05003B
:10620800130604009305040013050900EFF09FCD61
:106218002320A40023200500130405006FF09FFA33
:106228008320C101032481011385090083244101CE
:10623800032901018329C100032A810013010102F6
:1062480067800000130101FD232291029384050059
:10625800232E310183A904012324810283A545004B
:106268001354564083A78400B30934012320210323
:10627800232A510123261102232C4101930A0500E8
:106288001389190063C6270D13850A002326C10048
:10629800EFF08FFF0326C10093074501130A05009D
:1062A8009386070013070000938646006348870A11
:1062B800635404001304000083A60401131424008B
:1062C8003387870093962600938744011376F60157
:1062D800B386D700630E0608130800023308C840C7
:1062E8009305000003A5070093084700938747001C
:1062F8003315C500B365B50023AEB8FE83A5C7FF47
:10630800B3D5050163E2D7062322B70063840500ED
:10631800138929001309F9FF23282A0113850A0084
:1063280093850400EFF0DF808320C10203248102FB
:1063380013050A0083244102032901028329C101AC
:10634800032A8101832A41011301010367800000A8
:1063580093851500939717006FF0DFF223AE06FEC2
:10636800130717006FF05FF4138708006FF09FF7AB
:106378009387470003A6C7FF13074700232EC7FECE
:10638800E3E8D7FE6FF01FF98327050103A705018E
:10639800B387E740639C07021317270013054501DD
:1063A80093854501B306E500B385E5009386C6FFEE
:1063B8009385C5FF03A6060003A70500630CE60046
:1063C8009307F0FF6364E600930710001385070046
:1063D80067800000E36CD5FC6FF05FFF130101FEDE
:1063E800232A910093840500232631019305060092
:1063F8009309050013850400232C8100232E110026
:106408002328210113040600EFF01FF8631C05027E
:106418009305000013850900EFF00FE793071000BC
:106428002328F500232A05008320C10103248101C4
:1064380083244101032901018329C10013010102B9
:106448006780000013091000634A050093070400E1
:106458001309000013840400938407008325440073
:1064680013850900EFF04FE20323040183A8040118
:1064780013064401131E230013884401939828002F
:10648800B70E010023262501330EC601B3081801F3
:1064980093064501130F0000938EFEFF03270600A5
:1064A800832F080093864600B375D701B3F7DF0141
:1064B800B385E501B385F54093DF0F0193570701D5
:1064C800B387F74113D70541B387E70013DF0741C7
:1064D800B3F5D50193970701B3E7B7001308480050
:1064E80023AEF6FE13064600E36A18FBB705010063
:1064F8009385F5FF636CC6019386C6FF83A70600E4
:1065080063820704232865006FF01FF283270600C3
:10651800938646001306460033F7B7003307E701B2
:106528001358074193D70701B387070113DF0741C2
:106538003377B70093970701B3E7E70023AEF6FE7A
:106548006FF05FFB1303F3FF6FF01FFBB707F07FDC
:10655800B3F5B700B707C0FCB385F5006358B000C2
:10656800930700001385070067800000B305B0405B
:1065780093D74541130730016348F700B705080072
:10658800B3D5F5406FF0DFFD9387C7FE9306E001B2
:10659800930500001307100063C6F60093C7F7FFC2
:1065A8003317F700930707006FF0DFFB130101FDB6
:1065B8002322910283240501232E310193094501E9
:1065C80093942400B38499002324810203A4C4FF74
:1065D800232021032326B1001305040023261102DA
:1065E800EFF0CFFA8325C10093070002B387A740D5
:1065F80023A0F5009307A0001389C4FF63CCA70468
:106608009307B000B387A7403707F03FB356F400AD
:10661800B3E6E6001307000063F4290103A784FF2B
:10662800130555013315A400B357F700B367F500F8
:106638008320C10203248102832441020329010229
:106648008329C101138507009385060013010103FF
:10665800678000009307000063F6290183A784FF81
:10666800138984FF130555FF630E05021307000203
:106678003306A7403314A4003707F03F3364E4001F
:10668800B3D6C700B366D4001307000063F429012A
:106698000327C9FFB397A7003357C700B3E7E7003D
:1066A8006FF01FF9B706F03FB366D4006FF05FF8DC
:1066B800130101FD232481021384050093051000B2
:1066C800232291022320210393040600232E310163
:1066D800232C41011309070023261102138A0600FF
:1066E800EFF08FBA370710009307F7FFB3F797005B
:1066F80093D4440193F4F47F93090500639A040842
:106708002326F100630E0408130581002324810069
:10671800EFF00FEF83268100630005080327C1000F
:1067280093070002B387A740B317F700B3E7D70072
:106738003357A70023AAF9002326E1000324C10048
:1067480023AC8900333480001304140023A8890083
:10675800638A04069384D4BCB384A40093075003CB
:1067680023209A003385A7402320A9008320C10253
:1067780003248102138509008324410203290102AD
:106788008329C101032A81011301010367800000E5
:10679800B3E7E7006FF0DFF623AAD9006FF01FFA1E
:1067A8001305C100EFF0CFE58327C10013050502EB
:1067B8001304100023AAF9009307100023A8F90076
:1067C8006FF01FF9931724001305E5BCB387F90090
:1067D8002320AA0003A5070113145400EFF00FDBD0
:1067E8003304A440232089006FF05FF8130101FDF2
:1067F800232C4101138A05009305810023261102E9
:106808002324810223229102232E3101232A5101BC
:106818002328610123202103130B0500EFF01FD962
:1068280013040500938905009384050013050A00E5
:106838009305C100EFF09FD7930A050083270B014A
:1068480003250A010327C100B387A7400325810058
:10685800939757003305E5403385A7006358A00494
:106868001315450193860500B30435019387060087
:1068780013860A0013050400938504009386070015
:10688800EF60C0128320C1020324810283244102E5
:10689800032901028329C101032A8101832A4101B5
:1068A800032B010113010103678000001389050010
:1068B800B705F0FFEFA04057B30625016FF01FFBA7
:1068C800130101FF23248100232611002322210123
:1068D80023203101930770011304050063CAA7023E
:1068E8001314350097B70000938747DF3384870078
:1068F80003250401832544018320C100032481006A
:106908000329410083290100130101016780000068
:1069180097B700009387076503A5070083A547007D
:1069280097B700009387876403A9070083A94700E6
:1069380013060900938609001304F4FFEF6010089A
:10694800E31804FE6FF05FFB9387F5FF032706014A
:1069580093D75740938717009397270093064601CC
:1069680013172700B307F5003387E60063E6E60050
:10697800636EF500678000009386460003A6C6FF95
:1069880013054500232EC5FE6FF05FFE1305450075
:10699800232E05FE6FF0DFFD8326050193D75540B2
:1069A8001307450163C0F60463D4D70293F5F501D4
:1069B8006380050293962700B306D70003A6060056
:1069C80013051000B356B600B395B6006318B602A7
:1069D80093972700B307F700636AF70013050000D1
:1069E80067800000938706006FF09FFE9387C7FFBC
:1069F80083A60700E38206FE1305100067800000E7
:106A0800130101FF232481001304050013850500E9
:106A180097C7000023AC071223261100EFA0806B54
:106A28009307F0FF631CF50097C7000093870712D0
:106A380083A70700638407002320F4008320C10094
:106A4800032481001301010167800000130101FF85
:106A580023229100B70400802324810023261100FB
:106A680093C4F4FF33F7B400232006003708F07FFF
:106A7800930605009387050013040600635407076F
:106A88003368A70063000806B707100013860500DF
:106A98006356F70297B700009387C74D03A6070010
:106AA80083A64700EF6080719307A0FC930605005A
:106AB8001386050033F7B4002320F400832704006D
:106AC80013574741130727C03387E700B7071080DC
:106AD8009387F7FF3376F600B707E03F2320E400FB
:106AE800B367F6008320C10003248100832441009A
:106AF80013850600938507001301010167800000D4
:106B0800130101F6232AF108B707008093C7F7FF9E
:106B1800232EF1002328F100B707FFFF2326D10811
:106B28002324B100232CB100938787209306C10842
:106B380093058100232E1106232AF1002328E1085A
:106B4800232C0109232E11092322D100EF00803CB8
:106B580083278100238007008320C1071301010ACE
:106B680067800000130101F6232AF108B7070080A7
:106B780093C7F7FF232EF1002328F100B707FFFF83
:106B8800938787202324C1082326D1082328E108D6
:106B9800232C0109232E1109232AF10097C700008D
:106BA800938747F62324A100232CA10003A50700FF
:106BB800930681081386050093058100232E11068C
:106BC8002322D100EF0000358327810023800700AE
:106BD8008320C1071301010A67800000130101FF28
:106BE80023248100138405008395E50023261100E2
:106BF800EF30D03E6340050283270405B387A70022
:106C08002328F4048320C100032481001301010117
:106C1800678000008357C40037F7FFFF1307F7FFAB
:106C2800B3F7E7002316F4006FF0DFFD130500004B
:106C38006780000083D7C500130101FE232C810063
:106C4800232A91002328210123263101232E110014
:106C580093F7071093040500138405001309060031
:106C680093890600638A07008395E5009306200050
:106C780013060000EF30901D8357C40037F7FFFF5D
:106C88001307F7FFB3F7E7002316F4008315E400B2
:106C9800032481018320C10193860900130609009A
:106CA8008329C100032901011385040083244101BC
:106CB800130101026F30C00B130101FF232481006F
:106CC800138405008395E50023261100EF30101882
:106CD8009307F0FF0357C4006312F502B7F7FFFFED
:106CE8009387F7FFB3F7E7002316F4008320C1006A
:106CF800032481001301010167800000B717000019
:106D0800B367F7002316F4002328A4046FF01FFECE
:106D18008395E5006F3000163367B5009303F0FFE5
:106D28001377370063100710B7877F7F9387F7F7CC
:106D38000326050083A60500B372F6003363F60048
:106D4800B382F200B3E26200639272106316D6084F
:106D58000326450083A64500B372F6003363F600A8
:106D6800B382F200B3E26200639E720C6316D60629
:106D78000326850083A68500B372F6003363F60008
:106D8800B382F200B3E262006398720C6316D60411
:106D98000326C50083A6C500B372F6003363F60068
:106DA800B382F200B3E262006392720C6316D602F9
:106DB8000326050183A60501B372F6003363F600C6
:106DC800B382F200B3E26200639C720A13054501C4
:106DD80093854501E30ED6F4131706019397060130
:106DE800631EF7001357060193D706013305F740D2
:106DF8009375F50F6390050267800000135707012C
:106E080093D707013305F7409375F50F6394050091
:106E1800678000001377F70F93F7F70F3305F740F4
:106E2800678000000346050083C6050013051500AA
:106E3800938515006314D600E31606FE3305D64085
:106E4800678000001305450093854500E31CD6FCC8
:106E580013050000678000001305850093858500F1
:106E6800E312D6FC13050000678000001305C50077
:106E78009385C500E318D6FA130500006780000063
:106E88001305050193850501E31ED6F813050000D7
:106E9800678000009307050003C705009387170064
:106EA80093851500A38FE7FEE31807FE67800000AF
:106EB800930705009387170003C7F7FFE31C07FE36
:106EC8003385A7401305F5FF678000001307050009
:106ED80063140600678000009385150083C6F5FFDC
:106EE800930717001308F6FFA38FD7FE63980600D1
:106EF8003307C700639AE70067800000138707001D
:106F0800130608006FF0DFFC93871700A38F07FEB6
:106F18006FF05FFE130101E32326111C2322911C4D
:106F28002320211D232E311B2322911B9389050029
:106F380093040600938C06002324811C232C411BF8
:106F4800232A511B2328611B2326711B2324811B01
:106F58002320A11B232EB11913090500EFE00F848C
:106F680083270500138507002324F102EFF05FF45F
:106F780083D7C900232AA1002328010C232A010C46
:106F8800232C010C232E010C93F7070863800704B8
:106F980083A70901639C07029305000413050900F0
:106FA800EFE08FAB23A0A90023A8A900631C05006C
:106FB8009307C0002320F9009307F0FF232CF1006A
:106FC8006F00405A9307000423AAF9009307C10EE3
:106FD8002322F10C2326010C2324010C130A0000A0
:106FE80093880700232A0102232801022324010091
:106FF8002322010223260102232C0100138404000A
:107008001307500283470400638407006392E70C68
:10701800B30A9440638A0A048327C10C23A098000A
:1070280023A25801B38757012326F10C8327810C2B
:107038001307700093888800938717002324F10CA6
:10704800635EF7001306410C9385090013050900D8
:10705800EF305068631205509308C10E83278101F1
:10706800B3875701232CF10083470400639407007A
:107078006F109061930714002328F100A303010AFD
:10708800930BF0FF232E010013040000930A9000D5
:10709800130CA0028327010103CB07009387170075
:1070A8002328F10093070BFE1307A0056374F7006C
:1070B8006F10C02D17A700001307C77493972700F8
:1070C800B387E70083A70700B387E7006780070057
:1070D800130414006FF01FF397A7000093878735F8
:1070E800232AF10293770402639407006F10C00B00
:1070F800938C7C0093FC8CFF93878C0003AD0C0071
:1071080083AC4C002326F10093771400638E0700AC
:10711800B3679D01638A0700930700032304F10AFC
:10712800A304610B136424001374F4BF93072000B5
:107138006F0010481305090023221101EFD01FE644
:1071480083274500138507002326F102EFF05FD659
:107158002322A10213050900EFD05FE483278500ED
:10716800832841002324F10083274102E38407F2A6
:1071780083278100E38007F283C70700E38C07F0C9
:10718800136404406FF01FF18347710AE39407F01A
:1071980093070002A303F10A6FF0DFEF13641400F2
:1071A8006FF05FEF83A70C00938C4C00232EF10047
:1071B800E3D207EEB307F040232EF1001364440036
:1071C8006FF05FED9307B0026FF0DFFC83270101DA
:1071D80003CB0700138D170063188B0583AB0C00D6
:1071E80093874C0063D40B00930BF0FF938C07003C
:1071F8002328A1016FF01FEA13850B009305A00057
:1072080023221101130D1D00EF9010428328410025
:10721800034BFDFFB30BB501930D0BFDE3FEBAFD68
:107228002328A1016FF01FE8930B00006FF0DFFE29
:10723800136404086FF01FE6032D0101232E0100DB
:107248000325C1019305A00023221101130B0BFD97
:10725800EF90903D130D1D00B307AB00034BFDFFEE
:10726800232EF1008328410093070BFDE3FAFAFC73
:107278006FF01FFB136484006FF0DFE183270101C7
:1072880003C7070093078006631CF70083270101E3
:1072980013640420938717002328F1006FF09FDF01
:1072A800136404046FF01FDF8327010103C707007D
:1072B8009307C006631CF700832701019387170013
:1072C8002328F100136404026FF0DFDC1364040167
:1072D8006FF05FDC93874C002326F10083A70C0036
:1072E800A303010A2306F11223220100930B1000C5
:1072F800930D0000930C0000130C0000130D000008
:107308009304C1126F00503B136404019377040285
:10731800638E0704938C7C0093FC8CFF93878C000E
:1073280003AD0C0083AC4C002326F10063DE0C0097
:10733800330DA041B337A001B30C9041B38CFC408E
:107348009307D002A303F10A9307F0FFE39CFB68BD
:10735800E39E0C7093079000E3EAA771130D0D03E9
:10736800A307A1199304F1186F00D06D93874C00FF
:107378002326F100937704016388070003AD0C000E
:10738800935CFD416FF09FFA9377040403AD0C0002
:1073980063880700131D0D01135D0D416FF05FFE3B
:1073A80093770420E38E07FC131D8D01135D8D4137
:1073B8006FF01FFD937784006382070C93874C005E
:1073C8002326F10083A70C0003A6070083A6470025
:1073D80003A7870083A7C7002328C10C232AD10C41
:1073E800232CE10C232EF10C1305010D232211018E
:1073F800EFD01FB42326A10A930720008328410059
:107408006314F50C8327010D930501081305010981
:107418002328F1088327410D23200108232201088E
:10742800232AF1088327810D232401082326010834
:10743800232CF1088327C10D232EF108EF60C069C2
:1074480083284100635605009307D002A303F10A7D
:107458009307700497A400009384C4FB63C6670174
:1074680097A400009384C4FA1374F4F7232201004C
:10747800930B3000930D00006F00D05D938C7C005F
:1074880093FC8CFF83A50C0003A64C0093878C000B
:1074980013050109232211012326F100EF90403E34
:1074A80083270109832841002328F10C83274109F8
:1074B800232AF10C83278109232CF10C8327C10986
:1074C800232EF10C6FF05FF2930710006318F5029A
:1074D8008327C10D63D607009307D002A303F10ADF
:1074E8009307700497A40000938444F3E3CE67F7EE
:1074F80097A40000938444F26FF01FF7137CFBFD00
:10750800930710046310FC0A930700032304F10A8D
:1075180013071006930780056314EB009307800791
:10752800A304F10A930730061364240063D2775149
:1075380093851B001305090023221101EFD0DFD129
:107548009304050083284100631A054E83D7C900B8
:1075580093E707042396F90083D7C90093F7070434
:10756800E39C07A48320C11C0324811C03258101FB
:107578008324411C0329011C8329C11B032A811B65
:10758800832A411B032B011B832BC11A032C811A4D
:10759800832C411A032D011A832DC1191301011DD2
:1075A800678000009307F0FF638EFB489307700421
:1075B800232201006314FC00638C0B48832AC10D4D
:1075C800936704102320F102232C0102032E010DDE
:1075D800832D410D032D810D63DA0A00B707008062
:1075E800B3CA57019307D002232CF1029307100462
:1075F8006314FC4A13050109232411052328C10932
:10760800232CA109232AB109232E5109EF90404CBC
:107618001306C10AEFF08FC3138605009305050012
:1076280013050109EF90C0258327010913060106F8
:10763800930501072328F10683274109130501084B
:1076480023200106232AF106832781092322010624
:1076580023240106232CF1068327C109232EF106D2
:10766800B707FC3F2326F106EF60005D03280108F9
:107678000326410883268108032DC10893050108C4
:10768800130501092328010923220105232AC1081A
:107698002320C104232CD108232ED102232EA10993
:1076A8002320010823220108232401082326010896
:1076B800EF60C01F8326C103032601040328410489
:1076C8008328810463160500130710002326E10AA6
:1076D8001307100697AA0000938ACAD56316EB0011
:1076E80097AA0000938ACAD3138EFBFF938D0400D8
:1076F800B7070340930501082322C10813050109B0
:1077080013060107232411052322C105232001099B
:10771800232EF1062324D1082326A10923280106B4
:10772800232A0106232C0106EF60005103260109D4
:1077380083264109130501092320C104232ED10200
:10774800EF80D06593050500130A050013050109AC
:10775800032D8109832CC109EF80907A83270109C1
:10776800032601048326C1032320F1068327410948
:107778002328C106930501072322F10683278109DF
:1077880013060106130501082324F1068327C109FE
:10779800232CA107232E91072326F106232AD1069D
:1077A800EF70900FB3854A0183C50500032E41048D
:1077B800832CC108938D1D0083220108832F410863
:1077C800032F8108232EC103A38FBDFE9307F0FF6B
:1077D800138D0C0083288104630CFE06130EFEFF34
:1077E8009305010813050109232EE105232CF10552
:1077F800232A5104232811052326C10523285108CB
:1078080023245104232AF1092322F105232CE10919
:107818002320E105232E91092320010823220108B2
:107828002324010823260108EF6040088326010469
:107838000326410403288104032EC104832801057B
:1078480083224105832F8105032FC105E31205EA31
:10785800370DFE3F93050108130501092320110583
:107868002328510823265104232AF1092324F1054A
:10787800232CE1092322E105232E91092320010865
:1078880023220108232401082326A109EF60C00E42
:10789800832801046346A0048322C104832F810442
:1078A800032F4104930501081305010923285108F2
:1078B800232AF109232CE109232E91092320010809
:1078C80023220108232401082326A109EF50107E52
:1078D800832801046318051A137A1A0063040A1A24
:1078E80003C6FA00232EB10B930500038326C10BB0
:1078F8009387F6FF232EF10A83C7F6FF6380C71626
:10790800130690036390C71683C7AA00A38FF6FED9
:10791800138A0D0013077004330A9A40032DC10A15
:10792800631EEC2A1307D0FF6344ED0063DAAB3320
:10793800130BEBFF930AFDFF2326510B9376FBFDF8
:10794800930510041377FB0F130600006398B60025
:107958001307F7001377F70F13061000230AE10A3D
:107968009307B00263D80A00930A1000B38AAA41A9
:107978009307D002A30AF10A9307900063D4572B08
:10798800130C310C130D0C00930D90009305A000FF
:1079980013850A0023201103EF9080531305050374
:1079A800A30FACFE9305A00013850A00EF90004AD0
:1079B800930CFCFF930A05008328010263C6AD24DB
:1079C800930A0503130CECFFA38F5CFF9307610B6D
:1079D8006360AC251307410BB387E7402328F10206
:1079E800B38B47019307100063C6470193771400D0
:1079F8006386070083274101B38BFB001374F4BF30
:107A0800936704102320F102930C0000130C00006C
:107A1800130D000083278103638607001307D00234
:107A2800A303E10A03240102930D00006F00C0487C
:107A3800232201009304C1126FF05FB82322A10032
:107A48006FF0DFB723220100930B60006FF01FB7C0
:107A580023227101930B10006FF05FB6A38FB6FE5F
:107A68006FF0DFE89387170093F7F70F6FF01FEABF
:107A7800130A1A00A30FEAFEB3874C41E3DA07FEA4
:107A88006FF05FE98327C103138A0D001307000312
:107A9800B38CFD006FF05FFE93076004630EFC007B
:107AA80093075004938C1B006304FC00938C0B0019
:107AB800130620006F00C000938C0B0013063000E3
:107AC8009307010B1308C10B1307C10A93860C0017
:107AD8009305010913050900232011052328C1096D
:107AE800232EC103232AB109232CA109232E5109CE
:107AF800EFC0CFFF9307700493040500032EC10362
:107B0800832801046316FC00937714006388070A2E
:107B180093076004338A94016312FC0603C70400C8
:107B2800930700036318F704930501081305010977
:107B3800232011052328C109232EC103232AB109B3
:107B4800232CA109232E51092320010823220108EF
:107B58002324010823260108EF505055032EC103A2
:107B6800832801046308050093071000B38C97412C
:107B78002326910B8327C10A330AFA0093050108CB
:107B880013050109232E11032328C109232AB1094A
:107B9800232CA109232E510923200108232201089F
:107BA8002324010823260108EF5050508328C103DD
:107BB80013070003631E0500232E410B032AC10B84
:107BC8006FF05FD593861700232ED10A2380E70034
:107BD8008327C10BE3E847FF6FF05FFE13076004DC
:107BE800E31AECD46352A00763960B0013771400D2
:107BF8006302070C832741013307FD00B38BEB00B9
:107C0800130B60066F004009138C0C006FF01FD82F
:107C1800130C1C000347FCFF93871700A38FE7FE94
:107C28006FF01FDB1307610B63180600930700034F
:107C3800230BF10A1307710B938A0A0393071700A2
:107C4800230057016FF01FD963960B0013771400B8
:107C58006306070683274101138717006FF01FFA91
:107C680063404D0313771400930B0D006306070060
:107C780083274101B30BFD00130B70066F00C00191
:107C880083274101130B7006B30BFA006346A0016A
:107C98003383AB41930B1300137C0440930C000017
:107CA800E30A0CD6130C0000E356A0D79306F00F96
:107CB8006F008003930B0D006FF09FF4130B6006A9
:107CC800930B10006FF05FFD6356A70383278100B5
:107CD800330DED4003C71700630C070293871700A5
:107CE800130C1C002324F1008327810003C707001D
:107CF800E31CD7FC8325410233059C01232E110385
:107D0800EF908012B30B75018328C1036FF09FD0E9
:107D1800938C1C006FF05FFD13874C002326E10055
:107D28001377040283A70C0063000702032781016D
:107D380023A0E7001357F74123A2E700832CC100D3
:107D4800832401016FF08FAB1377040163080700E8
:107D58000327810123A0E7006FF05FFE1377040477
:107D680063080700035781012390E7006FF01FFDA8
:107D780013740420E30E04FC034781012380E70009
:107D88006FF0DFFB13640401937704026388070430
:107D9800938C7C0093FC8CFF93878C0003AD0C00C4
:107DA80083AC4C002326F1001374F4BF9307000042
:107DB800A303010A1307F0FF638CEB4213070400C7
:107DC800B3669D011374F4F76394064263820B5AF9
:107DD800130710006392E7426FF04FD893874C0067
:107DE8002326F100937704016386070003AD0C0096
:107DF8006F000001937704046388070003DD0C001B
:107E0800930C00006FF05FFA93770420E38007FE7D
:107E180003CD0C006FF0DFFE93874C002326F100A2
:107E2800B787FFFF93C707832314F10A97970000CA
:107E38009387075F03AD0C00232AF102930C00001F
:107E48001364240093072000130B80076FF05FF67C
:107E580093874C002326F100A303010A9307F0FF40
:107E68002320110383A40C006386FB0213860B00F6
:107E78009305000013850400EFD09FB02322A100D2
:107E880083280102630805DEB30B95402322010015
:107E98006FF04FDE13850400EFF08F818328010215
:107EA800930B050023220100930D0000930C0000A2
:107EB800130C0000130D00002320B10363D47D01CF
:107EC800232071030347710A63080700832701020F
:107ED800938717002320F102937A240063880A000D
:107EE80083270102938727002320F1029377440810
:107EF800232CF102639807068327C1010327010297
:107F0800338EE7406350C007130F000197AE00009F
:107F1800938E0EA6930F70008326810C23A0D801A0
:107F28000327C10C9386160013868800634ACF473F
:107F38003307EE0023A2C8012326E10C2324D10C29
:107F48001307700093080600635ED7001306410C00
:107F58009385090013050900EF20D077E314056C19
:107F68009308C10E0347710A630807041307710ACF
:107F780023A0E8001307100023A2E8000327C10C80
:107F88009306700093888800130717002326E10CD6
:107F98000327810C130717002324E10C63DEE60096
:107FA8001306410C9385090013050900EF20907210
:107FB800E31A05669308C10E63880A041307810A49
:107FC80023A0E8001307200023A2E8000327C10C20
:107FD8009306700093888800130727002326E10C76
:107FE8000327810C130717002324E10C63DEE60046
:107FF8001306410C9385090013050900EF20906DC5
:10800800E31205629308C10E832781031307000852
:108018006398E7068327C10103270102B38AE74073
:1080280063505007130E000197A7000093874795E8
:10803800930E70008326810C23A0F8000327C10C3F
:10804800938616001386880063485E3B3387EA00F0
:1080580023A258012326E10C2324D10C1307700016
:1080680093080600635ED7001306410C9385090048
:1080780013050900EF201066E316055A9308C10E90
:10808800B38A7D41635050071308000197AD000083
:10809800938D0D8F130E70000327810C23A0B80158
:1080A8008326C10C1307170013868800634E5839BE
:1080B80023A25801B38ADA002326510D2324E10CA8
:1080C800930670009308060063DEE6001306410C71
:1080D8009385090013050900EF20D05FE3140554C8
:1080E8009308C10E13770410832DC10C6312073A4D
:1080F8003383BB0123A0980023A278012326610CB7
:108108008327810C130770009388880093871700D2
:108118002324F10C6352F74C1306410C9385090094
:1081280013050900EF20105BE31E054E9308C10EEE
:108138006F00804A13640401937704026382070284
:10814800938C7C0093FC8CFF93878C0003AD0C0010
:1081580083AC4C002326F100930710006FF05FC535
:1081680093874C002326F100937704016386070068
:1081780003AD0C006F0000019377040463880700C7
:1081880003DD0C00930C00006FF01FFD93770420B3
:10819800E38007FE03CD0C006FF0DFFE9797000029
:1081A800938707286FE0DFF393874C002326F100BD
:1081B800937704016386070003AD0C006F0000018C
:1081C800937704046388070003DD0C00930C000018
:1081D8006FE09FF393770420E38007FE03CD0C0044
:1081E8006FF0DFFE13070400930710006FF05FBD08
:1081F80013071000638EE79413072000638EE712BD
:10820800930701199396DC0113777D00135D3D00F8
:108218001307070333EDA60193DC3C00A38FE7FEA9
:10822800B3669D019384F7FF639E0602937614005C
:10823800638A0600930600036306D700A38FD4FE63
:108248009384E7FF93070119938D0B002322010004
:10825800B38B9740930C0000130C0000130D000023
:108268006FF09FC5938704006FF0DFF9130A0000D1
:10827800930D0119937A0440130C90001306A00083
:108288009306000013050D0093850C0023221101AD
:10829800EF40C02113050503A38FADFE9384FDFFB6
:1082A800130A1A0083284100638E0A048327810079
:1082B80083C707006318FA049307F00F6304FA04EE
:1082C80063940C006370AC05832741028325C102C7
:1082D80023221101B384F440138607001385040098
:1082E800EFE0DFBE83278100130A000083284100E6
:1082F80083C71700638807008327810093871700C7
:108308002324F10013050D0093850C001306A0002B
:108318009306000023221101EF30903B938C050057
:10832800B3E5A500130D050083284100E38C05F093
:10833800938D04006FF09FF4930401190327410300
:108348009377FD009384F4FFB307F70083C7070012
:10835800135D4D002380F4009397CC0133EDA70102
:1083680093DC4C00B3679D01E39A07FC6FF09FED27
:1083780093040119E39807EC13771700E30407EC5B
:1083880093070003A307F1186FE0DFFDE30E0B2E40
:1083980023066113A303010A232691016FE0DFF48A
:1083A8001307070123A2E8012326E10C2324D10C9B
:1083B80063DEDF021306410C9385090013050900EB
:1083C8002324F1052322D1052320E105232EC1030F
:1083D800EF205030E3180524832F8104832E4104B5
:1083E800032F0104032EC1031306C10E130E0EFF43
:1083F800930806006FF05FB21307070123A2C801B4
:108408002326E10C2324D10C63DADE021306410C87
:1084180093850900130509002320D105232EF102B5
:10842800232CC103EF20102BE31E051E832E01040D
:108438008327C103032E81031306C10E938A0AFF03
:10844800930806006FF01FBF9386060123A2080158
:108458002326D10C2324E10C6356EE021306410CAB
:108468009385090013050900232EC103232C01035A
:10847800EF205026E318051A032EC10303288103B1
:108488001306C10E938A0AFF930806006FF0DFC037
:1084980013075006635467730327010D93050108FA
:1084A800130501092328E1080327410D232C110393
:1084B80023200108232AE1080327810D232201082C
:1084C80023240108232CE1080327C10D23260108D2
:1084D800232EE108EF50803D83288103631405189B
:1084E80097970000938747F623A0F800930710009A
:1084F80023A2F8008327810C938D1D002326B10D3C
:10850800938717002324F10C1307700093888800C1
:10851800635EF7001306410C9385090013050900F3
:10852800EF20501BE31005109308C10E8327C10AE2
:1085380063C64701937714006380070A8327810283
:10854800032741019388880023ACF8FE8327410163
:1085580023AEF8FE8327C10CB387E7002326F10C6E
:108568008327810C13077000938717002324F10CCD
:10857800635EF7001306410C938509001305090093
:10858800EF205015E310050A9308C10E9304FAFF73
:1085980063549004130B0001979A0000938A4A3E93
:1085A800130C70008327810C23A058010327C10CEA
:1085B8009387170093868800634A9B0623A2980036
:1085C800B384E4002326910C2324F10C13077000D4
:1085D80093880600E342F7B4137444006314047EDE
:1085E800032BC101832701026354FB00138B07008F
:1085F80083278101B3876701232CF1008327C10CEE
:10860800638C07001306410C9385090013050900C4
:10861800EF20500CE3180500832741002324010CA8
:10862800E39C07049308C10E6FF04FF1130707018D
:1086380023A268012326E10C2324F10C635EFC00CD
:108648001306410C9385090013050900EF209008D3
:10865800631A057C9306C10E938404FF9388060071
:108668006FF05FF40327C10A6346E016979700008E
:10867800938787DD23A0F8009307100023A2F80052
:108688008327810C938D1D002326B10D9387170036
:108698002324F10C1307700093888800635EF700A9
:1086A8001306410C9385090013050900EF20900279
:1086B800631A05769308C10E8327C10A63980700D9
:1086C80063160A0093771400E38807F08327810272
:1086D800032741019388880023ACF8FE83274101D2
:1086E80023AEF8FE8327C10CB387E7002326F10CDD
:1086F8008327810C13077000938717002324F10C3C
:10870800635EF7001306410C938509001305090001
:10871800EF20407C631805709308C10E832AC10AB4
:1087280063D20A06B30A504113870800130C0001EC
:10873800179B0000130BCB24930C70008327810C2C
:10874800232067018326C10C93871700938888002C
:1087580063465C0523225701B38ADA002326510DAC
:108768002324F10C13077000635EF7001306410C15
:108778009385090013050900EF20C0756314056A85
:108788009308C10E8327C10C23A0980023A2480197
:10879800B38747012326F10C6FF09F969386060155
:1087A800232287012326D10C2324F10C63DEFC004D
:1087B8001306410C9385090013050900EF20807109
:1087C800631205669308C10E938A0AFF138708008F
:1087D8006FF0DFF6930A0D006354AA01930A0A00AA
:1087E800635250050327810CB38DBA0123A098006A
:1087F8001307170023A258012326B10D2324E10CE7
:10880800930670009388880063DEE6001306410C27
:108818009385090013050900EF20C06B63140560F8
:108828009308C10E63D40A00930A0000B30A5D419D
:1088380063505007930D0001179B0000130B4B1456
:10884800930B70000327810C23A068018326C10CB9
:10885800130717001386880063C25D1B23A2580103
:10886800B38ADA002326510D2324E10C9306700005
:108878009308060063DEE6001306410C93850900A1
:1088880013050900EF200065631E05589308C10E03
:1088980093770440B38AA40163840702130B700022
:1088A800B38B4401979D0000938D8D0D63140C18B4
:1088B80063940C18B387440163F45701938A070043
:1088C8008327C10A63C6470193771400638A0704A4
:1088D80083278102032741019388880023ACF8FE8F
:1088E8008327410123AEF8FE8327C10CB387E70035
:1088F8002326F10C8327810C130770009387170038
:108908002324F10C635EF7001306410C93850900DC
:1089180013050900EF20005C631605509308C10E8B
:10892800B3844401B38754418324C10AB3049A40F1
:1089380063D4970093840700635490048327C10C81
:1089480023A0580123A29800B387F4002326F10C32
:108958008327810C1307700093888800938717007A
:108968002324F10C635EF7001306410C938509007C
:1089780013050900EF2000566316054A9308C10E37
:108988009387040063D40400930700008324C10A7A
:10899800B3049A40B384F440E35090C4130B00012D
:1089A800979A0000938ACAFD130C70008327810CE4
:1089B80023A058010327C10C9387170093868800CA
:1089C800E35E9BBE1307070123A268012326E10C7F
:1089D8002324F10C635EFC001306410C9385090007
:1089E80013050900EF20004F631E05429306C10ED0
:1089F800938404FF938806006FF05FFB938606015B
:108A080023A2B8012326D10C2324E10C63DEEB005A
:108A18001306410C9385090013050900EF20804BCC
:108A2800631205401306C10E938A0AFF93080600D5
:108A38006FF05FE163820C0E938CFCFF8327C10209
:108A4800032741029388880023ACF8FE832741025C
:108A580023AEF8FE8327C10CB387E7002326F10C69
:108A68008327810C938717002324F10C635EFB0096
:108A78001306410C9385090013050900EF20804572
:108A88006312053A9308C10E8327810033875B413F
:108A980083C707006354F700930707006356F00481
:108AA8000327C10C23A0580123A2F8003387E7004D
:108AB8002326E10C0327810C9388880013071700ED
:108AC8002324E10C6352EB021306410C9385090041
:108AD80013050900232CF102EF20C03F631405346D
:108AE800832781039308C10E1387070063D4070007
:108AF80013070000832781001308000183C70700BC
:108B0800B387E7406346F0068327810083C70700E1
:108B1800B38AFA006FF09FD983278100130CFCFFFA
:108B28009387F7FF2324F1006FF05FF19386060126
:108B380023A208012326D10C2324E10C6356EB025F
:108B48001306410C9385090013050900232E010320
:108B5800232CF102EF2000386316052C0328C103EB
:108B6800832781031306C10E938707FF9308060026
:108B78000327810C23A0B8018326C10C1307170013
:108B880013868800E344F8FA23A2F800B387D700D5
:108B98002326F10C2324E10C93080600E356EBF698
:108BA8001306410C9385090013050900EF20803254
:108BB800631A05269308C10E6FF01FF58327810CF1
:108BC8001307100023A09800938D1D0093871700AA
:108BD800138B880063464701937614006388061C4C
:108BE8001307100023A2E8002326B10D2324F10C5B
:108BF80013077000635EF7001306410C93850900A4
:108C080013050900EF20002D631E0520130BC10E6C
:108C18008327810203274101130B8B00232CFBFEC2
:108C280083274101232EFBFE8327C10CB387E7006E
:108C38002326F10C8327810C1307700093871700F4
:108C48002324F10C635EF7001306410C9385090099
:108C580013050900EF2000286316051C130BC10E2D
:108C68008327010D93050108130501092328F1083D
:108C78008327410D930AFAFF23200108232AF108CC
:108C88008327810D2322010823240108232CF108BE
:108C98008327C10D23260108232EF108EF40104138
:108CA800630605088327C10C0327810C93841400ED
:108CB8009387F7FFB38747011307170023209B000B
:108CC80023225B012326F10C2324E10C9307700077
:108CD800130B8B0063DEE7001306410C9385090034
:108CE80013050900EF20001F631E0512130BC10EA8
:108CF8009307410B2320FB0083270103032701036C
:108D080093088B002322FB008327C10CB387E7005D
:108D18002326F10C8327810C130770009387170013
:108D28002324F10CE35AF78A6FF00FBFE35250FD8A
:108D3800130C000197940000938484C4930C700072
:108D48000327810C23209B008327C10C13071700DE
:108D580093068B0063405C03B387FA0023225B0110
:108D68002326F10C2324E10C93077000138B0600D3
:108D78006FF05FF69387070123228B012326F10CFE
:108D88002324E10C63DEEC001306410C93850900F3
:108D980013050900EF200014631605089306C10E99
:108DA800938A0AFF138B06006FF09FF923A2E8004D
:108DB8002326B10D2324F10C13077000E35AF7F2B0
:108DC8006FF09FF18327C101032701023384E74035
:108DD800E3588080930A000197940000938444B973
:108DE800130B70008327810C23A098000327C10C64
:108DF8009387170063C68A0423A288003304E4001B
:108E08002326810C2324F10C13077000635AF7FC06
:108E18001306410C9385090013050900EF20800B08
:108E2800630005FC83274100639407006FE0CFF2DD
:108E38009385070013050900EF901FD26FE0CFF16B
:108E48001307070123A258012326E10C2324F10C60
:108E580093888800635EFB001306410C9385090024
:108E680013050900EF200007E31E05FA9308C10E59
:108E7800130404FF6FF01FF7832541001305090051
:108E8800EF909FCD6FF00FFA8327C10C6394070012
:108E98006FE08FEC1306410C938509001305090058
:108EA800EF2040036FE04FEB83278600130101FD9D
:108EB8002324810223261102232291022320210345
:108EC800232E3101232C4101232A5101232861013A
:108ED800232671012324810113040600639E0702DF
:108EE80023220600130500008320C1020324810207
:108EF80083244102032901028329C101032A810134
:108F0800832A4101032B0101832BC100032C81001B
:108F1800130101036780000083A745061389050034
:108F280013972701635A070683240600130A0500CE
:108F3800930BF0FF83278400639A07001305000052
:108F480023240400232204006FF01FFA83A944009D
:108F580003AB0400930A000013DC290063CE8A01E6
:108F68008327840093F9C9FF93848400B389374128
:108F7800232434016FF01FFC83250B00130609001E
:108F880013050A00EF100014130B4B00630A750158
:108F9800938A1A006FF09FFCEF1040206FF05FFA81
:108FA8001305F0FF6FF0DFF9130101ED232481129F
:108FB800232E3111232C41112320A1112326111214
:108FC8002322911223202113232A511123286111CE
:108FD800232671112324811123229111232EB10FED
:108FE8009309050013840500130A0600138D060073
:108FF800630805008327850363940700EF901F88A3
:109008008317C4001397270163420702B72600009D
:1090180003274406B3E7D7002316F400B7E7FFFF9A
:109028009387F7FFB377F7002322F4068357C4002A
:1090380093F78700638E070683270401638A070670
:109048008357C4001307A00093F7A7016390E708AC
:109058008317E40063CC070693060D0013060A0085
:109068009305040013850900EF00903F2322A10017
:109078008320C11203248112032541008324411255
:10908800032901128329C111032A8111832A41115D
:10909800032B0111832BC110032C8110832C411049
:1090A800032D0110832DC10F1301011367800000E8
:1090B8009305040013850900EF90CFACE30205F88F
:1090C8009307F0FF2322F1006FF09FFA930BC1047E
:1090D800232071052324010423220104938D0B000E
:1090E800232601002324010023280100232A01004C
:1090F8002322010093040A009306500283C7040048
:10910800638407006396D70A33894441630A0904D4
:109118008327810423A04D0123A22D01B3872701B2
:109128002324F1048327410493067000938D8D0056
:10913800938717002322F10463DEF6001306010467
:109148009305040013850900EFF01FD6E31A0528DC
:10915800938D0B0083274100B38727012322F10059
:1091680083C70400E382072C138A1400A30D0102AD
:109178001309F0FF130B0000130C00009304A00266
:10918800930AA00503460A00130A1A00930606FE6E
:10919800E3E2DA0E978700009387877F939626008D
:1091A800B386F60083A60600B386F600678006003D
:1091B800938414006FF09FF49787000093878727A4
:1091C8002326F10093760C02638C066C130D7D0048
:1091D800137D8DFF83280D00832A4D00930C8D008D
:1091E80093761C00638E0600B3E65801638A060076
:1091F80093060003230ED102A30EC102136C2C00A8
:10920800137CFCBF6F00403413850900EFB01FD9F1
:109218008327450013850700232AF100EFD05FC993
:109228002328A10013850900EFB05FD783278500A5
:109238002324F10083270101E38407F483278100B5
:10924800E38007F483C60700E38C06F2136C0C4036
:109258006FF01FF38346B103E39406F2930600020E
:10926800A30DD1026FF0DFF1136C1C006FF05FF1FA
:10927800032B0D00130D4D00E3540BF0330B60412D
:10928800136C4C006FF0DFEF9306B0026FF05FFDD8
:1092980003460A00930C1A006316960403290D006E
:1092A80093064D00635409001309F0FF138D06005F
:1092B800138A0C006FF0DFEC130509009305A0007A
:1092C800EF709036938C1C0003C6FCFF33094501F0
:1092D800130A06FD93079000E3F047FF138A0C007A
:1092E8006FF0DFEA130900006FF09FFE136C0C08A3
:1092F8006FF01FE9930C0A00130B000013050B0015
:109308009305A000232CC100EF70103203268101C1
:10931800938C1C0093079000130B06FD03C6FCFFFB
:10932800330BAB00930606FDE3FAD7FC6FF01FFB87
:1093380003460A00930680066318D600130A1A002B
:10934800136C0C206FF0DFE3136C0C046FF05FE319
:1093580003460A009306C0066318D600130A1A00CB
:10936800136C0C026FF0DFE1136C0C016FF05FE11E
:1093780083260D00930C4D00A30D01022306D1088E
:1093880013091000930A00009304C1086F00401FDE
:10939800136C0C0193760C02638C0604130D7D008C
:1093A800137D8DFF83280D00832A4D00930C8D00BB
:1093B80063DE0A00B3081041B3361001330350418D
:1093C800B30AD3409306D002A30DD1029306F0FF4F
:1093D8006314D950639E0A569307900063EA17579F
:1093E80093880803A307110F9304F10E6F00C0546C
:1093F80093760C01930C4D006388060083280D00BA
:1094080093DAF8416FF0DFFA93760C0483280D00A5
:10941800638806009398080193D808416FF05FFEAF
:1094280093760C20E38E06FC9398880193D88841A4
:109438006FF01FFD13760C0283260D00130D4D00EF
:10944800630C06008327410023A0F60093D7F74159
:1094580023A2F6006FF01FCA13760C0163080600FA
:109468008327410023A0F6006FF0DFC813760C04B1
:1094780063080600835741002390F6006FF09FC7EA
:1094880093770C20E38E07FC834741002380F60086
:109498006FF05FC6136C0C0193760C0263860604AA
:1094A800130D7D00137D8DFF83280D00832A4D0049
:1094B800930C8D00137CFCBF93060000A30D0102E2
:1094C8001306F0FF6300C94213060C00B3E5580108
:1094D800137CFCF7639805406300095813061000D5
:1094E8006396C6406FF0DFEF93760C01930C4D0046
:1094F8006386060083280D006F00000193760C0434
:109508006388060083580D00930A00006FF09FFAE5
:1095180093760C20E38006FE83480D006FF0DFFE93
:10952800B786FFFF83280D0093C606839787000040
:10953800938707EF930C4D00930A0000136C2C00DF
:10954800231ED1022326F100930620006FF01FF797
:10955800A30D01029306F0FF930C4D0083240D0028
:109568006300D92C13060900930500001385040035
:10957800EFC00FC1930A000063040500330995404A
:10958800138D0A0063D42A01130D09008346B10321
:1095980063840600130D1D0093772C00232CF10023
:1095A80063840700130D2D0093774C08232EF100D8
:1095B80063940706B306AB416350D00693080001D5
:1095C800178800001308885313037000032641040A
:1095D80023A00D01832581041306160013858D0031
:1095E80063C4D84A23A2DD00B386B6002324D1047D
:1095F8002322C10493067000930D050063DEC600A4
:10960800130601049305040013850900EFF0DF89B0
:109618006318055C938D0B008346B10363880604C9
:109628001306B10323A0CD001306100083264104BE
:1096380023A2CD0003268104938616002322D10499
:10964800130616002324C10413067000938D8D00A1
:10965800635ED60013060104930504001385090010
:10966800EFF09F84631E0556938D0B0083278101BD
:10967800638807041306C10323A0CD001306200046
:109688008326410423A2CD00032681049386160075
:109698002322D104130626002324C10413067000D4
:1096A800938D8D00635ED6001306010493050400B4
:1096B80013850900EFF04FFF63140552938D0B00DB
:1096C8008327C101930600086394D706B306AB410C
:1096D8006350D00693080001178800001308084358
:1096E800130370000326410423A00D018325810480
:1096F8001306160013858D0063C4D83E23A2DD002F
:10970800B386B6002324D1042322C1049306700033
:10971800930D050063DEC6001306010493050400DB
:1097280013850900EFF04FF8631C054A938D0B0071
:10973800B38A2A4163505007930800011788000034
:109748001308C83C130370008326410423A00D01AD
:10975800032681049386160093858D0063CE583DB9
:1097680023A25D01B38ACA00232451052322D10410
:1097780013067000938D0500635ED600130601047E
:109788009305040013850900EFF00FF2631A0544EE
:10979800938D0B008326810423A22D0123A09D0015
:1097A80033892601832641042324210513067000EA
:1097B800938616002322D10413878D00635ED6009A
:1097C800130601049305040013850900EFF0CFED9B
:1097D8006318054013870B0093774C006396073A8C
:1097E8006354AB01130B0D0083274100B387670156
:1097F8002322F10083278104638C070013060104E8
:109808009305040013850900EFF00FEA631A053C7D
:1098180023220104138D0C00938D0B006FF09F8D94
:1098280013850400EFD0CFE813090500930A000060
:109838006FF01FD5136C0C0193760C02638006023F
:10984800130D7D00137D8DFF83280D00832A4D00A5
:10985800930C8D00930610006FF05FC693760C0191
:10986800930C4D006386060083280D006F000001ED
:1098780093760C046388060083580D00930A000051
:109888006FF05FFD93760C20E38006FE83480D00A1
:109898006FF0DFFE97870000938787B86FF05F92BD
:1098A80093760C01930C4D006386060083280D0007
:1098B8006F00000193760C046388060083580D003E
:1098C800930A00006FF0DF9193760C20E38006FE88
:1098D80083480D006FF0DFFE13060C00930610009E
:1098E8006FF0DFBE13061000E386C6AE1306200035
:1098F8006388C6129306010F9395DA0113F6780070
:1099080093D8380013060603B3E8150193DA3A0032
:10991800A38FC6FEB3E558019384F6FF639605024C
:1099280093751C00638A0500930500036306B6005F
:10993800A38FB4FE9384E6FF9307010F930A0900EF
:10994800338997406FF0DFC3938604006FF0DFFA26
:1099580093770C40130D0000130E010F232CF10018
:10996800138508001306A0009306000093850A00DB
:109978009304FEFF2320C103232E1101EF2010338F
:10998800032E01028327810113050503A30FAEFEF1
:10999800130D1D008328C101638E070483278100EE
:1099A80083C607006398A6059307F00F6304FD04B8
:1099B80063960A009307900063FE1703832701014B
:1099C80083254101232E1101B384F4401386070037
:1099D80013850400EFD08FCF83278100130D00007B
:1099E8008328C10183C61700638606009387170082
:1099F8002324F1001385080093850A001306A000AC
:109A080093060000EF20C04C938A0500B3E5A5003B
:109A180093080500E38205F2138E04006FF05FF4EB
:109A28009304010F8327C10093F6F8009384F4FF91
:109A3800B386D70083C6060093D848002380D40095
:109A48009396CA01B3E8160193DA4A00B3E65801BF
:109A5800E39A06FC6FF05FEE9304010FE39E06ECB9
:109A680013761600E30A06EC93060003A307D10E4B
:109A78006FF09F97630A061A2306C108A30D010217
:109A8800930C0D006FF0DF8F9385050123A21D0154
:109A98002324B1042322C104635EC3021306010414
:109AA800930504001385090023266102232401037A
:109AB800232211032320D102EFF00FBF63120512F6
:109AC8000323C1020328810283284102832601025D
:109AD80013850B00938606FF930D05006FF01FAFEB
:109AE8009385050123A21D012324B1042322C10467
:109AF800635EC3021306010493050400138509007D
:109B08002322610223200103232E1101232CD100DB
:109B1800EFF08FB96316050C0323410203280102F5
:109B28008328C1018326810113850B00938606FFD4
:109B3800930D05006FF01FBB1306060123A21D013C
:109B48002324C1042322D104635AD3021306010437
:109B5800930504001385090023206102232E0101C7
:109B6800232C1101EFF04FB4631C050603230102F7
:109B78000328C1018328810193850B00938A0AFF7A
:109B8800938D05006FF05FBCB304AB41E35A90C4FA
:109B9800930A000117890000130949F6130C700095
:109BA80083274104232027018326810493871700F4
:109BB80063C09A0423229700B384D4002324910419
:109BC8002322F10413077000E35CF7C013060104B5
:109BD8009305040013850900EFF00FADE30205C0FB
:109BE8008357C40093F70704638407C86FF04FCD09
:109BF80093860601232257012324D1042322F1044A
:109C080013078700635EFC00130601049305040034
:109C180013850900EFF04FA9E31405FC13870B0027
:109C2800938404FF6FF0DFF783278104E38A07FA40
:109C3800130601049305040013850900EFF0CFA66D
:109C48006FF01FFA979700009387C7EB93060600FB
:109C5800138605009305050003A507006FF0CFB430
:109C680083D7C500130101B8232C814693F7D7FF8A
:109C7800231AF10083A7450613840500232A914679
:109C88002326F10683D7E50023282147232E1146F2
:109C9800231BF10083A7C501130905002320010236
:109CA8002322F10283A74502930581002326F102AE
:109CB800930701072324F100232CF10093070040A8
:109CC8002328F100232EF100EFF00FAE93040500D6
:109CD800634C05009305810013050900EF80DF9EA2
:109CE800630405009304F0FF8357410193F70704C9
:109CF800638807008357C40093E707042316F4001A
:109D08008320C147032481471385040003290147A1
:109D1800832441471301014867800000979700009A
:109D2800938747DE83A7070083A747036396070047
:109D3800979700009387878503A3070E67000300A2
:109D4800638405029307F00F63FAC7009307A0081E
:109D58002320F5001305F0FF678000002380C5006D
:109D680013051000678000001305000067800000DD
:109D7800130101FF23248100130405001385050046
:109D880093050600138606009797000023A007DCBA
:109D980023261100EF7080419307F0FF631CF50044
:109DA80097970000938787DA83A7070063840700E3
:109DB8002320F4008320C100032481001301010142
:109DC80067800000130101FF2324810013040500AC
:109DD800138505009305060023261100EF70C004C3
:109DE8009305050013050400EFB00FC71304050021
:109DF800630205040326C5FF130740021376C6FF56
:109E08001306C6FF6362C706930630019307050071
:109E180063FCC60023200500232205009307B00138
:109E280063E4C7029307850023A0070023A2070065
:109E380023A40700130504008320C1000324810024
:109E48001301010167800000232405002326050073
:109E580093070501E31AE6FC23280500930785010B
:109E6800232A05006FF05FFC93050000EFB09FB355
:109E78006FF05FFC130101FF232481001304050028
:109E8800138505009797000023A207CC232611000D
:109E9800EF70C00B9307F0FF631CF5009797000065
:109EA8009387C7CA83A70700638407002320F400A9
:109EB8008320C10003248100130101016780000091
:109EC800130101FF2326110023248100232291007E
:109ED8002320210163920502130900008320C10099
:109EE800032481001305090083244100032901008C
:109EF8001301010167800000930405001384050025
:109F0800630805008327850363940700EF801F9784
:109F18008317C400E38207FC93050400138504003B
:109F2800EF800FDA8327C40213090500638C07004A
:109F38008325C40113850400E780070063540500E6
:109F48001309F0FF8357C40093F7070863880700D5
:109F58008325040113850400EF801FC083250403B3
:109F6800638C0500930704046386F50013850400D9
:109F7800EF809FBE232804028325440463880500DC
:109F880013850400EF805FBD23220404EF805FA6E1
:109F980023160400EF801FA66FF05FF49797000068
:109FA800938747B69305050003A507006FF05FF197
:109FB800130101FD2324810223229102232C410154
:109FC8002326110223202103232E3101232A5101A4
:109FD80023286101130A0500938405001304060071
:109FE800EFB04F8893071000631AF5049387F4FFC6
:109FF8001307E00F6364F704230691009309100028
:10A0080013090000930AF0FF130BA000631239072D
:10A01800138504008320C1020324810283244102A2
:10A02800032901028329C101032A8101832A4101ED
:10A03800032B010113010103678000009306C40587
:10A04800138604009305C10013050A00EF10905D04
:10A058009307F0FF93090500E314F5FA8357C4004A
:10A0680093E707042316F4001305F0FF6FF09FFA37
:10A078009307C100B387270183C50700832784009E
:10A088009387F7FF2324F40063D80700032784018C
:10A0980063C0E702638E65018327040013871700F6
:10A0A8002320E4002380B700130919006FF01FF67E
:10A0B8001306040013050A00EF105042E31655FF7B
:10A0C8006FF09FFA8317C6001397270163400702B2
:10A0D80003274606B7260000B3E7D7002316F60085
:10A0E800B7270000B367F7002322F6066FF05FEC8E
:10A0F800130101FE979700009387C7A0232C8100C6
:10A1080003A40700232A9100232E110093040500BD
:10A1180013860500630E040083278403639A0700EF
:10A12800130504002326B100EF804FF50326C10074
:10A1380013050400032481018320C10193850400D1
:10A1480083244101130101026FF0DFF7130101FFBE
:10A1580023248100130405001385050093050600D8
:10A168009797000023A4079E23261100EF605063F1
:10A178009307F0FF631CF500979700009387079DEE
:10A1880083A70700638407002320F4008320C1000D
:10A1980003248100130101016780000083278600E2
:10A1A8006398070093070000138507006780000085
:10A1B80083D7C500130101FC232C81022328210326
:10A1C80023206103232E1102232A9102232631031F
:10A1D8002324410323225103232E7101232C8101BF
:10A1E800232A91012328A1012326B10193F787008F
:10A1F800130B060013840500130905006382070E7C
:10A2080083A70501638E070C8357C400032A0B003C
:10A2180013F72700631A071693F71700930B00002C
:10A22800638A072013050000930A000093090000C1
:10A238006386093663120502138609009305A00098
:10A2480013850A00EFB0CFF3938B1900630605005E
:10A2580013051500B30B5541138C0B0063F47901FA
:10A26800138C090003250400832704018326440175
:10A2780063F0A73483248400B384960063DA8433BC
:10A2880093850A0013860400EF000050832704001A
:10A298009305040013050900B38797002320F400F1
:10A2A800EF808FC2631E0516B38B9B401305100009
:10A2B800639A0B009305040013050900EF80CFC0D3
:10A2C8006310051683278B00B38A9A00B3899940D7
:10A2D800B384974023249B00E39C04F46F0080061A
:10A2E8009305040013050900EF80CF899307F0FF59
:10A2F800E30C05F06F00400583290A0083244A0017
:10A30800130A8A00E38A04FE9386040063F49A0021
:10A3180093860A00832744028325C4011386090013
:10A3280013050900E7800700635CA00E83278B00F4
:10A33800B389A900B384A4403385A7402324AB0084
:10A34800E31205FC930700008320C1030324810363
:10A3580083244103032901038329C102032A8102BB
:10A36800832A4102032B0102832BC101032C8101A3
:10A37800832C4101032D0101832DC10013850700A2
:10A388001301010467800000B70A008093090000E8
:10A398009304000093CA0AC06FF0DFF6832B0A000B
:10A3A80083244A00130A8A00E38A04FE8359C400FE
:10A3B800832D84000325040093F709206384071480
:10A3C80063E0B40D93F70948638C070A832D0401F1
:10A3D80093053000330DB54103254401EF60D024C7
:10A3E800935AF501B38AAA0093071D0093DA1A401D
:10A3F800B387970063F4FA00938A070093F909403A
:10A408006388090C93850A0013050900EFA0DFE4AF
:10A4180093090500631A05029307C0002320F90079
:10A428008357C40093E707042316F4009307F0FF4B
:10A438006FF09FF1370C0080934CECFF9304000001
:10A44800134CFCFF6FF05FF68325040113060D0023
:10A45800EF0000258357C40093F7F7B793E7070881
:10A468002316F40023283401232A5401B389A901AF
:10A47800B38AAA4123203401938D04002324540174
:10A488009389040063F4B401938D04000325040048
:10A4980013860D0093850B00EF00002F832784009F
:10A4A800B387B7412324F40083270400B38DB70191
:10A4B8002320B40183278B00B38B3B01B384344141
:10A4C800B389374123243B01E39009EE6FF09FE7FE
:10A4D80013860A0093850D0013050900EF00403527
:10A4E80093090500E31005F8832504011305090005
:10A4F800EF808FE68357C40093F7F7F72316F4002D
:10A508006FF09FF18327040163E6A70083294401C4
:10A5180063F6340593890D0063F4B401938904004C
:10A528001386090093850B00EF000026832784001B
:10A5380003270400B3873741330737012324F40086
:10A548002320E400E39807F69305040013050900A7
:10A55800EF808F97E30005F66FF09FEC13050C0072
:10A5680063E49C001385040093850900EF60100ED6
:10A5780093850900EF60500B832744028325C401AB
:10A588009306050013860B0013050900E7800700F2
:10A5980093090500E340A0F26FF09FE8832A0A00C0
:10A5A80083294A0013050000130A8A006FF05FC868
:10A5B8006342DC02832744028325C40113860A0010
:10A5C80013050900E780070093040500E34EA0CCBB
:10A5D8006FF01FE513060C0093850A00EF00C01A00
:10A5E8008327840093040C00B38787412324F40055
:10A5F80083270400B38787012320F4006FF0DFCAA4
:10A60800130101FF232481001304050013850500AD
:10A618009787000023AC075223261100EF60101F14
:10A628009307F0FF631CF500978700009387075294
:10A6380083A70700638407002320F4008320C10058
:10A64800032481001301010167800000130101FF49
:10A6580023248100130405001385050093050600D3
:10A66800138606009787000023A2074E23261100B1
:10A67800EF60D01C9307F0FF631CF500978700007C
:10A688009387C74C83A70700638407002320F4003F
:10A698008320C100032481001301010167800000A9
:10A6A800B3C7A50093F737003307C50063960700C3
:10A6B8009307300063E4C70293070500636CE50065
:10A6C8006780000083C605009387170093851500EF
:10A6D800A38FD7FEE3E8E7FE678000009377350095
:10A6E80063920708930705009376C7FF138606FE53
:10A6F80063F6C70883A3050083A2450083AF8500DE
:10A7080003AFC50083AE050103AE450103A3850170
:10A7180083A8C501938545029387470203A8C5FF0F
:10A7280023AE77FC23A057FE23A2F7FF23A4E7FF5D
:10A7380023A6D7FF23A8C7FF23AA67FE23AC17FFCA
:10A7480023AE07FF6FF0DFFA83C605009387170073
:10A7580093851500A38FD7FE93F63700E39606FE80
:10A768006FF09FF8930705006FF01FFF03A6050021
:10A77800938747009385450023AEC7FEE3E8D7FEDD
:10A78800E3EAE7F4678000003307C50063E8A50043
:10A7980093070500639AE70267800000B387C50046
:10A7A8003306F640E376F5FEB386C70063940600E9
:10A7B800678000009387F7FF83C607001307F7FF3A
:10A7C8002300D7006FF05FFE9385150083C6F5FF61
:10A7D80093871700A38FD7FE6FF0DFFB130101FFEC
:10A7E8002324810013040500138505009305060042
:10A7F800138606009787000023AA07342326110032
:10A80800EF6090089307F0FF631CF500978700003E
:10A818009387C73383A70700638407002320F400C6
:10A828008320C10003248100130101016780000017
:10A83800130101FC232C8102232E1102138405002D
:10A84800232A9102232821032326310323244103A9
:10A858002322510323206103232E7101930506004F
:10A8680063180402032481038320C1038324410362
:10A87800032901038329C102032A8102832A410291
:10A88800032B0102832BC101130101046FA0DF9C7C
:10A89800930A05002326C100EFB08F9E8325C100CF
:10A8A8008326C4FF930760019389B500930B84FF47
:10A8B80013F9C6FF63F4370513FB89FF63520B04D2
:10A8C8009307C00023A0FA00130A00008320C103E5
:10A8D8000324810313050A00832441030329010388
:10A8E8008329C102032A8102832A4102032B010220
:10A8F800832BC1011301010467800000130B0001C1
:10A90800E360BBFC635E6945178700001307C7DE79
:10A9180003268700B3872B0103A74700630CF600C3
:10A928001375E7FF3385A700032545001375150048
:10A93800631C050A1377C7FFB309E9006312F6041D
:10A9480013050B0163C6A90AB38B6B01B38969416F
:10A958009787000023A677DB93E9190023A23B0120
:10A968008329C4FF13850A00130A040093F9190008
:10A97800B3E96901232E34FFEFB0CF906FF01FF5D4
:10A9880063C8690703A7C70083A7870023A6E70052
:10A998002324F70003A74B00B38669411306F00090
:10A9A80013771700B3873B016370D63CB369EB009C
:10A9B80023A23B01B3856B0193E6160023A2D500C1
:10A9C80003A747009385850013850A0013671700BE
:10A9D80023A2E700EF804F9813850A00EFB08F8A13
:10A9E800138A8B006FF09FEE130700009307000097
:10A9F80093F6160063940628832484FFB3849B404F
:10AA080003AA4400137ACAFF330A2A01638E071A7D
:10AA1800B30947016318F60E93070B0163C6F91AC9
:10AA280003A7840083A7C4001306C9FF138A840000
:10AA38002326F70023A4E70013074002636CC70A24
:10AA48009306300193070A0063F2C60283270400C5
:10AA580023A4F4008327440023A6F4009307B0013D
:10AA680063ECC704130484009387040103270400DC
:10AA780023A0E7000327440023A2E700032784005C
:10AA880023A4E700B3876401B389694117870000ED
:10AA98002328F7C693E9190023A2370183A74400A6
:10AAA80093F71700B3E9670123A2340113850A005D
:10AAB800EFA05FFD6FF09FE18327840023A8F400D7
:10AAC8008327C40023AAF4006308E60013040401E2
:10AAD800938784016FF09FF983270401130484018D
:10AAE80023ACF4000327C4FF9387040223AEE400D9
:10AAF8006FF0DFF79305040013050A00EFF0DFC8D5
:10AB08006FF05FF863C2690D03A7C70083A78700CA
:10AB18001306C9FF1385840023A6E7002324F70042
:10AB280003A7840083A7C4002326F70023A4E70013
:10AB38009307400263E4C708130730016372C70232
:10AB48000327040023A4E4000327440023A6E40009
:10AB58001307B0016366C702130484001385040158
:10AB6800832704002320F500832744002322F500CF
:10AB7800832784002324F500938B04006FF09FE162
:10AB88000327840023A8E4000327C40023AAE400C1
:10AB98006308F60013040401138584016FF05FFC59
:10ABA80083270401138504021304840123ACF400F1
:10ABB8008327C4FF23AEF4006FF09FFA93050400C7
:10ABC800EFF09FBC6FF05FFB634A6A0B83A7C4007A
:10ABD80003A784001306C9FF138584002326F70002
:10ABE80023A4E7009307400263E4C7081307300172
:10ABF8006372C7020327040023A4E4000327440068
:10AC080023A6E4001307B0016366C7021304840097
:10AC180013850401832704002320F50083274400BB
:10AC28002322F500832784002324F50093090A00D2
:10AC38006FF09FF40327840023A8E4000327C400CF
:10AC480023AAE4006308F6001304040113858401B1
:10AC58006FF05FFC83270401138504021304840149
:10AC680023ACF4008327C4FF23AEF4006FF09FFAEF
:10AC780093050400EFF05FB16FF05FFB13850A00E6
:10AC8800EFA08FDD130A0500E30205E28327C4FF66
:10AC9800130785FF93F7E7FFB387FB00639AE70085
:10ACA8008329C5FF93F9C9FFB38929016FF09FCEA6
:10ACB8001306C9FF9307400263EEC7081307300164
:10ACC8006374C708032704002320E5000327440012
:10ACD8002322E5001307B001636AC7021307840043
:10ACE800930785008326070023A0D7008326470003
:10ACF80023A2D7000327870023A4E70093050400B5
:10AD080013850A00EF705FE56FF05FDA03278400B0
:10AD18002324E5000327C4002326E5006308F60082
:10AD280013070401930705016FF0DFFB8327040174
:10AD3800130784012328F50083264401930785011E
:10AD4800232AD5006FF01FFA9307050013070400A4
:10AD58006FF05FF993050400EFF01FA36FF01FFA7F
:10AD6800930909006FF01FC3B3E9E90023A23B016F
:10AD780003A747001367170023A2E7006FF0DFC59A
:10AD8800130101FF232481001384050083A5050016
:10AD980023229100232611009304050063840500F3
:10ADA800EFF01FFE93050400032481008320C100F7
:10ADB8001385040083244100130101016F70DFD95A
:10ADC80097870000938707D483A707006382A7109B
:10ADD8008327C504130101FE232C8100232A910037
:10ADE80023282101232E11002326310113040500F5
:10ADF80093040000130900086394070483250404DE
:10AE08006386050013050400EF701FD5832584149D
:10AE1800638C05049304C4146388950403A905008E
:10AE280013050400EF705FD3930509006FF0DFFE90
:10AE3800B385950083A50500639E050093844400AF
:10AE48008325C404E39624FF13050400EF70DFD0C4
:10AE58006FF0DFFA83A9050013050400EF70DFCF58
:10AE6800938509006FF05FFD83254405638605001F
:10AE780013050400EF705FCE83278403638C0702F9
:10AE88008327C40313050400E78007008325042EE5
:10AE98006382050213050400032481018320C10194
:10AEA80083244101032901018329C10013010102FF
:10AEB8006FF01FED8320C101032481018324410128
:10AEC800032901018329C1001301010267800000E1
:10AED8006780000083278600130101FD232E3101BE
:10AEE80023261102232481022322910223202103F5
:10AEF800232C4101232A51012328610123267101B2
:10AF080023248101232291019309060063860712F5
:10AF1800032B0600930A050013840500930B000019
:10AF28001309000063060908032A84006366490DB3
:10AF3800835CC40093F70C486380070C0325440125
:10AF480083240400032A040193053000EF50D06DD8
:10AF5800338C44419354F501B384A40093071C0037
:10AF680093D41440B387270163F4F4009384070053
:10AF780093FC0C4063800C109385040013850A0031
:10AF8800EFA08FAD130A0500631C05029307C000EC
:10AF980023A0FA008357C4001305F0FF93E70704C2
:10AFA8002316F40023A4090023A209006F00400916
:10AFB800832B0B0003294B00130B8B006FF09FF6BC
:10AFC8008325040113060C00EFF08FED8357C400AE
:10AFD80093F7F7B793E707082316F40023284401EB
:10AFE800232A9400330A8A01B3848441232044012C
:10AFF80023249400130A090063744901130A090001
:10B008000325040013060A0093850B00EFF0CFF721
:10B0180083278400B38747412324F400832704004F
:10B02800338A470183A789002320440133892741B4
:10B0380023A42901E31E09F623A209001305000031
:10B048008320C102032481028324410203290102CF
:10B058008329C101032A8101832A4101032B0101AC
:10B06800832BC100032C8100832C410013010103B1
:10B078006780000093050A001386040013850A0000
:10B08800EFF00FFB130A0500E31A05F4832504010A
:10B0980013850A00EF705FAC6FF05FEF83D7C500D0
:10B0A800130101ED23202113232E3111232C4111EB
:10B0B8002320A11123261112232481122322911265
:10B0C800232A511123286111232671112324811168
:10B0D80023229111232EB10F93F70708130A0500B5
:10B0E8001389050093090600138D0600638E070275
:10B0F80083A70501639A070293050004EFA0CF9583
:10B108002320A9002328A900631C05009307C00079
:10B118002320FA009307F0FF2322F1006F00D032BA
:10B1280093070004232AF900930BC1042320710517
:10B138002324010423220104938D0B0023260100FC
:10B148002324010023280100232A010023220100CF
:10B1580013840900930650028347040063840700A0
:10B168006396D70AB3043441638A040483278104AD
:10B1780023A03D0123A29D00B38797002324F10457
:10B188008327410493067000938D8D0093871700E1
:10B198002322F10463DEF600130601049305090077
:10B1A80013050A00EFF01FD3E31A0528938D0B004F
:10B1B80083274100B38797002322F10083470400C7
:10B1C800E380073093091400A30D01029304F0FFF4
:10B1D800130B0000130C00001304A002930AA0052F
:10B1E80003C6090093891900930606FEE3E2DA0E06
:10B1F800977700009387C7A293962600B386F60038
:10B2080083A60600B386F6006780060013041400C0
:10B218006FF09FF4976700009387C7212326F100FA
:10B2280093760C02638C066C130D7D00137D8DFFE5
:10B2380083280D00832A4D00930C8D0093761C0003
:10B24800638E0600B3E65801638A0600930600037E
:10B25800230ED102A30EC102136C2C00137CFCBF79
:10B268006F00403413050A00EF905FD38327450031
:10B2780013850700232AF100EFB09FC32328A100FC
:10B2880013050A00EF909FD1832785002324F1003E
:10B2980083270101E38407F483278100E38007F40F
:10B2A80083C60700E38C06F2136C0C406FF01FF3A3
:10B2B8008346B103E39406F293060002A30DD1027C
:10B2C8006FF0DFF1136C1C006FF05FF1032B0D00C2
:10B2D800130D4D00E3540BF0330B6041136C4C001D
:10B2E8006FF0DFEF9306B0026FF05FFD03C6090051
:10B2F800938C19006316860483240D0093064D0071
:10B3080063D404009304F0FF138D060093890C00A6
:10B318006FF0DFEC138504009305A000EF50D030E8
:10B32800938C1C0003C6FCFFB3043501930906FD8A
:10B3380093079000E3F037FF93890C006FF0DFEA82
:10B34800930400006FF09FFE136C0C086FF01FE968
:10B35800938C0900130B000013050B009305A00044
:10B36800232CC100EF50502C03268101938C1C0024
:10B3780093079000130B06FD03C6FCFF330BAB00CD
:10B38800930606FDE3FAD7FC6FF01FFB03C609001E
:10B39800930680066318D60093891900136C0C2055
:10B3A8006FF0DFE3136C0C046FF05FE303C6090072
:10B3B8009306C0066318D60093891900136C0C0213
:10B3C8006FF0DFE1136C0C016FF05FE183260D0075
:10B3D800930C4D00A30D01022306D108930410001D
:10B3E800930A00001304C1086F00401F136C0C017E
:10B3F80093760C02638C0604130D7D00137D8DFF7C
:10B4080083280D00832A4D00930C8D0063DE0A000B
:10B41800B3081041B336100133035041B30AD34087
:10B428009306D002A30DD1029306F0FF6394D45083
:10B43800639E0A569307900063EA17579388080398
:10B44800A307110F1304F10E6F00C05493760C017B
:10B45800930C4D006388060083280D0093DAF841A9
:10B468006FF0DFFA93760C0483280D0063880600DA
:10B478009398080193D808416FF05FFE93760C20EB
:10B48800E38E06FC9398880193D888416FF01FFDDE
:10B4980013760C0283260D00130D4D00630C060075
:10B4A8008327410023A0F60093D7F74123A2F60093
:10B4B8006FF01FCA13760C0163080600832741004A
:10B4C80023A0F6006FF0DFC813760C0463080600AB
:10B4D800835741002390F6006FF09FC793770C20A5
:10B4E800E38E07FC834741002380F6006FF05FC6B8
:10B4F800136C0C0193760C0263860604130D7D0011
:10B50800137D8DFF83280D00832A4D00930C8D0039
:10B51800137CFCBF93060000A30D01021306F0FF85
:10B528006380C44213060C00B3E55801137CFCF792
:10B538006398054063800458130610006396C6405C
:10B548006FF0DFEF93760C01930C4D0063860600D5
:10B5580083280D006F00000193760C0463880600B1
:10B5680083580D00930A00006FF09FFA93760C2021
:10B57800E38006FE83480D006FF0DFFEB786FFFF0D
:10B5880083280D0093C6068397670000938747E9D1
:10B59800930C4D00930A0000136C2C00231ED1025B
:10B5A8002326F100930620006FF01FF7A30D010278
:10B5B8009306F0FF930C4D0003240D006380D42CF8
:10B5C800138604009305000013050400EFA04FBB89
:10B5D800930A000063040500B3048540138D0A0034
:10B5E80063D49A00138D04008346B1036384060074
:10B5F800130D1D0093772C00232CF10063840700A2
:10B60800130D2D0093774C08232EF1006394070641
:10B61800B306AB416350D0069308000117680000D9
:10B628001308C876130370000326410423A00D01F4
:10B63800832581041306160013858D0063C4D84A38
:10B6480023A2DD00B386B6002324D1042322C1043B
:10B6580093067000930D050063DEC600130601040F
:10B668009305090013050A00EFF0DF866318055CEF
:10B67800938D0B008346B103638806041306B10358
:10B6880023A0CD00130610008326410423A2CD0079
:10B6980003268104938616002322D104130616007C
:10B6A8002324C10413067000938D8D00635ED600B9
:10B6B800130601049305090013050A00EFF09F81A2
:10B6C800631E0556938D0B00832781016388070449
:10B6D8001306C10323A0CD001306200083264104CE
:10B6E80023A2CD0003268104938616002322D104C9
:10B6F800130626002324C10413067000938D8D00C1
:10B70800635ED600130601049305090013050A00B9
:10B71800EFF04FFC63140552938D0B008327C10192
:10B72800930600086394D706B306AB416350D0066E
:10B738009308000117680000130848661303700097
:10B748000326410423A00D01832581041306160056
:10B7580013858D0063C4D83E23A2DD00B386B600EE
:10B768002324D1042322C10493067000930D0500FD
:10B7780063DEC600130601049305090013050A00D9
:10B78800EFF04FF5631C054A938D0B00B38A9A407E
:10B7980063505007930800011768000013080860F9
:10B7A800130370008326410423A00D01032681049E
:10B7B8009386160093858D0063CE583D23A25D01C4
:10B7C800B38ACA00232451052322D104130670002A
:10B7D800938D0500635ED6001306010493050900E6
:10B7E80013050A00EFF00FEF631A0544938D0B0061
:10B7F8008326810423A29D0023A08D00B384960094
:10B8080083264104232491041306700093861600AE
:10B818002322D10413878D00635ED600130601042A
:10B828009305090013050A00EFF0CFEA63180540F5
:10B8380013870B0093774C006396073A6354AB0168
:10B84800130B0D0083274100B38767012322F10002
:10B8580083278104638C07001306010493050900FC
:10B8680013050A00EFF00FE7631A053C23220104D1
:10B87800138D0C00938D0B006FF09F8D1305040042
:10B88800EFB00FE393040500930A00006FF01FD593
:10B89800136C0C0193760C0263800602130D7D0075
:10B8A800137D8DFF83280D00832A4D00930C8D0096
:10B8B800930610006FF05FC693760C01930C4D0051
:10B8C8006386060083280D006F00000193760C0440
:10B8D8006388060083580D00930A00006FF05FFD2F
:10B8E80093760C20E38006FE83480D006FF0DFFEA0
:10B8F800976700009387C7B26FF05F9293760C0149
:10B90800930C4D006386060083280D006F0000012C
:10B9180093760C046388060083580D00930A000090
:10B928006FF0DF9193760C20E38006FE83480D00CC
:10B938006FF0DFFE13060C00930610006FF0DFBEF9
:10B9480013061000E386C6AE130620006388C612ED
:10B958009306010F9395DA0113F6780093D838000F
:10B9680013060603B3E8150193DA3A00A38FC6FE5F
:10B97800B3E558011384F6FF6396050293751C001E
:10B98800638A0500930500036306B600A30FB4FE9F
:10B998001384E6FF9307010F938A0400B38487405A
:10B9A8006FF0DFC3930604006FF0DFFA93770C4063
:10B9B800130D0000130E010F232CF100138508004E
:10B9C8001306A0009306000093850A001304FEFFE7
:10B9D8002320C103232E1101EF00502D032E010255
:10B9E8008327810113050503A30FAEFE130D1D0068
:10B9F8008328C101638E07048327810083C607005B
:10BA08006398A6059307F00F6304FD0463960A0084
:10BA18009307900063FE17038327010183254101E3
:10BA2800232E11013304F440138607001305040084
:10BA3800EFB0CFC983278100130D00008328C1010F
:10BA480083C6170063860600938717002324F10036
:10BA58001385080093850A001306A00093060000CA
:10BA6800EF000047938A0500B3E5A5009308050099
:10BA7800E38205F2130E04006FF05FF41304010F64
:10BA88008327C10093F6F8001304F4FFB386D700A8
:10BA980083C6060093D848002300D4009396CA01B1
:10BAA800B3E8160193DA4A00B3E65801E39A06FCB4
:10BAB8006FF05FEE1304010FE39E06EC1376160099
:10BAC800E30A06EC93060003A307D10E6FF09F97D5
:10BAD8006308061E2306C108A30D0102930C0D007E
:10BAE8006FF0DF8F9385050123A21D012324B10484
:10BAF8002322C104635EC3021306010493050900EF
:10BB080013050A00232661022324010323221103BB
:10BB18002320D102EFF00FBC631205120323C102E8
:10BB280003288102832841028326010213850B0022
:10BB3800938606FF930D05006FF01FAF93850501EF
:10BB480023A21D012324B1042322C104635EC3027E
:10BB5800130601049305090013050A002322610254
:10BB680023200103232E1101232CD100EFF08FB6DF
:10BB78006316050C03234102032801028328C1012F
:10BB88008326810113850B00938606FF930D05001C
:10BB98006FF01FBB1306060123A21D012324C10455
:10BBA8002322D104635AD302130601049305090022
:10BBB80013050A0023206102232E0101232C110101
:10BBC800EFF04FB1631C0506032301020328C101EE
:10BBD8008328810193850B00938A0AFF938D0500C2
:10BBE8006FF05FBC3304AB41E35A80C4930A000191
:10BBF8009764000093848419130C70008327410410
:10BC080023209700832681049387170063CE8A0632
:10BC1800232287003304D400232481042322F1043F
:10BC280013077000E35CF7C01306010493050900CD
:10BC380013050A00EFF00FAAE30205C08357C900F5
:10BC480093F70704639807CC8320C1120324811259
:10BC58000325410083244112032901128329C111BC
:10BC6800032A8111832A4111032B0111832BC1104F
:10BC7800032C8110832C4110032D0110832DC10F3B
:10BC880013010113678000009386060123225701E0
:10BC98002324D1042322F10413078700635EFC00E8
:10BCA800130601049305090013050A00EFF08FA29B
:10BCB800E31605F813870B00130404FF6FF01FF455
:10BCC80083278104E38C07F6130601049305090012
:10BCD80013050A00EFF00FA06FF05FF6130101FEE5
:10BCE800232C8100232A910023282101232E1100CF
:10BCF8002326310113090500938405001304060067
:10BD0800630805008327850363940700EF601FB766
:10BD1800832784012324F4008357C40093F7870002
:10BD2800638A070883270401638607088317C4000A
:10BD380093F9F40F93F4F40F139727016356070A46
:10BD480083270401032504003305F54083274401B4
:10BD5800634AF5009305040013050900EF60DF96B8
:10BD68006312050683278400130515009387F7FFE0
:10BD78002324F40083270400138717002320E400FA
:10BD88002380370183274401638CA7008357C400AD
:10BD980093F71700638A07029307A0006396F402DB
:10BDA8009305040013050900EF601F92630E050058
:10BDB8006F0040019305040013050900EF608FDC54
:10BDC800E30605F69304F0FF8320C10103248101F3
:10BDD8001385040003290101832441018329C1003B
:10BDE800130101026780000037270000B3E7E7006E
:10BDF8002316F4008327440637E7FFFF1307F7FFEE
:10BE0800B3F7E7002322F4066FF09FF3977700005B
:10BE1800938747CF138605009305050003A5070000
:10BE28006FF0DFEB977700009387C7CD83A70700F4
:10BE3800130101FE232C8100232A9100232E1100D7
:10BE4800130405009384060083A747036398050439
:10BE580063960700976700009387477383A7070EC9
:10BE6800938604001306000093054100130504009F
:10BE7800E78007009307F0FF6318F50023A004008C
:10BE88009307A0082320F4008320C1010324810123
:10BE980083244101130101026780000063960700B3
:10BEA800976700009387876E83A7070E9386040021
:10BEB8006FF0DFFB977700009387C7C493060600EF
:10BEC800138605009305050003A507006FF09FF58D
:10BED800130101FD23229102232A51012326110275
:10BEE8002324810223202103232E3101232C410105
:10BEF8002328610123267101232481012322910132
:10BF08002320A101930A050093840500639E063847
:10BF1800130406009309050017690000130949F482
:10BF280063F8C512B7070100138B05006378F61094
:10BF38001307F00F3337C70013173700B357E6005E
:10BF48003309F900834609003387E60093060002A7
:10BF5800B386E640638C0600B394D40033D7EA0076
:10BF68003314D600336B9700B399DA00935A04015F
:10BF780093850A0013050B00EF4050721309050062
:10BF880093850A00931B040113050B00EF40906C86
:10BF980093DB0B01930405009305050013850B0043
:10BFA800EF4090681319090193D70901B367F900A5
:10BFB800138A040063FEA700B3878700138AF4FF7F
:10BFC80063E8870063F6A700138AE4FFB387870056
:10BFD800B384A74093850A0013850400EF40106CD2
:10BFE8001309050093850A0013850400EF40906645
:10BFF8009399090193040500930505001319090194
:10C0080013850B0093D90901EF401062B369390118
:10C018001386040063FCA900B30934011386F4FFF6
:10C0280063E6890063F4A9001386E4FF13140A0188
:10C038003364C400130A00006F000013B70700013F
:10C0480013070001E36CF6EE130780016FF01FEF92
:10C05800138A0600631A06009305000013051000F2
:10C06800EF40505F13040500B7070100637EF41228
:10C078009307F00F63F48700130A8000B357440155
:10C088003309F90003470900930600023307470103
:10C09800B386E64063940612B3848440130A100002
:10C0A800135B040193050B0013850400EF40105F38
:10C0B8001309050093050B0013850400931B040165
:10C0C800EF40505993DB0B019304050093050500DD
:10C0D80013850B00EF4050551319090193D7090137
:10C0E800B367F900938A040063FEA700B38787004B
:10C0F800938AF4FF63E8870063F6A700938AE4FF56
:10C10800B3878700B384A74093050B001385040009
:10C11800EF40D0581309050093050B001385040060
:10C12800EF405053939909019304050093050500C6
:10C138001319090113850B0093D90901EF40D04E5B
:10C14800B36939011386040063FCA900B3093401FB
:10C158001386F4FF63E6890063F4A9001386E4FFFD
:10C1680013940A013364C4001305040093050A00FC
:10C178008320C1020324810283244102032901028E
:10C188008329C101032A8101832A4101032B01016B
:10C19800832BC100032C8100832C4100032D010057
:10C1A8001301010367800000B7070001130A0001AB
:10C1B800E366F4EC130A80016FF05FEC3314D400EB
:10C1C80033DAE400B399DA0033D7EA00935A04016A
:10C1D800B394D40093850A0013050A00336B9700C3
:10C1E800EF40D04B1309050093850A0013050A0098
:10C1F800931B0401EF40104693DB0B0193040500E9
:10C208009305050013850B00EF401042131909012F
:10C2180013570B013367E900138A0400637EA700F4
:10C2280033078700138AF4FF636887006376A700E3
:10C23800138AE4FF33078700B304A74093850A00F5
:10C2480013850400EF4090451309050093850A0003
:10C2580013850400EF401040930405009305050082
:10C2680013850B00EF40503C13170B0113570701C0
:10C2780013190901B367E9001387040063FEA700D7
:10C28800B38787001387F4FF63E8870063F6A70086
:10C298001387E4FFB3878700131A0A01B384A74002
:10C2A800336AEA006FF0DFDF63ECD51EB7070100E1
:10C2B80063F4F6041307F00FB335D70093953500F0
:10C2C80033D7B60097670000938787B9B387E7002D
:10C2D80003C70700130A00023307B700330AEA400E
:10C2E80063160A0213041000E3E096E833B6CA00A6
:10C2F800134416006FF05FE7B707000193050001CC
:10C30800E3E0F6FC930580016FF09FFBB35CE60069
:10C31800B3964601B3ECDC0033D4E40093DB0C01A4
:10C32800B397440133D7EA0093850B001305040043
:10C33800336BF700B3194601EF4050361309050077
:10C3480093850B0013050400139C0C01EF409030FB
:10C35800135C0C01930405009305050013050C00FC
:10C36800EF40902C1319090113570B013367E900AB
:10C3780013840400637EA700330797011384F4FF36
:10C38800636897016376A7001384E4FF3307970176
:10C39800B304A74093850B0013850400EF401030C9
:10C3A8001309050093850B0013850400EF40902ABC
:10C3B800930405009305050013050C00EF40D026F3
:10C3C80093170B011319090193D70701B367F900F4
:10C3D8001386040063FEA700B38797011386F4FF52
:10C3E80063E8970163F6A7001386E4FFB387970114
:10C3F80013140401B70B01003364C4001389FBFF55
:10C40800337D240133F92901B384A740930509003A
:10C4180013050D00EF405021935C040193050900BA
:10C42800130B050013850C00EF40102093D9090168
:10C43800130C05009385090013850C00EF40D01EEE
:10C44800130905009385090013050D00EF40D01D61
:10C458003305850193570B013385A7006374850164
:10C468003309790193570501B387270163E6F4027D
:10C47800E392F4BCB70701009387F7FF3375F50023
:10C4880013150501337BFB0033964A01330565011B
:10C49800130A0000E37AA6CC1304F4FF6FF09FB9E7
:10C4A800130A0000130400006FF01FCC130101FBF6
:10C4B8002324810423229104232E31032322910370
:10C4C8002326110423202105232C4103232A510369
:10C4D8002328610323267103232481032320A10336
:10C4E800232EB101930C0500938905001304050060
:10C4F80093840500639E062613090600138A060026
:10C50800976A0000938ACA9563F4C514B7070100B7
:10C518006376F6129307F00F63F4C700130A8000DE
:10C52800B3574601B38AFA0003C70A00130500028D
:10C5380033074701330AE540630C0A00B395490104
:10C5480033D7EC0033194601B364B70033944C0178
:10C55800935A090193850A0013850400EF401014CB
:10C568009309050093850A00131B0901138504002C
:10C57800EF40500E135B0B019305050013050B00EC
:10C58800EF40900A9399090193570401B3E7F90022
:10C5980063FAA700B387270163E6270163F4A700BE
:10C5A800B3872701B384A74093850A001385040045
:10C5B800EF40D00E9309050093850A001385040007
:10C5C800EF405009131404019305050093990901DC
:10C5D80013050B0013540401EF40100533E48900E0
:10C5E800637AA40033042401636624016374A400FD
:10C5F800330424013304A440335544019305000057
:10C608008320C104032481048324410403290104F1
:10C618008329C103032A8103832A4103032B0103CE
:10C62800832BC102032C8102832C4102032D0102BA
:10C63800832DC1011301010567800000B7070001C0
:10C64800130A0001E36EF6EC130A80016FF05FED48
:10C65800631A06009305000013051000EF40807F61
:10C6680013090500B7070100637AF90E9307F00F65
:10C6780063F42701130A8000B3574901B38AFA000B
:10C6880003C70A0013050002B38429413307470191
:10C69800330AE540E30E0AEA33194901B3DAE9003F
:10C6A800B395490133D7EC0093540901336BB700B4
:10C6B80013850A0093850400EF40407E9309050026
:10C6C80093850400931B090113850A00EF408078C5
:10C6D80093DB0B019305050013850B00EF40C07435
:10C6E8009399090193570B01B3E7F90033944C016F
:10C6F80063FAA700B387270163E6270163F4A7005D
:10C70800B3872701B38AA7409385040013850A00DD
:10C71800EF40C078930905009385040013850A004B
:10C72800EF4040739305050013850B00EF40C06F81
:10C7380093150B019399090193D50501B3E5B90048
:10C7480063FAA500B385250163E6250163F4A50016
:10C75800B3852501B384A5406FF09FDFB7070001BB
:10C76800130A0001E36AF9F0130A80016FF0DFF0A1
:10C77800E3E8D5E8B707010063FCF604930BF00F74
:10C7880033B5DB001315350033D7A60097570000E3
:10C798009387076DB387E70083CB070093050002F3
:10C7A800B38BAB00338B7541631E0B0263E4360118
:10C7B80063EACC003384CC40B386D94033B58C00CF
:10C7C800B384A64013050400938504006FF05FE36B
:10C7D800B707000113050001E3E8F6FA1305800125
:10C7E8006FF09FFAB3966601335D7601336DDD0015
:10C7F80033D47901B395690133DC7C0193540D017D
:10C80800336CBC001305040093850400B31A660159
:10C81800EF40C068130A050093850400130504005F
:10C8280033996C01931C0D01EF40C06293DC0C013D
:10C83800130405009305050013850C00EF40C05E46
:10C84800131A0A0113570C013367EA00130A04008C
:10C85800637EA7003307A701130AF4FF6368A701E3
:10C868006376A700130AE4FF3307A701B309A740BB
:10C878009385040013850900EF4040629385040006
:10C888001304050013850900EF40C05C93050500FB
:10C898009304050013850C00EF40005993150C0113
:10C8A8001314040193D50501B365B400138704007C
:10C8B80063FEA500B385A5011387F4FF63E8A5010E
:10C8C80063F6A5001387E4FFB385A501131A0A01CF
:10C8D800B70C0100336AEA001384FCFFB3778A00BF
:10C8E80033F48A00B384A540138507009305040038
:10C8F8002326F100135A0A01EF400053930905005B
:10C908009305040013050A00EF40005213DC0A01E6
:10C91800930D050093050C0013050A00EF40C05065
:10C928008327C100130A050093050C00138507002F
:10C93800EF40804F3305B50113D709013307A7002E
:10C948006374B701330A9A01B70701009387F7FFA9
:10C95800935507013377F70013170701B3F7F90069
:10C96800B3854501B307F70063E6B400639EB400DE
:10C97800637CF90033865741B3B7C700B385A54137
:10C98800B385F54093070600B307F9403339F9003A
:10C99800B385B440B385254133947501B3D7670196
:10C9A8003365F400B3D565016FF09FC5130101FB32
:10C9B80023248104232C41033704100013DA450192
:10C9C80023202105232E3103232A51032324810305
:10C9D8001304F4FF2326110423229104232861035E
:10C9E80023267103232291032320A103232EB101BF
:10C9F800137AFA7F13090500130C0600938A0600C0
:10CA08003374B40093D9F50163060A0A9307F07FDB
:10CA18006304FA1013143400B70780003364F40079
:10CA2800135BD501336B8B0093143500130A1AC0BE
:10CA3800930B000013D54A01370910001309F9FFB9
:10CA48001375F57F3379590193050C0093DAFA01D0
:10CA5800630205109307F07F6302F5163704800020
:10CA680013193900336989001354DC013364240134
:10CA780093153C00130515C09307000013972B006E
:10CA88003367F7001307F7FF9306E00033C959012E
:10CA9800330AAA4063E0E6169756000093860631EB
:10CAA800131727003307D700032707003307D700DA
:10CAB80067000700336BA400630E0B0663000404D1
:10CAC80013050400EF40C043930755FF1307C00147
:10CAD800634CF702130BD001930485FF330BFB4023
:10CAE80033149400335B6901336B8B00B3149900E2
:10CAF800130AD0C0330AAA406FF09FF3EF404040BA
:10CB0800130505026FF05FFC130485FD331B8900D4
:10CB1800930400006FF0DFFD336BA40063040B0285
:10CB280093040500130B0400130AF07F930B3000E5
:10CB38006FF05FF093040000130A0000930B1000DD
:10CB48006FF05FEF93040000130AF07F930B20004F
:10CB58006FF05FEE33648901630E04066300090415
:10CB680013050900EF40C039930755FF1307C001AB
:10CB7800634EF7021304D001930585FF3304F44094
:10CB88003319B90033548C0033642401B315BC0045
:10CB98001307D0C03305A7406FF01FEE13050C0034
:10CBA800EF400036130505026FF01FFC130485FDE6
:10CBB80033148C00930500006FF09FFD33648901E6
:10CBC80063020402130409001305F07F9307300081
:10CBD8006FF0DFEA930500001305000093071000CB
:10CBE8006FF0DFE9930500001305F07F930720003D
:10CBF8006FF0DFE86366640163128B4863E0B44852
:10CC08009316FB0113D71400139CF401135B1B004C
:10CC1800B3E4E6001314840093DC8501B3EC8C00C4
:10CC280093DA0C0193970C0193D70701139D8500A4
:10CC380013050B0093850A002322F100EF408021A1
:10CC480093050500930B050013950C011355050179
:10CC5800EF40801D1304050093850A0013050B009F
:10CC6800EF40C0231315050113D704013365A7004E
:10CC780093890B00637E8500330595019389FBFF3B
:10CC880063689501637685009389EBFF3305950109
:10CC98003304854093850A0013050400EF40801B88
:10CCA80093050500930B050013950C011355050119
:10CCB800EF408017130B050093850A001305040045
:10CCC800EF40C01D939D04011315050193DD0D016F
:10CCD800B3EDAD0013870B0063FE6D01B38D9D01AD
:10CCE8001387FBFF63E89D0163F66D011387EBFF74
:10CCF800B38D9D0193960901B7040100B3E6E600E0
:10CD0800B38D6D41138BF4FF33F76601337B6D01EF
:10CD18001305070093050B0013D406012326D10041
:10CD28002324E100EF4040102322A10093050B00CB
:10CD380013050400EF40400F935B0D0193090500B4
:10CD480093850B0013050400EF40000E03278100B4
:10CD58001304050013850B0093050700EF40C00C72
:10CD680003264100330535018326C1001357060108
:10CD78003307A700637437013304940037050100B3
:10CD88001305F5FF93540701B379A7009399090197
:10CD98003376A600B3848400B389C90063E89D0094
:10CDA8001384060063949D0463723C05330CAC0144
:10CDB8003337AC0133079701B38DED001384F6FFC9
:10CDC80063E6BC016394BC036362AC0363E69D0045
:10CDD800639EB401637C3C01330CAC013337AC0176
:10CDE800330797011384E6FFB38DED00B3093C4187
:10CDF800B3849D40B3373C01B384F4409305F0FFFE
:10CE080063889C1A93850A0013850400EF40800408
:10CE1800930505002324A10013950C011355050162
:10CE2800EF4080002322A10093850A0013850400A7
:10CE3800EF40C00683268100032741001315050132
:10CE480093D7090133E5A700938D0600637EE500BB
:10CE580033059501938DF6FF636895016376E500C8
:10CE6800938DE6FF33059501B304E54093850A00E9
:10CE780013850400EF30107E930505002322A100DE
:10CE880013950C0113550501EF30107A130C0500AA
:10CE980093850A0013850400EF4040009399090127
:10CEA800032741001315050193D9090133E5A900AA
:10CEB80093070700637E8501330595019307F7FF04
:10CEC80063689501637685019307E7FF330595014C
:10CED80093940D01B3E4F4009397040193D70701E9
:10CEE80093050B00B3098541138507002322F10040
:10CEF80093DD0401EF30507393050B00930A05008E
:10CF080013850D00EF305072130C050093850D004A
:10CF180013850B00EF30507183274100130B050078
:10CF280013850B0093850700EF30107033058501DA
:10CF380093D70A013385A70063768501B7070100F7
:10CF4800330BFB00B70601009386F6FF93570501E4
:10CF58003377D50013170701B3FADA00B3876701EF
:10CF68003307570163E8F900938504006390F904D7
:10CF78006300070433853C019385F4FF63649503DC
:10CF88006366F5006314F5026370ED0293161D00E5
:10CF980033BDA601B30C9D019385E4FF33059501CC
:10CFA800138D06006314F5006304A70193E51500CB
:10CFB8001307FA3F6352E01293F775006380070284
:10CFC80093F7F50093064000638AD70093864500DF
:10CFD800B3B5B6003304B400938506009317740004
:10CFE80063DA0700B70700FF9387F7FF3374F4008D
:10CFF80013070A409307E07F63C2E71A9317D40127
:10D0080093D53500B3E7B70013543400B7061000C2
:10D018009386F6FF3374D400B70610801377F77F32
:10D028009386F6FF131747013374D4001319F901D7
:10D038003364E400336724018320C104032481049A
:10D0480083244104032901048329C103032A81039A
:10D05800832A4103032B0103832BC102032C810282
:10D06800832C4102032D0102832DC1011385070082
:10D07800930507001301010567800000130AFAFFF2
:10D08800130C00006FF01FB91389090013040B007B
:10D098009385040093870B00130720006380E71033
:10D0A800130730006382E70E13071000E392E7F0DE
:10D0B80013040000930700006F00400913890A0059
:10D0C8006FF09FFD37040800930500001309000066
:10D0D800930730006FF05FFC93061000B386E640BC
:10D0E80093078003E3C6D7FC9307F00163C4D70610
:10D0F800130AEA41B317440133D7D500339A4501DF
:10D10800B3E7E700333A4001B3E747013354D400AB
:10D1180013F777006300070213F7F7009306400040
:10D12800630AD70013874700B337F7003304F400C6
:10D138009307070013178400634A07061317D401DF
:10D1480093D73700B367F700135434001307000070
:10D158006FF0DFEB930710FEB387E7401307000279
:10D16800B357F400130500006386E600130AEA4388
:10D1780033154401336AB500333A4001B3E7470138
:10D18800130400006FF0DFF837040800930700006D
:10D198001307F07F130900006FF05FE71304000026
:10D1A800930700001307F07F6FF05FE61304000099
:10D1B80093070000130710006FF05FE5130101FAF1
:10D1C800232C8104232631053704100093D9450107
:10D1D800232A910423206105232E7103232C810324
:10D1E8001304F4FF232E11042328210523244105C9
:10D1F80023225105232A91032328A1032326B103BF
:10D2080093F9F97F93040500930B0600138C06002D
:10D218003374B40013DBF5016388090A9307F07FC0
:10D228006386F9103709800013143400336424012D
:10D238001359D50133698900131D3500938919C025
:10D24800930C000013554C01370A1000130AFAFF1B
:10D258001375F57F337A8A0193840B00135CFC0104
:10D26800630405109307F07F6304F5163704800004
:10D27800131A3A00336A8A0013D4DB013364440179
:10D2880093943B00130515C09307000013972C00D7
:10D298003367F700B389A9001307F7FF9306E00087
:10D2A800B34B8B01938A190063E0E616975600008A
:10D2B800938686B3131727003307D7000327070081
:10D2C8003307D700670007003369A400630E090617
:10D2D8006300040413050400EF309042930755FFE0
:10D2E8001307C001634CF7021309D001130D85FF22
:10D2F8003309F9403314A40133D92401336989006F
:10D30800339DA4019309D0C0B389A9406FF05FF39E
:10D31800EF30103F130505026FF05FFC130985FD20
:10D3280033992401130D00006FF0DFFD3369A40069
:10D3380063040902130D0500130904009309F07F23
:10D34800930C30006FF01FF0130D000093090000DC
:10D35800930C10006FF01FEF130D00009309F07F7E
:10D36800930C20006FF01FEE33647A01630E0406FD
:10D3780063000A0413050A00EF309038930755FF3D
:10D388001307C001634EF7021304D001930485FF0D
:10D398003304F440331A9A0033D48B0033644401C5
:10D3A800B3949B009307D0C03385A7406FF0DFED9F
:10D3B80013850B00EF30D034130505026FF01FFC06
:10D3C800130485FD33948B00930400006FF09FFDD8
:10D3D80033647A016302040213040A001305F07F20
:10D3E800930730006FF09FEA9304000013050000D4
:10D3F800930710006FF09FE9930400001305F07F76
:10D40800930720006FF09FE837070100130AF7FF22
:10D41800135C0D0193DD0401337D4D01B3F4440128
:10D4280093050D00138504002328E100EF30D01F79
:10D43800930C05009385040013050C00EF30D01EF3
:10D448002326A10093850D0013050C00EF30D01D95
:10D45800130B050093050D0013850D00EF30D01C4C
:10D468008326C10093D70C013305D5003385A70067
:10D478006376D50003270101330BEB0093560501B2
:10D4880033754501B3FC4C0113150501B30795012C
:10D49800935C04013374440193050D0013050400E3
:10D4A800232AD1002326F100EF3010182328A100E9
:10D4B8009305040013050C00EF301017130A05003C
:10D4C80093850C0013050C00EF301016130C0500A3
:10D4D80093050D0013850C00EF301015032701018B
:10D4E8003305450183264101935707013385A7007A
:10D4F80063764501B7070100330CFC0037060100CD
:10D5080093570501338C87019307F6FF337AF500AB
:10D518003377F700131A0A01135D0901330AEA0089
:10D528003379F90033874601930509001385040010
:10D538002328E100232EC100EF30100F938504004B
:10D54800232CA10013050D00EF30100E232AA10093
:10D5580093050D0013850D00EF30100D93040500A1
:10D568009305090013850D00EF30100C8326410147
:10D57800032781013305D500935707013385A70099
:10D588006376D5000326C101B384C400B706010041
:10D598009387F6FF935D0501B3849D00B37DF50085
:10D5A8003377F7009305090013050400939D0D01D7
:10D5B800B38DED00232CD100EF3010079305040044
:10D5C800232AA10013050D00EF30100693050D0066
:10D5D8001304050013850C00EF301005130D05002A
:10D5E8009305090013850C00EF301004032741014F
:10D5F80033058500935707013385A70063768500B7
:10D6080083268101330DDD0083270101B706010060
:10D618009386F6FF330BFB00B377D5003377D7003B
:10D6280093970701B387E700333A4B01B387870124
:10D6380033844701330BBB0133079400B33DBB016F
:10D64800B306B70133BC870133344401935705014E
:10D658003337970033648C00B3BDB6013304F4004C
:10D66800B36DB7013304B4013304A40193D7760131
:10D67800131494003364F4008327C10093149B00AF
:10D68800135B7B01B3E4F400B334900093979600E6
:10D69800B3E46401B3E4F4009317740063D207128F
:10D6A80093D7140093F41400B3E497009317F4018C
:10D6B800B3E4F400135414001387FA3F6356E010E0
:10D6C80093F774006380070293F7F4009306400011
:10D6D800638AD70093874400B3B497003304940057
:10D6E800938407009317740063DA0700B70700FFF5
:10D6F8009387F7FF3374F40013870A409307E07F9A
:10D7080063C6E71893DA34009314D401B3E45401E0
:10D7180013543400B70710009387F7FF3374F400ED
:10D728009377F77F370710801307F7FF9397470121
:10D738003374E400939BFB013364F400B367740112
:10D748008320C105032481051385040003290105ED
:10D75800832441058329C104032A8104832A4104BF
:10D76800032B0104832BC103032C8103832C410366
:10D77800032D0103832DC1029385070013010106C0
:10D7880067800000930B0B001304090093040D003D
:10D7980093870C0013072000638AE70E13073000F5
:10D7A800638CE70C13071000E398E7F013040000FC
:10D7B800930400006F008008930B0C006FF09FFD2E
:10D7C800938A09006FF05FEF93061000B386E64076
:10D7D80093078003E3CCD7FC9307F00163C4D70613
:10D7E800938AEA41B317540133D7D400B394540150
:10D7F800B3E7E700B3349000B3E497003354D400A0
:10D8080093F774006380070293F7F400130740004E
:10D81800638AE70093874400B3B497003304940005
:10D82800938407009317840063CA07069317D401EB
:10D8380093D43400B3E49700135434001307000062
:10D848006FF05FED930710FEB387E7401306000201
:10D85800B357F400130700006386C600938AEA43AF
:10D8680033175401B3649700B3349000B3E49700BE
:10D87800130400006FF0DFF8370408009304000079
:10D888001307F07F930B00006FF0DFE8130400002C
:10D89800930400001307F07F6FF0DFE71304000024
:10D8A80093040000130710006FF0DFE68327C5001C
:10D8B80003AF050083AF450083A2850083A5C5009B
:10D8C8003787000093D607011307F7FF139807015E
:10D8D800939E050113D6F701B3F6E60093D7050129
:10D8E800130101FF8328050003234500032E85004B
:10D8F8001358080193DE0E01B3F7E70093D5F5013D
:10D908006390E60233E768003367C70133670701AE
:10D9180013051000631A07046398D7046F0080008A
:10D92800639CE7003367FF01336757003367D7010C
:10D9380013051000631A0702130510006396D70237
:10D948006394E8036312F30363105E02631ED80155
:10D958006300B602639A070033E568003365C501C2
:10D96800336505013335A00013010101678000000C
:10D97800130500006FF05FFF8327C50083A8C5006B
:10D98800032F05000326450003288500378500007E
:10D9980013D707011305F5FF939E080193D60801D5
:10D9A80083A2050003A3450003AE85003377A700D3
:10D9B80093950701130101FF93D5050193D7F7014B
:10D9C80093DE0E01B3F6A60093D8F8016310A70200
:10D9D800B36FCF00B3EF0F01B3EFBF001305E0FF44
:10D9E80063800F0E13010101678000006398A6028F
:10D9F800B3EF6200B3EFCF01B3EFDF011305E0FF30
:10DA0800E3920FFE631207043365CF003365050107
:10DA18003365B500133515006F00C0026314070A9B
:10DA28003365CF00336505013365B500133515003F
:10DA3800639A0600B3EF6200B3EFCF01B3EFDF01E3
:10DA4800638C0F06631A0500638E17011305100017
:10DA5800E38A07F86F008000E39608F81305F0FFE3
:10DA68006FF05FF8E3C4E6FE635AD7001305F0FFD2
:10DA7800E38A07F6130510006FF0DFF6E3E8BEFC53
:10DA88006396D503E3640EFD6314C805E360C3FC25
:10DA980063146600E3ECE2FBE36A66FC130500002E
:10DAA800E31266F4E3645FFC6FF0DFF3E3E0D5FDB7
:10DAB800130500006FF01FF3E31C05FE6FF01FF95C
:10DAC800E388E6F213050000E38606F66FF0DFF759
:10DAD800E36EC8F96FF0DFFD8327C50083A8C50092
:10DAE800032F05000326450003288500378500001D
:10DAF80013D707011305F5FF939E080193D6080174
:10DB080083A2050003A3450003AE85003377A70071
:10DB180093950701130101FF93D5050193D7F701E9
:10DB280093DE0E01B3F6A60093D8F8016310A7029E
:10DB3800B36FCF00B3EF0F01B3EFBF0013052000A1
:10DB480063800F0E13010101678000006398A6022D
:10DB5800B3EF6200B3EFCF01B3EFDF01130520008D
:10DB6800E3920FFE631207043365CF0033650501A6
:10DB78003365B500133515006F00C0026314070A3A
:10DB88003365CF00336505013365B50013351500DE
:10DB9800639A0600B3EF6200B3EFCF01B3EFDF0182
:10DBA800638C0F06631A0500638E170113051000B6
:10DBB800E38A07F86F008000E39608F81305F0FF82
:10DBC8006FF05FF8E3C4E6FE635AD7001305F0FF71
:10DBD800E38A07F6130510006FF0DFF6E3E8BEFCF2
:10DBE8006396D503E3640EFD6314C805E360C3FCC4
:10DBF80063146600E3ECE2FBE36A66FC13050000CD
:10DC0800E31266F4E3645FFC6FF0DFF3E3E0D5FD55
:10DC1800130500006FF01FF3E31C05FE6FF01FF9FA
:10DC2800E388E6F213050000E38606F66FF0DFF7F7
:10DC3800E36EC8F96FF0DFFD130101F22326310D01
:10DC480083A9C50083A6050083A745002328A10052
:10DC580003A58500139709012328210D2324410DCD
:10DC68002322510D2320610D032A0600032B4600B1
:10DC7800832A86000329C60037860000232C810CDE
:10DC88001357070113D409011306F6FF2326310998
:10DC9800232E110C232A910C232E710B232C810B7C
:10DCA800232A910B2328A10B2326B10B2320D1086B
:10DCB8002322F1082324A1082328D104232AF104CC
:10DCC800232CA104232EE1043374C40093D9F90151
:10DCD800630A04126300C426370501003365A700F0
:10DCE800232EA104130601059307C10503A7070006
:10DCF80083A6C7FF9387C7FF1317370093D6D601AC
:10DD08003367D70023A2E700E312F6FE8327010555
:10DD1800939737002328F104B7C7FFFF93871700AD
:10DD28003304F400930400009317090137870000B7
:10DD38001355090193D707011307F7FF2326210974
:10DD48002320410923226109232451092320410763
:10DD580023226107232451072326F1063375E500A2
:10DD68001359F901630C051E6304E532B70A010073
:10DD7800B3EA570123265107130601069307C10684
:10DD880003A7070083A6C7FF9387C7FF13173700AA
:10DD980093D6D6013367D70023A2E700E312F6FE35
:10DDA80083270106939737002320F106B7C7FFFFA3
:10DDB800938717003305F50013070000B3C729013F
:10DDC800232AF100B30785002324F1029387170063
:10DDD8002322F10293972400B3E7E7009387F7FF24
:10DDE8009306E00063EAF62C9746000093868603C4
:10DDF80093972700B387D70083A70700B387D70077
:10DE08006780070033E6D7003366A6003366E6006E
:10DE1800630006146302070613050700EF30400E7F
:10DE2800130C0500930B4CFF93D45B4093FBFB0151
:10DE3800638E0B069305C0FF13850400EF20D07E88
:10DE48009306000213972400130800FFB386764157
:10DE58001305C5FF631605099307010A3387E70011
:10DE6800832701059384F4FFB39B7701232877FB6D
:10DE78001307F0FF6F00C00A63080500EF30400881
:10DE8800130C05026FF01FFA638A07001385070059
:10DE9800EF300007130C05046FF0DFF81385060058
:10DEA800EF300006130C05066FF0DFF79305C0FF8F
:10DEB80013850400EF205077130401059307300001
:10DEC8003307A4000327C7009387F7FF1304C4FF91
:10DED8002328E400E3D697FE9384F4FF6FF05FF9FC
:10DEE80093070105B385A7003306A7003386C7004B
:10DEF80083A7C50083A50501B3D7D700B3957501DE
:10DF0800B3E7B7002328F6006FF09FF49397240037
:10DF180093060105B387F60023A007009384F4FF56
:10DF2800E396E4FE37C4FFFF13041401330484416D
:10DF38006FF05FDFB3E7D700B3E7A70033E5E7008B
:10DF480093042000E30205DE930430006FF0DFDD68
:10DF580013040000930410006FF01FDD33676A019B
:10DF6800336757013367F7006302071463820706B4
:10DF780013850700EF20D078130B0500930A4BFF99
:10DF880013DA5A4093FAFA0163800A089305C0FF2E
:10DF980013050A00EF2050699306000213172A00A0
:10DFA800130800FFB38656411305C5FF631805091A
:10DFB8009307010A3387E70083270106130AFAFF4C
:10DFC800B39A5701232057FD1307F0FF6F00000B8A
:10DFD800638A0A0013850A00EF209072130B05026A
:10DFE8006FF0DFF9630A0B0013050B00EF20507187
:10DFF800130B05046FF09FF813050A00EF2050700B
:10E00800130B05066FF09FF79305C0FF13050A0071
:10E01800EF209061930A0106930730003387AA0026
:10E028000327C7009387F7FF938ACAFF23A8EA004C
:10E03800E3D647FF130AFAFF6FF01FF993070106AB
:10E04800B385A7003306A7003386C70083A7C5009A
:10E0580083A50501B3D7D700B3955501B3E7B7003A
:10E068002328F6006FF05FF493172A009306010641
:10E07800B387F60023A00700130AFAFFE316EAFEA7
:10E0880037C5FFFF13051501330565416FF0DFD272
:10E09800336A6A01B36A5A01B3EAFA001307200027
:10E0A800E38E0AD0130730006FF05FD1130500002C
:10E0B800130710006FF09FD0832901050324010680
:10E0C800370B01009304FBFF93DA0901135904018C
:10E0D800B3F999003374940093850900130504007B
:10E0E800EF209054130A05009305040013850A00D5
:10E0F800EF209053130C05009305090013850A00BF
:10E10800EF209052930B0500938509001305090031
:10E11800EF2090513305850193570A013385A700F5
:10E1280063748501B38B6B01832C4106135D050174
:10E1380033759500337A9A0013150501B307450125
:10E1480013DA0C01B3FC9C009385090013850C00BD
:10E158002326F1022320F108EF20104D130B0500B0
:10E1680093850C0013850A00EF20104C93040500DA
:10E1780093050A0013850A00EF20104B130C0500C5
:10E188009385090013050A00EF20104A330595000E
:10E1980093570B013385A70063769500B7070100F5
:10E1A800330CFC00B706010093570501232CF1003E
:10E1B8009387F6FFB37DF50083244105337BFB008D
:10E1C800939D0D01B38D6D013307BD0113DD04016E
:10E1D800B3F4F4009385040013050400232AE10234
:10E1E8002324D100EF2050442322A10093050400EA
:10E1F80013050D00EF2050432320A10093050D00C7
:10E2080013050900EF205042130B05009385040005
:10E2180013050900EF2050410326010003274100A0
:10E228003305C500935707013385A7006376C500FA
:10E2380083268100330BDB00935705013706010065
:10E24800B3876701232EF1009307F6FF337BF500B0
:10E258003377F70093850C00131B0B01138504001B
:10E26800330BEB002326C100EF20103C2324A10030
:10E2780093850C0013050D00EF20103B2322A1000D
:10E2880093050D0013050A00EF20103A2320A10082
:10E298009385040013050A00EF2010390328410074
:10E2A80003278100832601003305050193570701E1
:10E2B8003385A700637605010326C100B386C6002F
:10E2C8009357050137060100B387D7002320F102D1
:10E2D8009307F6FF3375F500131505013377F7003B
:10E2E8003307E5002328E102032781069385090007
:10E2F800232EC102B377F700935607011385070051
:10E308002320D1002324F100EF201032832581003F
:10E31800232CA10213850A00EF2010318325010068
:10E328002326A10013850A00EF2010302322A10024
:10E338000325010093850900EF20102F0328C10051
:10E3480003278103832641003305050193570701FD
:10E358003385A700637605010326C103B386C6008B
:10E368003708010093570501B386D7009307F8FFD4
:10E378003376F5003377F700131606013306E60007
:10E38800032781052326D10493050400B377F700FA
:10E3980093560701138507002322C1042322D100C5
:10E3A8002326F10023240105EF2010282320A104AF
:10E3B8000325410093050400EF2010278325410021
:10E3C800232EA10213050900EF2010268325C10082
:10E3D800232CA10213050900EF2010258328C1036F
:10E3E8000323010403278103330515019357030110
:10E3F800B387A700032641048326C10463F61701E7
:10E40800032881043307070113D807013308E800FC
:10E41800370701009305F7FFB3F7B7003373B3006D
:10E4280093970701B38E670083274103232CE102EA
:10E4380003270103B38BFB0083278101B3BDBB0115
:10E44800B388B701B3876B0133BB6701232CF10095
:10E458002322F1088327C101B3888801B387F80014
:10E46800338C67013303EC00333EE3000327C1011B
:10E47800333C6C01B3B8B801B3B7E70033EC87019C
:10E4880083270102330C1C013303C300330CFC0047
:10E498003305CC01B308D500032701023336C30086
:10E4A800B307D301338FC80033B3D701232EF1004C
:10E4B8002324F108032BC106B3070F01333EC5011E
:10E4C800333CEC00B3B6D8003336CF00B38D6700C9
:10E4D800B3E6C600336CCC01B3B7070133B36D00A4
:10E4E800330CDC00B3E76700935B0B01337BBB00A5
:10E4F800B307FC009385090013050B002320F102E4
:10E50800EF209012130C050093050B0013850A00E9
:10E51800EF2090112328A10293850B0013850A0090
:10E52800EF209010930A05009385090013850B00CE
:10E53800EF20900F8326010393570C013305D50074
:10E548003385A7006376D50003278103B38AEA00E1
:10E5580093570501B7060100B38757012328F10235
:10E56800832AC1059387F6FFB379F500337CFC0055
:10E5780093990901B389890113DC0A01B3FAFA00F6
:10E5880093850A0013050400232ED102EF20D00939
:10E5980093050400232CA10213050C00EF20D008DA
:10E5A800232AA10293050C0013050900EF20D007C8
:10E5B8001304050093850A0013050900EF20D0060F
:10E5C80003264103032781033305C5009357070139
:10E5D8003385A7006376C5008326C1033304D400BE
:10E5E8003708010093570501338487009307F8FF24
:10E5F8003379F500032581003377F700938504000C
:10E6080013190901232001053309E900EF20D0017E
:10E6180083258100232EA10213050D00EF20D000D1
:10E6280083250100232CA10213050D00EF20C07FD4
:10E63800232AA1020325010093850400EF20C07E50
:10E64800832881038326C10303264103330515016B
:10E6580093D706013385A7006376150103280104C3
:10E6680033060601B70801009387F8FF3377F500F2
:10E67800135E05010325C100B3F6F6001317070161
:10E68800330ECE003307D70093850C002324C10531
:10E698002320E10423221105EF200079232EA10273
:10E6A8000325410093850C00EF2000788325410065
:10E6B800232CA10213050A00EF2000778325C1004F
:10E6C800232AA10213050A00EF2000760323810301
:10E6D8000328C10303264103330565009356080147
:10E6E8003385A60003270104032E810463766500A1
:10E6F8008328410433061601370301009306F3FF0C
:10E7080093580501B388C800B377D5003378D8008B
:10E718000326010383260102B38D3D01B3BF3D01EA
:10E72800B386C600338FF601B38D2D019397070189
:10E73800B387070133B92D0133088F00B30E2801C1
:10E74800B38DED00232A610203230103B385CE01B3
:10E7580033B7ED003386FD003385E50033B92E016C
:10E76800B3B5C501B3B66600333FFF013334880043
:10E77800B337F6002320C1022326C1083337E5004A
:10E788003306150133E7E50033EFE601B309F60078
:10E79800336424018325C1000325810033048F00DD
:10E7A80033361601B3B7F9003304E400B367F60053
:10E7B8003304F400EF2040672328A1028325810059
:10E7C80003254100EF204066130905008325410019
:10E7D80003250100EF204065930D05008325C10046
:10E7E80003250100EF2040640327010333052501B9
:10E7F800935707013385A700637625010323410357
:10E80800B38D6D00B706010093570501B38DB701AD
:10E818009387F6FF3379F5003377F7009385040083
:10E828001319090113050B003309E900232CD10240
:10E83800EF20805F232AA10293050B0013050D002A
:10E84800EF20805E2328A10293850B0013050D009D
:10E85800EF20805D130D05009385040013850B00E0
:10E86800EF20805C03260103032741033305C5001D
:10E87800935707013385A7006376C5008326810374
:10E88800330DDD00B706010093570501338DA7014D
:10E898009387F6FFB374F5003377F70093850C0080
:10E8A8009394040113850A00B384E400232CD10255
:10E8B800EF20805793850C00232AA10213050C0032
:10E8C800EF2080562328A10293050C0013050A00A7
:10E8D800EF208055930C050093850A0013050A0064
:10E8E800EF20805403260103032741033305C500A5
:10E8F800935707013385A7006376C50083268103F4
:10E90800B38CDC003708010093570501B38C9701DD
:10E918009307F8FF337AF5000325C1003377F70032
:10E9280093050B00131A0A01330AEA00232C01038A
:10E93800EF20804F232AA1020325410093050B00F5
:10E94800EF20804E2328A1020325410093850B0068
:10E95800EF20804D8325C1002322A10013850B00E1
:10E96800EF20804C832801038326410303264100BE
:10E978003305150113D706013305A7006376150182
:10E988000328810333060601370801001307F8FF3F
:10E99800B377E5001353050103258100B3F6E600BC
:10E9A800939707013303C300B387D70093850A0001
:10E9B800232C61022328F102232A0103EF20C046F9
:10E9C800832581002326A10013050C00EF20C045F4
:10E9D8002324A1000325010093050C00EF20C04467
:10E9E8002322A1000325010093850A00EF20C043DC
:10E9F80083288100032EC100032641003305150139
:10EA080093560E013385A600832701030323810350
:10EA18006376150103284103330606013708010010
:10EA280093580501B3892901B388C80033B929016E
:10EA38001306F8FF3304B401B30E24013377C5007D
:10EA4800B3899900337ECE00B385AE01B3B4990083
:10EA5800131707013307C701B3894901338E95009E
:10EA6800330F9E0133BA4901B30F4F0133B52E015D
:10EA78003334B40133BDA501B3349E00336E9D0019
:10EA8800B33C9F0133BA4F013365A4003305C50178
:10EA980033EA4C01B386FF003305450133056500B1
:10EAA800B3B7F600B305F500B3B7F5003335650025
:10EAB800B386E60033B7E6003364F5003385150105
:10EAC800B304E50033B7E4003335150123283109D1
:10EAD80093850A00B369E50013050B002320C100E4
:10EAE80023220101232AD108EF20003493050B00CB
:10EAF800130A050013050C00EF200033130B050063
:10EB080093050C0013850B00EF2000321309050054
:10EB180093850A0013850B00EF200031330565014A
:10EB280013570A013305A700032601006376650120
:10EB38000328410033090901B377C50093970701FA
:10EB48003376CA003386C700032781018327C102B1
:10EB580013550501B384C400B3E7E7000327C101D7
:10EB68003305850033B6C400B36BF7008327010271
:10EB7800330535013305C500330525019397D700C3
:10EB8800232EA108232C9108B3E777011307010866
:10EB980013060000130540008326C70083250701DC
:10EBA8001306160093D636019395D500B3E6B60042
:10EBB8002320D70013074700E310A6FE0327010808
:10EBC80083268108B337F000B3E7E700232CD1068A
:10EBD8000327C108832641082328F106232EE106CE
:10EBE800232AD1069316B70063D406249397F70116
:10EBF80013070107130600001305300083260700DA
:10EC0800832547001306160093D616009395F50141
:10EC1800B3E6B6002320D70013074700E310A6FE8B
:10EC28000327C107B337F00013571700232EE10657
:10EC380003270107B367F7002328F10603274102DA
:10EC4800B74700009387F7FFB307F7006354F02036
:10EC58000327010793767700638406049376F70009
:10EC680013064000638EC602832641071307470038
:10EC78002328E10613374700B306D70033B7E60069
:10EC8800232AD10683268107B306D700232CD10671
:10EC9800B3B6E6000327C107B386E600232ED106E4
:10ECA8000327C1079316B70063D00602B707F0FF22
:10ECB8009387F7FF3377F700232EE10603274102F6
:10ECC800B7470000B307F700130701071306000052
:10ECD8001305300083260700832547001306160016
:10ECE80093D636009395D501B3E6B6002320D70016
:10ECF80013074700E310A6FE378700009306E7FFD7
:10ED080063CEF6120327C10713573700232EE106F7
:10ED18000327C107B70601809386F6FF2316E1088B
:10ED2800378700001307F7FFB3F7E7000327C10889
:10ED3800939707018320C10D3377D700B367F70096
:10ED480003274101B706008093C6F6FF1317F701A2
:10ED5800B3F7D700B3E7E7008326010103270107CC
:10ED68000324810D23A6F60023A0E600032741070C
:10ED78008324410D0329010D23A2E60003278107FF
:10ED88008329C10C032A810C23A4E600832A410CA1
:10ED9800032B010C832BC10B032C810B832C410B00
:10EDA800032D010B832DC10A138506001301010EE3
:10EDB80067800000232A3101832701052328F106F3
:10EDC80083274105232AF10683278105232CF10691
:10EDD8008327C105232EF106930720006380F428BA
:10EDE80093073000638AF42893071000E398F4E44B
:10EDF800232E0106232C0106232A010623280106B7
:10EE08006F00C021232A21018327010693040700EC
:10EE18002328F10683274106232AF1068327810642
:10EE2800232CF1068327C106232EF1066FF0DFFAA3
:10EE3800832781022322F1026FF05FE0232E01066F
:10EE4800232C0106232A0106232801069307F7FF2E
:10EE58006FF01FEC93061000B387F64013074007C6
:10EE68006342F71C13D6574093F6F70113070000C7
:10EE780093070000931527006312C70263980604DE
:10EE880013053000130601073305E5406354D50226
:10EE9800930640003387E6406F00400813050107DA
:10EEA800B305B50083A5050013071700B3E7B7003E
:10EEB8006FF05FFC3308B60003280800938616003D
:10EEC80013064600232E06FF6FF05FFC1306010AA7
:10EED8003306B600032606FD130800023308D8409F
:10EEE80033160601B3E7C70013063000930801077D
:10EEF800130300003306E6406346C302930540004F
:10EF08003387E540131626009305010A3386C500AA
:10EF18008325C107B3D6D5002328D6FC13064000A5
:10EF28006F000004338EB80003250E00032E4E0038
:10EF3800130313003355D500331E0E013365C50185
:10EF480023A0A800938848006FF01FFB93162700A2
:10EF580093050107B386D50023A006001307170001
:10EF6800E316C7FE83260107B337F000B3E7D700DF
:10EF78002328F10693F677006382060493F6F700D8
:10EF8800638EE60203274107938747002328F1068B
:10EF980093B747003387E700B337F700232AE10622
:10EFA800032781073387E700232CE1063337F7006F
:10EFB8008327C1073307F700232EE1068327C107FC
:10EFC8001397C700635E0700232E0106232C010652
:10EFD800232A010623280106930710006FF05FD348
:10EFE80093070107930600009305300003A7070065
:10EFF80003A6470093861600135737001316D60149
:10F008003367C70023A0E70093874700E390B6FE65
:10F018008327C10793D73700232EF10693070000F3
:10F028006FF01FCF83274107032701073367F700D6
:10F03800832781073367F7008327C1073367F70002
:10F0480093070000E30607CC232E0106232C0106B4
:10F05800232A0106232801066FF09FCBB7870000FB
:10F06800232E0106232C0106232A01062328010644
:10F078009387F7FF6FF0DFC9B7870000232EF106EB
:10F08800232C0106232A0106232801069387F7FF6C
:10F09800232A01006FF0DFC7130101FA83A7850057
:10F0A8002324410503AAC50083A6050003A745003C
:10F0B800232CF102232CF10093170A01232C81043D
:10F0C80093D7070113141A00232A91040323060077
:10F0D8009304050083284600832586000325C6007F
:10F0E800232E4103232E110423282105232631052D
:10F0F800232251052328D102232AE1022328D10003
:10F10800232AE100232EF10013541401135AFA01A3
:10F11800130801011306C101832706000327C6FF50
:10F128001306C6FF939737001357D701B3E7E700D5
:10F138002322F600E312C8FE832601019317050176
:10F14800232CB102939636002324B10293D70701EA
:10F158009315150023286102232A1103232EA102E7
:10F1680023206102232211032328D1002326F10240
:10F1780093D515011355F501930801021303C10234
:10F18800832703000327C3FF1303C3FF93973700A5
:10F198001357D701B3E7E7002322F300E39268FE91
:10F1A80083270102378700001307F7FF939737007B
:10F1B8002320F1026390E502032E81020327410216
:10F1C8003367C701032EC1023367C7013367F700EE
:10F1D80063140700134515003307B440E3164511BF
:10F1E8006352E030639605140325410283258102AA
:10F1F8000328C1023366B500336606013366F6009C
:10F2080063140602832741012328D102130407004F
:10F21800232AF10283278101232CF1028327C101CC
:10F22800232EF1026F0040301306F7FF631E060C11
:10F2380003274101B387F600B3B6D7003306E500CC
:10F248002328F102B307D600B3B6D700232AF10268
:10F25800832781013337E600B366D7003387F5008B
:10F268003306D700B337F7000327C101B336D600FA
:10F27800B3E7D7003308E800B3870701232CC1029E
:10F28800232EF102130410008327C1031397C7002C
:10F29800635C07283707F8FF1307F7FFB3F7E700A2
:10F2A800232EF1028327010313041400130701031B
:10F2B8009397F70113060000130530008326070013
:10F2C800832547001306160093D616009395F5017B
:10F2D800B3E6B6002320D70013074700E310A6FEC5
:10F2E8000327C103B337F00013571700232EE10299
:10F2F80003270103B367F7002328F102B78700004B
:10F308009387F7FF6F00C07CB78700009387F7FFEC
:10F31800E30AF7EE9307400763D0C70623260102E6
:10F328002324010223220102930710006F00801496
:10F33800B78700009387F7FF6312F4028327410120
:10F348002328D102232AF10283278101232CF102E9
:10F358008327C101232EF1026F00001D8327C102FC
:10F36800B7060800B3E7D7002326F1029307400742
:10F37800E3C6E7FA13060700135756409305000043
:10F388001376F60193070000939627006390E7022F
:10F3980063140604130730003307F7406352C702AB
:10F3A80013074000B307F7406F00C007B386D800C3
:10F3B80083A6060093871700B3E5D5006FF0DFFC3E
:10F3C8003305D30003250500130616001303430075
:10F3D800232EA3FE6FF09FFC130701043307D70009
:10F3E800032707FE130800023308C8403317070134
:10F3F800B3E5E50013073000130E00003307F740AC
:10F408006346EE0293064000B387F64013172700C1
:10F41800930601043387E6008326C10233D6C6006B
:10F428002320C7FE930640006F00C003B30ED3002D
:10F4380003A50E0083AE4E00130E1E003355C50003
:10F44800B39E0E013365D5012320A30013034300A7
:10F458006FF01FFB139727003387E800232007006E
:10F4680093871700E398D7FE03270102B337B0004C
:10F47800B367F7002320F1028326010183270102E5
:10F488000327410183258102B387F600B3B6D7006D
:10F498002328F102832741020325C102B307F7009D
:10F4A8003386D70033B7E700B337D600B367F70022
:10F4B800032781018326C101232AC102B305B700AE
:10F4C8003386F50033B7E500B337F600B386A600F8
:10F4D8003367F7003387E600232CC102232EE102AD
:10F4E8006FF09FDA6300073E631604248328410106
:10F4F80003258101032EC10133E3A8003363C3014F
:10F508003363D3006310031A2328F10283274102CF
:10F5180013840500232AF10283278102232CF10298
:10F528008327C102232EF1028327010313F77700F3
:10F538006304070413F7F70093064000630ED7022D
:10F5480003274103938747002328F10293B7470015
:10F558003387E700B337F700232AE1020327810343
:10F568003387E700232CE1023337F7008327C103F1
:10F578003307F700232EE1028327C1031397C7003F
:10F588006354070237870000130414001307F7FFBA
:10F598006314E4006F00507F3707F8FF1307F7FF85
:10F5A800B3F7E700232EF102930701039306000047
:10F5B8009305300003A7070003A6470093861600AB
:10F5C800135737001316D6013367C70023A0E70087
:10F5D80093874700E390B6FE8327C103B7860000F0
:10F5E80013D73700232EE1029387F6FF631AF4023C
:10F5F8000326410383270103B3E7C70003268103DA
:10F60800B3E7C700B3E7E700638C0700232ED102F6
:10F61800232C0102232A010223280102130A0000D5
:10F628008327C103370701801307F7FF2316F1006B
:10F63800B78700009387F7FF3374F400931704012A
:10F648000324C1008320C105138504003374E4003A
:10F658003364F4009317FA01370A0080134AFAFF5B
:10F6680033744401336AF4008327010303248105BA
:10F6780023A6440123A0F40083274103032901059D
:10F688008329C10423A2F40083278103032A810468
:10F69800832A410423A4F4008324410513010106AD
:10F6A800678000001303F0FF63106706032641021A
:10F6B800B386F600B3B7F6003388C8003307F800FE
:10F6C800B337F700232AE102032781023336C80043
:10F6D800B367F6002328D102B306E5003386F600A7
:10F6E800B337F60033B7E6003367F7008327C10264
:10F6F800232CC102330EFE003307C701232EE1027B
:10F70800138405006FF05FB8B78600009386F6FF94
:10F71800E38CD5DE1347F7FF9307400763D0E70470
:10F72800232E0100232C0100232A01009307100037
:10F738006F008012B78600009386F6FFE386D5DC5B
:10F748008327C101B7060800B3E7D700232EF100CD
:10F758009307C0F8E346F7FC3307E0409356574059
:10F76800930800001377F70193070000139527000B
:10F778006390D7026314070493063000B386F640FB
:10F7880063D2E60213074000B307F7406F00C007D3
:10F798003305A8000325050093871700B3E8A800E0
:10F7A8006FF0DFFC3303A6000323030013071700E1
:10F7B80013064600232E66FE6FF09FFC9306010495
:10F7C800B386A60083A606FD130E0002330EEE4094
:10F7D800B396C601B3E8D80093063000930E000034
:10F7E800B386F64063C6DE0213064000B307F64050
:10F7F8009396260013060104B306D6000326C1011A
:10F808003357E60023A8E6FC930640006F00C003C8
:10F81800330FA60003230F00032F4F00938E1E0003
:10F828003353E300331FCF013363E3012320660022
:10F83800130646006FF01FFB139727003307E800F5
:10F848002320070093871700E398D7FE03270101B9
:10F85800B3371001B367F7002328F10083260102AC
:10F86800832701010327410203258101B387F6009D
:10F87800B3B6D7002328F102832741010328C10129
:10F88800B307F7003386D70033B7E700B337D6009E
:10F89800B367F700032781028326C102232AC10226
:10F8A8003305A7003306F5003337E500B337F60014
:10F8B800B38606013367F700232CC1023387E600BD
:10F8C8006FF0DFE3378F000013051400930EFFFF7E
:10F8D800B372D501930F100003274102032681025A
:10F8E8000328C10283254101032E81010323C1019D
:10F8F8009308010363C65F1433E5C50133656500EA
:10F908003365D5006316040A631C05002328F10239
:10F91800232AE102232CC102232E01036FF0DFC04A
:10F928003365C700336505013365F500631C0500C1
:10F938002328D102232AB102232CC103232E6102DA
:10F948006FF09FBEB387F6003307B7002328F10294
:10F95800B3B7D700B306F700232AD1023337B7006D
:10F96800B3B6F600B366D700B305C601B387D500B2
:10F9780033B6C501B3B6D700B366D6003306680000
:10F988003386C600232CF1029317C60063C607000E
:10F99800232EC1026FF05FB9B706F8FF9386F6FF12
:10F9A8003376D600232EC102130410006FF0DFB7A0
:10F9B800631E05002328F102232AE102232CC10239
:10F9C800232E010313840E006FF01FB63366C700A1
:10F9D80033660601B367F600639C07002328D1024B
:10F9E800232AB102232CC103232E61026FF09FFD4D
:10F9F800232EE103232C0102232A010223280102DA
:10FA08001307C103832707008326C7FF1307C7FF10
:10FA18009397370093D6D601B3E7D7002322F70090
:10FA2800E392E8FE83270103378400001304F4FF00
:10FA3800939737002328F102130A00006FF0DFAE16
:10FA4800B387F6003307B7002328F102B3B7D7000E
:10FA5800B306F700232AD1023337B700B3B6F6004E
:10FA6800B366D7003306C6013307D600B336D700CE
:10FA78003336C6013366D600B30668003306D600AF
:10FA8800232CE102232EC10293870800930600006D
:10FA98009305300003A7070003A6470093861600C6
:10FAA800135717001316F6013367C70023A0E700A2
:10FAB80093874700E390B6FE8327C103130405002C
:10FAC80093D71700232EF102B78700009387F7FF1B
:10FAD800E31CF4A4232E0102232C0102232A010291
:10FAE800232801026FF05FA46352E028639E050C8F
:10FAF8000325410283258102032EC1023368B50024
:10FB08003368C8013368F800630E08EE1306F7FF80
:10FB18006318060883284101B387F64033B7F60017
:10FB28003388A84033B308013308E8402328F1029A
:10FB3800232A01031307000063F6F6003307154173
:10FB4800133717000328810133676700B306B840ED
:10FB58003335D800B386E640232CD102630607006C
:10FB6800B385054113B615008327C1013366A60086
:10FB780013041000B387C7413386C740232EC10240
:10FB88008327C1031397C700E350079A3707080074
:10FB98001307F7FFB3F7E700232EF1026F00C072D7
:10FBA800B78700009387F7FF630EF7E493074007D2
:10FBB80063D0C70423260102232401022322010261
:10FBC800930710006F008012B78700009387F7FF34
:10FBD8006306F4F68327C102B7060800B3E7D70027
:10FBE8002326F10293074007E3C6E7FC1306070044
:10FBF80013575640930500001376F601930700004B
:10FC0800939627006390E7026314060413073000F5
:10FC18003307F7406352C70213074000B307F740A2
:10FC28006F00C007B386D80083A606009387170025
:10FC3800B3E5D5006FF0DFFC3305D30003250500DD
:10FC48001306160013034300232EA3FE6FF09FFC38
:10FC5800130701043307D700032707FE1308000220
:10FC68003308C84033170701B3E5E5001307300030
:10FC7800130E00003307F7406346EE029306400078
:10FC8800B387F64013172700930601043387E6006D
:10FC98008326C10233D6C6002320C7FE9306400040
:10FCA8006F00C003B30ED30003A50E0083AE4E0051
:10FCB800130E1E003355C500B39E0E013365D501E2
:10FCC8002320A300130343006FF01FFB13972700A3
:10FCD8003387E8002320070093871700E398D7FEAF
:10FCE80003270102B337B000B367F7002320F102FE
:10FCF800832641018325010103270102832741024D
:10FD08003387E540B387F64033B6F600B3B6E5006F
:10FD1800B386D740232AD1022328E10293060000A4
:10FD280063F4E50093B61700B3E6C6000327810223
:10FD3800032681013307E640B307D740232CF1029D
:10FD4800B335E60013060000638406001336170077
:10FD58008327C1010327C1023366B600B387E74092
:10FD6800B387C740232EF1026FF09FE1630C072889
:10FD7800631A040E0323410183288101832EC101E4
:10FD8800336E1301336EDE01336EDE0063160E022E
:10FD98002328F1028327410213840500232AF10254
:10FDA80083278102232CF1028327C102232EF1022B
:10FDB800130A05006FF04FF7130EF0FF631EC70715
:10FDC80003284102B386D74033B7D70033066840CB
:10FDD800333EC8003306E6402328D102232AC10255
:10FDE8001307000063F6D7003307034113371700E2
:10FDF800032881023367C7019306000033061841C0
:10FE08003333C8003306E640232CC10263060700DB
:10FE1800B388084193B618008327C102B3E8660087
:10FE2800B387D741B3871741232EF1021384050006
:10FE3800130A05006FF0DFD4B78600009386F6FF3B
:10FE4800E388D5F41347F7FF9307400763D0E70427
:10FE5800232E0100232C0100232A01009307100000
:10FE68006F008012B78600009386F6FFE382D5F212
:10FE78008327C101B7060800B3E7D700232EF10096
:10FE88009307C0F8E346F7FC3307E0409356574022
:10FE9800130300001377F7019307000093982700D6
:10FEA8006390D7026314070493063000B386F640C4
:10FEB80063D2E60213074000B307F7406F00C0079C
:10FEC800B308180183A80800938717003363130148
:10FED8006FF0DFFC330E1601032E0E001307170018
:10FEE80013064600232EC6FF6FF09FFC93060104FD
:10FEF800B386160183A606FD930E0002B38EEE406C
:10FF0800B396D6013363D30093063000130F000075
:10FF1800B386F6406346DF0213064000B307F64097
:10FF28009396260013060104B306D6000326C101E2
:10FF38003357E60023A8E6FC930640006F00C00391
:10FF4800B30F160103AE0F0083AF4F00130F1F004E
:10FF5800335EEE00B39FDF01336EFE012320C6013E
:10FF6800130646006FF01FFB139727003307E800BE
:10FF78002320070093871700E398D7FE0327010182
:10FF8800B3376000B367F7002328F10083264102E6
:10FF98000328010203270101832741013307E840B1
:10FFA800B387F64033B6F600B336E800B386D740D9
:10FFB800232AD1022328E102930600006374E80093
:10FFC80093B61700B3E6C600032781010326810212
:10FFD8003307E640B307D740232CF1023338E60055
:10FFE8001306000063840600133617008327C10236
:08FFF8000327C1013366060175
:02000004800179
:10000000B387E740B387C7406FF09FE2B78F000028
:10001000930E14009382FFFFB3FE5E00130F1000D7
:10002000832541020326410103288101032EC101DA
:10003000832881020323C102634EDF1DB3EE150145
:10004000336F0601B3EE6E00336FCF01B3EEFE00E7
:10005000336FDF006318041063120F022328F102CC
:10006000232AB102232C1103232E6102E3960ED41E
:1000700013040000130A00006FF08FD0639C0E0081
:100080002328D102232AC102232C0103232EC103DA
:100090006FF00FCAB38EF640B302B640B3BFD601BD
:1000A000333F5600B382F2412328D103232A510261
:1000B000930F000063F6D601B38FC54093BF1F00B6
:1000C000B3031841B3EFEF01B389F341232C31039C
:1000D000B33A78001309000063840F0013B91300CA
:1000E000330F6E4033695901330F2F41232EE10343
:1000F000931FCF0063DE0F04B386D7403386C5401D
:10010000B3BED700B30ED641232AD1032328D10290
:10011000B3B5C500930E000063F4D700933E1600FC
:10012000B3870841B3E5BE00B3B6F800B387B74064
:10013000232CF1026384050013B713003303C3417A
:100140003367D7003303E340232E61026FF0DFC62D
:10015000B3EE5E00B3EE3E01B3EEEE01E38A0EF0C5
:100160006FF00FBD93030103631E0F04639E0E0225
:10017000232EF103232C0102232A0102232801024A
:100180009307C10303A7070083A6C7FF9387C7FF91
:100190001317370093D6D6013367D70023A2E700A1
:1001A000E392F3FE6FF09F882328F102232AB10225
:1001B000232C1103232E6102130A0500138402006D
:1001C0006FF00FB7639C0E002328D102232AC102CF
:1001D000232C0103232EC1036FF05FFE232EF103B6
:1001E000232C0102232A0102232801029307C103C1
:1001F00003A7070083A6C7FF9387C7FF131737001E
:1002000093D6D6013367D70023A2E700E392F3FE2B
:100210006FF0DF81B38EF640B302B640B3BFD601B4
:10022000333F5600B382F2412328D103232A5102DF
:10023000930F000063F6D601B38FC54093BF1F0034
:10024000B3031841B3EFEF01B389F341232C31031A
:10025000B33A78001309000063840F0013B9130048
:10026000330F6E4033695901330F2F41232EE103C1
:10027000931FCF0063D00F0EB386D7403386C5409F
:10028000B3BED700B30ED641232AD1032328D1020F
:10029000B3B5C500930E000063F4D700933E16007B
:1002A000B3870841B3E5BE00B3B6F800B387B740E3
:1002B000232CF1026384050013B713003303C341F9
:1002C0003367D7003307E340232EE102130A05000A
:1002D0000325C103630A0508EF001043930A45FF95
:1002E00013D9FA41B70900801379F9019389F9010B
:1002F00033095901B3F93A011359594063D8090038
:100300009389F9FF93E909FE93891900638A090823
:100310009305C0FF13050900EF009031930600021A
:1003200013172900130800FFB38636411305C5FFD4
:100330006312050B930701043387E700832701034A
:100340001309F9FFB3993701232837FF1307F0FF8B
:100350006F00400CB3EE5E00B3EE3E01B3EEEE0173
:10036000E3880ED06FF0DFF60325810363080500F4
:10037000EF009039130505026FF05FF60325410386
:1003800063080500EF005038130505046FF01FF5F2
:1003900003250103EF005037130505066FF01FF426
:1003A0009305C0FF13050900EF009028930901038E
:1003B000930730003387A9000327C7009387F7FF0F
:1003C0009389C9FF23A8E900E3D627FF1309F9FFA2
:1003D0006FF0DFF793070103B385A7003306A7008B
:1003E0003386C70083A7C50083A50501B3D7D7000F
:1003F000B3953501B3E7B7002328F6006FF01FF37C
:100400009317290093060103B387F60023A0070082
:100410001309F9FFE316E9FE63C08A1633848A40A4
:10042000130414009357F4413707008093F7F70142
:100430001307F701B38787003374E40093D757405D
:10044000635804001304F4FF136404FE130414003F
:10045000930604001305000013070000634AF70227
:100460001387070063D407001307000013932700C6
:10047000631A040413063000130701033306F64021
:100480006356D60213074000B307F7406F00C00859
:1004900013162700930501033386C50003260600C3
:1004A000130717003365C5006FF05FFBB3056700E6
:1004B00083A505009386160013074700232EB7FE79
:1004C0006FF01FFC13172700930601043387E60023
:1004D000032707FF13060002330686403317C700C1
:1004E0003365E5001307300093050103130800008E
:1004F0003307F7406346E80293064000B387F640AF
:1005000013172700930601043387E6008326C103EF
:1005100033D48600232887FE930630006F00000442
:10052000B388650083A6080083A848001308180054
:10053000B3D68600B398C800B3E6160123A0D50051
:10054000938545006FF01FFB1397270013060103E7
:100550003307E6002320070093871700E3D6F6FE53
:1005600003270103B337A00013040000B367F700AB
:100570002328F1026FE0DFFB8327C1033707F8FF71
:100580001307F7FF33045441B3F7E7006FE01FDDB3
:10059000232E0102232C0102232A01022328010217
:1005A0006FF00F8103274500832785000326C500D0
:1005B00083260500130101FE2322E1002324F1001C
:1005C000232AE100232CF10037470000931716007F
:1005D0002320D1002328D1002326C10093D6170160
:1005E0009307E7FF1305000063D0D7029307D701F5
:1005F000931506011356F60163DCD700370500801A
:100600001345F5FF3305A6001301010267800000C2
:10061000B707010093D50501B3E5F5009307F70689
:10062000B387D74013D75740232EB10093F7F70174
:100630006392070A93053000930601011315270002
:10064000B385E54063DEF502930740003387E7405A
:100650009306010193172700B387F6009306400025
:1006600023A007001307170093874700E31AD7FE5C
:1006700003250101E30A06F83305A0406FF0DFF817
:100680003388A60003280800938717009386460046
:1006900023AE06FF6FF01FFB832605FF032307FF32
:1006A000B39616013353F300B3E666002328D10056
:1006B00093061000E3C206FF13871600130501021C
:1006C00093962600B306D500B3D7F50023A8F6FE0F
:1006D0006FF01FF81305170093080102130830008C
:1006E000131525003308E8403385A80013172700A9
:1006F000930800021303010293060000B388F84038
:100700003307E3006FF01FFB130101FD2322910269
:1007100023261102232481022320210393040500B0
:10072000638605141384050013D9F50163D405000D
:100730003304B04013050400EF00007D9305150558
:10074000B74700009387E70113D75540232881005E
:10075000232A0100232C0100232E010093F5F5012B
:10076000B387A740638C050293062000631CD70E55
:1007700093060002B386B640B356D400232ED100B0
:100780009306F7FF13060102131727003307E6004D
:100790003314B400232887FE6F0040039306300013
:1007A000B386E6401306010293962600B306D600F0
:1007B00083A606FF13062000232ED10093062000F7
:1007C0006316C700232C8100930610001306010155
:1007D000139726003307E6001306F0FF23200700D7
:1007E0009386F6FF1307C7FFE39AC6FE0327C101EE
:1007F000B70601809386F6FF2316E10037870000D5
:100800001307F7FFB3F7E700139707018327C1002A
:100810001319F9018320C102B3F7D700B3E7E7004A
:10082000370700801347F7FFB3F7E70003270101FD
:1008300003248102B3E7270123A0E4000327410139
:1008400023A6F4001385040023A2E40003278101FA
:100850000329010223A4E4008324410213010103BC
:1008600067800000130730006FF09FF1232E010016
:10087000232C0100232A01002328010093070000F4
:10088000130900006FF09FF69357460137071000D9
:100890001307F7FF93F7F77F130101FC3377C700C6
:1008A00093861700232C8102232A9102232E110202
:1008B0009354F601232821032326310323244103E3
:1008C000232251032328B100232AE100232E010013
:1008D000232C010093F6F67F130610001304050085
:1008E000635CD60AB7460000938606C013D5450060
:1008F000B387D700935647001317C7013367A70084
:100900009395C501232ED100232CE100232AB100A9
:10091000232801000327C101B70601809386F6FF53
:100920002316E100378700001307F7FFB3F7E7004E
:100930000327C100939707019394F4013377D700FD
:10094000B367F700370700801347F7FFB3F7E700F7
:10095000B3E49700832701012326940013050400C4
:100960002320F400832741018320C1038324410312
:100970002322F40083278101032901038329C10273
:100980002324F40003248103032A8102832A4102E1
:1009900013010104678000003365B70063900710FE
:1009A000E30A05F66304070613050700EF00C055C8
:1009B000130A050093091A0313D9594093F9F90151
:1009C000638C09049305C0FF13050900EF0040463E
:1009D00093070002930A0101130600FFB387374112
:1009E0001305C5FF938ACAFF6318C5089307010260
:1009F0009306F9FF13192900338927018327010181
:100A0000B3993701232839FF6F000004EF00C04F6E
:100A1000130A05026FF01FFA9305C0FF13050900C2
:100A2000EF00004193090101930730003387A900CB
:100A30000327C7009387F7FF9389C9FF23A8E9001D
:100A4000E3D627FF9306F9FF9307010113972600CA
:100A50003387E7009307F0FF232007009386F6FF14
:100A60001307C7FFE39AF6FEB74700009387C7C096
:100A7000B38747416FF01FEA13070101B306A700D0
:100A800003A7C60083A606013357F700B3963601C5
:100A90003367D70023A8EA006FF09FF4B787000000
:100AA000630805029317C70193D64500B3E7D70043
:100AB000232CF10013574700B78700009395C50119
:100AC0003367F700232AB10023280100232EE10019
:100AD0009387F7FF6FF01FE48325C5008327850008
:100AE00003274500130101FE832605002324F1009E
:100AF000232CF100939705012322E100232AE10032
:100B000093D70701139715002326B1002320D100A6
:100B10002328D100232EF1001357170193D5F50197
:100B2000130301011306C101832706008326C6FFB4
:100B30001306C6FF9397370093D6D601B3E7D700C5
:100B40002322F600E312C3FE832601019307170058
:100B500013953600B78600009386F6FFB3F7D700EB
:100B60002328A1009306100063DCF61AB7C7FFFF25
:100B7000938707403307F7009307E07F63CEE71EB4
:100B80006358E006032881010326C1018327410140
:100B90009356C801131646003366D6009396470055
:100BA000B3E6A60093D7C70113184800B336D000A8
:100BB000B3E70701B3E6F600232AC1002328D100DA
:100BC000832601018327410113F67600630C061A80
:100BD00013F6F600130540006306A61A13864600B6
:100BE000B336D600B387D700930606006F0080198E
:100BF0009307C0FC635AF700232A01002328D10081
:100C0000130700006FF0DFFB8327C101B706080060
:100C100093080000B3E7D700232EF1009307D00319
:100C20003387E74013555740930703001377F701C5
:100C30009306000003A807009386160093874700D9
:100C4000B3E80801E318D5FE939E2600631A070255
:100C500093073000B387D74063D8E700930740007D
:100C6000B386D7406F0080063305D6010325050003
:100C70001307170013064600232EA6FE6FF0DFFDB4
:100C800093070102B387D70183A707FF1308000268
:100C90003308E840B3970701B3E8F8009307300042
:100CA000130E0000B387D7406348FE0413064000CC
:100CB000B306D6409397270013060102B307F60048
:100CC0000326C1013357E60023A8E7FE13074000BF
:100CD00093972600B307F30023A00700938616001E
:100CE000E398E6FE03270101B3371001B367F7006D
:100CF0002328F1006FF0DFF0330FD60103250F003A
:100D0000032F4F00130E1E003355E500331F0F0154
:100D10003365E5012320A600130646006FF0DFF8D7
:100D200003264101832781010328C101B366F60030
:100D3000B3E60601B3E6A60063180700B336D00099
:100D4000930700006FF05FE8638A060C9356C601B4
:100D5000131848001396470093D7C7013707400080
:100D6000B3E6C600B3E70701B3E7E70093F686FFF3
:100D70001307F07F6FF05FE5930700009306000014
:100D80001307F07F13968700635E060013071700B2
:100D90001306F07F6308C708370680FF1306F6FFC7
:100DA000B3F7C7001396D70193D63600B366D600C3
:100DB0001306F07F93D73700631EC700B3E6F60033
:100DC0009307000063880600B70708009306000039
:100DD00093050000370610001306F6FFB3F7C700AF
:100DE000370610801377F77F1306F6FF13174701B6
:100DF000B3F7C700B3E7E700370700801347F7FFF3
:100E00009395F501B3F7E70033E7B70013850600C4
:100E1000930507001301010267800000930700009B
:100E20006FF01FF693070000930600006FF09FF726
:100E3000130605001305000093F6150063840600F1
:100E40003305C50093D5150013161600E39605FE6D
:100E5000678000006340050663C60506138605002B
:100E6000930505001305F0FF630C060293061000BE
:100E7000637AB6006358C0001316160093961600E6
:100E8000E36AB6FE1305000063E6C500B385C540FE
:100E90003365D50093D6160013561600E39606FE6A
:100EA0006780000093820000EFF05FFB1385050070
:100EB000678002003305A04063D80500B305B04049
:100EC0006FF0DFF9B305B04093820000EFF01FF937
:100ED0003305A040678002009382000063CA0500CA
:100EE000634C0500EFF09FF7138505006780020053
:100EF000B305B040E35805FE3305A040EFF01FF600
:100F00003305B04067800200B7070100637AF5023D
:100F10009307F00FB3B7A7009397370013070002AA
:100F20003307F740B357F500171500001305C5F355
:100F3000B307F50003C507003305A740678000002D
:100F40003707000193070001E36AE5FC930780017E
:100F50006FF0DFFC130101FF232611002324810021
:100F6000930500001306000093060000130700001D
:100F7000930700009308900373000000130405001A
:100F8000635A050033048040EF00402E2320850083
:100F90001304F0FF130504008320C1000324810023
:100FA0001301010167800000130101F8232A910653
:100FB000232E110693840500232C810693058100BE
:100FC00013060000930600001307000093070000BB
:100FD000930800057300000013040500635A050020
:100FE00033048040EF008028232085001304F0FFA5
:100FF0001385040093058100EF0080201305040091
:101000008320C107032481078324410713010108BA
:1010100067800000130101FB9305410023261104A2
:10102000EFF09FF89307F0FF6308F50003258100B8
:101030001355D500137515008320C1041301010554
:1010400067800000130101FF232611002324810083
:101050009306000013070000930700009308E003C5
:101060007300000013040500635A05003304804038
:10107000EF00C01F232085001304F0FF13050400B8
:101080008320C10003248100130101016780000057
:10109000130101FF23261100232481009306000081
:1010A00013070000930700009308F003730000008B
:1010B00013040500635A050033048040EF00001B51
:1010C000232085001304F0FF130504008320C100D2
:1010D000032481001301010167800000130101FF57
:1010E0002322910097240000938404A483A7040082
:1010F0002320210123261100232481001309050048
:10110000639C07041305000093050000130600000C
:1011100093060000130700009308600D73000000A1
:101120001304050063560502EF00401433048040A9
:10113000232085001305F0FF8320C10003248100D4
:10114000832441000329010013010101678000008D
:101150009727000023AAA79C03A50400930500007D
:10116000130600003305A9009306000013070000D2
:10117000930700009308600D73000000130405003E
:10118000635A050033048040EF00400E23208500A1
:101190001304F0FF83A704001305F0FF3309F900DF
:1011A000E31C24F9172700002320879813850700E4
:1011B0006FF09FF8130101FF232611002324810003
:1011C0009306000013070000930700009308000433
:1011D0007300000013040500635A050033048040C7
:1011E000EF00C008232085001304F0FF130504005E
:1011F0008320C100032481001301010167800000E6
:1012000083A705002310F50083A785002311F500AF
:1012100083A705012322F50083A745012314F500C8
:1012200083A785012315F50083A7C5012316F500C3
:1012300083A705022317F50083A705032328F500DC
:1012400083A705042328F50283A785032326F50237
:1012500083A78504232AF50083A70505232EF5001F
:1012600083A785052322F5026780000097270000E9
:101270009387C78903A50700678000004D69616FE8
:10128000752021210000000068F3FEFFE404FFFF49
:10129000E404FFFF7CF3FEFFE404FFFFE404FFFF30
:1012A000E404FFFF1CF3FEFFE404FFFFE404FFFF80
:1012B00084F3FEFFA4F3FEFFE404FFFF9CF3FEFFB4
:1012C000ACF3FEFFE404FFFF10F4FEFF18F4FEFF92
:1012D00018F4FEFF18F4FEFF18F4FEFF18F4FEFFEA
:1012E00018F4FEFF18F4FEFF18F4FEFF18F4FEFFDA
:1012F000E404FFFFE404FFFFE404FFFFE404FFFF56
:10130000E404FFFFE404FFFFE404FFFF2CF8FEFF0A
:10131000E404FFFFACF4FEFF80F7FEFF2CF8FEFFB5
:101320002CF8FEFF2CF8FEFFE404FFFFE404FFFFAF
:10133000E404FFFFE404FFFF4CF4FEFFE404FFFFBE
:10134000E404FFFF7C01FFFFE404FFFFE404FFFF70
:10135000E404FFFF4802FFFFE404FFFF9402FFFFE5
:10136000E404FFFFE404FFFFC0F2FEFFE404FFFF1C
:10137000E404FFFFE404FFFFE404FFFFE404FFFFD5
:10138000E404FFFFE404FFFFE404FFFF2CF8FEFF8A
:10139000E404FFFFACF4FEFF84F7FEFF2CF8FEFF31
:1013A0002CF8FEFF2CF8FEFF54F4FEFF84F7FEFF3E
:1013B0009CF4FEFFE404FFFF80F4FEFFE404FFFF63
:1013C0001001FFFF8001FFFF1002FFFF9CF4FEFFF2
:1013D000E404FFFF4802FFFF7CF2FEFF9802FFFFDC
:1013E000E404FFFFE404FFFFFC02FFFFE404FFFF4F
:1013F0007CF2FEFF20202020202020202020202002
:10140000202020203030303030303030303030301C
:1014100030303030494E4600696E66004E414E0015
:101420006E616E00303132333435363738396162AF
:10143000636465660000000030313233343536377E
:101440003839414243444546000000003000000066
:10145000000000000000000000000000000000008C
:10146000000000000000000000000000000000007C
:10147000000000000080FF3F7665924A4A803F15D9
:101480004CC99A97208A025260C42575326A52CE9E
:101490009A32CE284DA7E45D3DC55D3B8B9E925AA6
:1014A0006C52CE508BF1283D0D65170C75818675F9
:1014B00076C9484D669CF85850BC545C65CCC691C2
:1014C0000EA6AEA019E3A3461E85B7EAFE981B90B0
:1014D000BBDD8DDEF99DFBEB7EAA51433502370162
:1014E000B1366C336FC6DF8CE980C947BA93A84127
:1014F000F850FB256BC7716BBF3CD5A6CFFF491FCA
:1015000078C2D340000000000000000020F09DB52C
:10151000702BA8ADC59D69400000000000000000D0
:10152000000000000004BFC91B8E34400000000012
:10153000000000000000000000000020BCBE1940B8
:10154000000000000000000000000000000000009B
:10155000409C0C4000000000000000000000000063
:101560000000000000C8054000000000000000006E
:10157000000000000000000000A00240FFFFFEFF8E
:10158000FCFFF8FFF0FFE0FFC0FF80FF00FF00FE60
:1015900000FC00F800F000E000C000800000000047
:1015A0003020FCCFC3A12381E32DDE9FCED2C8041F
:1015B000DDA6D80A6482CBD2EAF2D4122549E42D02
:1015C00036344F53AECE6B253FF598F6D36B5801AA
:1015D000A687BDC057DAA582A6A2B53231E7D404EA
:1015E000F2E332D332711CD223DB32EE49905A3906
:1015F0003EA20853FBFE551191FA39197A6325432F
:1016000031C0AC3C6DE2DEDB5DD0F6B37CACA0E477
:10161000BC647C46D0DD553E202A2462B347D7986F
:10162000233FA5E939A527EA7FA82A3F5B0BF24AA9
:1016300081A5ED18DE67BA943945AD1EB1CF943F50
:1016400071BFB3A9897968BE2E4C5BE14DC4BE94CD
:1016500095E6C93F4D3D3D7CBA362B0DC2FDFCCE13
:1016600061841177CCABE43F55C1A8A44E4013610F
:10167000C3D32B6519E25817B7D1F13F0AD7A3702E
:101680003D0AD7A3703D0AD7A3703D0AD7A3F83F00
:10169000CDCCCCCCCCCCCCCCCCCCCCCCCCCCCCCC89
:1016A000CCCCFB3F204E614E20000000202D496E27
:1016B00066696E697479200020496E66696E697486
:1016C000792000004E614E00452564004300000073
:1016D000504F5349580000002E0000000000000049
:1016E00005000000190000007D000000000000005F
:1016F000000000000000F03F000000000000244057
:1017000000000000000059400000000000408F4031
:10171000000000000088C34000000000006AF8409C
:101720000000000080842E4100000000D0126341C0
:101730000000000084D797410000000065CDCD4136
:10174000000000205FA00242000000E87648374217
:10175000000000A2941A6D42000040E59C30A242B5
:101760000000901EC4BCD64200003426F56B0C432A
:101770000080E03779C3414300A0D88557347643D1
:1017800000C84E676DC1AB43003D9160E458E14332
:10179000408CB5781DAF154450EFE2D6E41A4B44A7
:1017A00092D54D06CFF08044F64AE1C7022DB544EC
:1017B000B49DD9794378EA44BC89D897B2D29C3C8D
:1017C00033A7A8D523F649393DA7F444FD0FA53228
:1017D0009D978CCF08BA5B25436FAC642806C80A76
:1017E0000080E03779C34143176E05B5B5B893461D
:1017F000F5F93FE9034F384D321D30F94877825AE9
:101800003CBF737FDD4F15758859FFFF8C6BFFFF61
:101810008C6BFFFF9C59FFFF8C6BFFFF8C6BFFFFF6
:101820008C6BFFFF3459FFFF8C6BFFFF8C6BFFFF4E
:10183000A459FFFFC459FFFF8C6BFFFFBC59FFFF8A
:10184000CC59FFFF8C6BFFFF305AFFFF385AFFFF68
:10185000385AFFFF385AFFFF385AFFFF385AFFFF48
:10186000385AFFFF385AFFFF385AFFFF385AFFFF38
:101870008C6BFFFF8C6BFFFF8C6BFFFF8C6BFFFF94
:101880008C6BFFFF8C6BFFFF8C6BFFFFB45BFFFF6C
:101890008C6BFFFFD45AFFFF085BFFFFB45BFFFFB9
:1018A000B45BFFFFB45BFFFF8C6BFFFF8C6BFFFF34
:1018B0008C6BFFFF8C6BFFFF745AFFFF8C6BFFFF7D
:1018C0008C6BFFFF8465FFFF8C6BFFFF8C6BFFFF52
:1018D0008C6BFFFF5066FFFF8C6BFFFF3469FFFFCF
:1018E0008C6BFFFF8C6BFFFFD858FFFF8C6BFFFFEB
:1018F0008C6BFFFF8C6BFFFF8C6BFFFF8C6BFFFF14
:101900008C6BFFFF8C6BFFFF8C6BFFFFB45BFFFFEB
:101910008C6BFFFFD45AFFFF0C5BFFFFB45BFFFF34
:10192000B45BFFFFB45BFFFF7C5AFFFF0C5BFFFF64
:10193000C45AFFFF8C6BFFFFA85AFFFF8C6BFFFFA1
:101940001865FFFF8865FFFF1866FFFFC45AFFFF99
:101950008C6BFFFF5066FFFF9458FFFF3869FFFF55
:101960008C6BFFFF8C6BFFFF9C69FFFF8C6BFFFF95
:101970009458FFFF202020202020202020202020FD
:101980002020202030303030303030303030303097
:1019900030303030C878FFFFE880FFFFE880FFFF7D
:1019A000DC78FFFFE880FFFFE880FFFFE880FFFFB3
:1019B0007C78FFFFE880FFFFE880FFFFE478FFFF0F
:1019C000FC78FFFFE880FFFFF478FFFF0479FFFF5A
:1019D000E880FFFF6079FFFF6879FFFF6879FFFF0C
:1019E0006879FFFF6879FFFF6879FFFF6879FFFF7B
:1019F0006879FFFF6879FFFF6879FFFFE880FFFFE4
:101A0000E880FFFFE880FFFFE880FFFFE880FFFF3E
:101A1000E880FFFFE880FFFFE880FFFFE880FFFF2E
:101A2000E479FFFF047AFFFFE880FFFFE880FFFF13
:101A3000E880FFFFE880FFFFE880FFFFE880FFFF0E
:101A4000E880FFFFE880FFFFE880FFFFE880FFFFFE
:101A5000087BFFFFE880FFFFE880FFFFE880FFFFD3
:101A6000C47BFFFFE880FFFFA87EFFFFE880FFFF49
:101A7000E880FFFF2C78FFFFE880FFFFE880FFFF92
:101A8000E880FFFFE880FFFFE880FFFFE880FFFFBE
:101A9000E880FFFFE880FFFFE880FFFFE880FFFFAE
:101AA000E479FFFF087AFFFFE880FFFFE880FFFF8F
:101AB000E880FFFFA479FFFF087AFFFFD479FFFFDA
:101AC000E880FFFFC479FFFFE880FFFFA87AFFFFEF
:101AD0000C7BFFFF947BFFFFD479FFFFE880FFFFC3
:101AE000C47BFFFFF877FFFFAC7EFFFFE880FFFFBE
:101AF000E880FFFF087FFFFFE880FFFFF877FFFF28
:101B000020202020202020202020202020202020D5
:101B100030303030303030303030303030303030C5
:101B200000202020202020202020282828282820AD
:101B300020202020202020202020202020202020A5
:101B4000208810101010101010101010101010100D
:101B500010040404040404040404041010101010FD
:101B600010104141414141410101010101010101C7
:101B70000101010101010101010101011010101019
:101B80001010424242424242020202020202020299
:101B900002020202020202020202020210101010ED
:101BA0002000000000000000000000000000000015
:101BB0000000000000000000000000000000000025
:101BC0000000000000000000000000000000000015
:101BD0000000000000000000000000000000000005
:101BE00000000000000000000000000000000000F5
:101BF00000000000000000000000000000000000E5
